:020000040800F2
:10000000002000107D160308C9A202089DC1000847
:10001000C7A20208C5A20208C3A20208000000008D
:10002000000000000000000000000000C1A2020863
:10003000BFA2020800000000BDA2020839DA0008D1
:10004000E5160308E5160308E5160308E516030898
:10005000E5160308E516030889150108B516010819
:10006000791601083D16010801160108351F000820
:10007000251F0008151F0008051F0008F51E0008B1
:10008000E11E0008CD1E0008E5160308E51603086A
:10009000E5A30208E5160308E5160308C5150108DF
:1000A000B1D10008E1D10008A1D10008F1D10008C8
:1000B000D1D10008C1D10008E5160308E5160308F0
:1000C000E5160308E5160308E5160308E516030818
:1000D000E516030855030108D90201085D0201086D
:1000E0004D150108E5160308ADA20208E516030840
:1000F000E5160308E5160308E5160308E5160308E8
:10010000000000000000000000000000E5160308E9
:10011000E5160308E5160308393301081D33010805
:10012000B91E0008A51E0008911E00087D1E0008CB
:10013000691E0008E516030800000000000000002A
:10014000E5160308E5160308E5160308000000009D
:10015000000000000000000000000000000000009F
:100160000000000000000000E5160308E516030883
:10017000E516030800000000000000000000000079
:0801800000000000E516030871
:10018800002870B51EDB0928044620DD012303EB97
:1001980083035B00B0FBF3F2092AF8D87BB10E4E5B
:1001A800B4FBF3F00928CCBF57223022A6FB03E5A5
:1001B800024403FB1044EB0801F8012BF0D10023A3
:1001C8000B7070BD2D230B7040420131DBE73030DE
:1001D80001F8010BF3E700BFCDCCCCCC884230B49A
:1001E8004FF001042ED301FB04F4B0FBF4F58D426B
:1001F800F9D284B1AAB901E0B0FBF4F5092DCCBF5E
:10020800572230222A4404FB150003F8012BB4FBC3
:10021800F1F4002CF0D100221A7030BC7047B0FB0A
:10022800F4F5092DCCBF372230222A4404FB1500EF
:1002380003F8012BB4FBF1F4002CF0D100221A7062
:1002480030BC70470546002AEBD1D7E703685A1C33
:1002580002601970704700BF2DE9F047089C2578A7
:10026800002B804689460CBF4FF0200A4FF0300A19
:10027800661C35B3002A29DD334601E0024698B1F1
:1002880013F8011B501E0029F8D1971E60B13D4696
:10029800013D51464046C8476B1C002BF8DC2578C9
:1002A80027EAE770013055B1041B29464046C84784
:1002B800301916F8015B002DF7D1BDE8F087BDE8CD
:1002C800F087002A04DC2846BDE8F0870020EBE729
:1002D800571EDCE783684268D0ED037A00EB8301A0
:1002E8000133934281ED040A836004BF00238360D5
:1002F80000EB830393ED047A036870EE277A9A4241
:10030800C0ED037A77EEC77AC0ED037A0CDA0133D1
:1003180007EE103AF8EEC76AB7EE007A87EEA60A3B
:10032800036030EE070A704707EE102AB8EEC77A66
:1003380087EE870A704700BF90ED057A90ED004A76
:10034800D0ED066AD0ED014AD0ED047A90ED035A5B
:10035800D0ED025AA4EE007AB0EE406AB0EE470A39
:10036800B0EE667AA6EE247A67EEC07AA0EE457AF9
:10037800E6EE257A80ED057AC0ED067A704700BF73
:10038800D0ED057A90ED013AD0ED003AD0ED064A6D
:1003980090ED024A90ED077A90ED035A90ED086AC5
:1003A800D0ED045AC0ED067AF0EE406A27EE830AD3
:1003B800C0ED056AA3EEA60A80ED087AA4EE240A29
:1003C800A5EE470AA5EEC60A80ED070A704700BFEA
:1003D800D0ED007A90ED017A30EE670AE7EE007A08
:1003E800B0EE670AC0ED007A704700BF704700BFE3
:1003F8000A44914214D030B40139551E41F2210209
:1004080011F8014F082380EA042004044CBF82EA53
:1004180040004000013B80B2F7D18D42F0D130BCA2
:10042800704700BF4FF4805383827047012380F8E0
:100438004530704790F8203033B1012B03D14FF489
:1004480000638382704770474FF4806383827047EC
:1004580070B40468037B2268022101FA03F31A428C
:1004680013D042690A495C2000FB02124FF6FE765F
:1004780050685289C5680068296831402960C16898
:10048800D24392B20A40C260636070BC704700BF3A
:100498008C4D002030B40A4B1D7875B1094B0020F3
:1004A80003EBC5051A6899885062D4682143D16066
:1004B800083323F8040CAB42F4D130BC704700BFBA
:1004C8006C5000207050002010B40268047B116842
:1004D8000223A340194209D00649406800240C7041
:1004E80001684FF6FE742140016053605DF8044BCB
:1004F800704700BF7D380020014B18680FF0D4BF4B
:100508000C210020F0B5836983B0054613B11A6841
:100518009B8813856869264F8389C3244FF47A73AF
:100528004FF0060E6E464FF6FF71013703E0013BB0
:100538009BB28B421DD002899207F8D504734FF401
:100548007A7302E0A3B28B4213D00289D20703F177
:10055800FF34F7D5027BD2B20EB132700136BEF14C
:10056800000F08D00EF1FF3EFF24002FE3D03C78A7
:10057800DBE711F003F9AB6913B11A689B88936143
:100588009DF805009DF801609DF802109DF8034054
:100598009DF804209DF8063041EA062143EA00232D
:1005A80042EA0422012029876A87AB8703B0F0BD9D
:1005B800302B030810B490E80600047B406902233E
:1005C800A3404B6013685DF8044B4FF6FE710B4077
:1005D80013600FF0F9BEF8B5174D2B78A52B28D16D
:1005E8006B78BE2B25D1022229464FF6FF70FFF704
:1005F800FFFE124FAC1C22884AB1A618BE4218D280
:10060800052A16D92146FFF7F3FE3446F3E72146BB
:100618000222FFF7EDFE0222A118FFF7E9FE0634D9
:10062800074B641B1C8041F60F53C31A58425841AC
:10063800F8BD0020F8BD00BF00F003080000040862
:100648000E2D00202DE9F04FDFF848914C4F8BB06C
:100658000326A7EB09071822002104A832F0F5F9B0
:10066800484BCDF8109005971A69120604D5464AEA
:100678005A6002F188325A6001228DF8242034220F
:10068800DA60424B424C1B88ADF8003002226946C2
:1006980004A811F0A7F9022269464FF6FF70FFF788
:1006A800A7FEDFF8F4A080464FF0000B544536D380
:1006B8000AAC002524F8245D0222214604A811F082
:1006C80091F9022221464046FFF792FE40BAC04304
:1006D800ADF80800022202A904A811F083F90798CE
:1006E80060B106ABC0F104022946184432F0ADF9F6
:1006F800069904A811F01CF9079508909DF8243074
:10070800089A23B11F490B6943F080030B61013E2E
:100718002DD0002A9FD1FFF75EFF50B32CE06588EB
:100728008DF80DB0C5F30B05AB1DADF80830238867
:10073800C3F30B02ADF80A201B0B062202A904A87A
:100748008DF80C3011F04EF9062202A94046FFF749
:100758004FFE616880462A4604A811F043F9616893
:1007680040462A46FFF744FE143480469EE7002A96
:10077800D1D005200BF04EFD0BB0BDE8F08F00BFC7
:10078800000004080020024023016745372B0308B6
:10079800A088030800F00308008D03080378202BC5
:1007A800024600F10100F9D0092BF7D02D2B2CD0EF
:1007B8002B2B03BF5378B7EE000A0246B7EE000AA8
:1007C800A3F13001C8B209289FED467A10D8F2EE9D
:1007D800046A07EE901AF8EEE77A12F8013FE7EE9E
:1007E800267AA3F13001C8B20928B0EE677AF0D9A9
:1007F8002E2B4CD003F0DF03452B0BD0F7EE007AFD
:1008080067EE276A20EE260A70475378BFEE000A83
:100818000246D5E710B451782D2959D02B290ABFA3
:100828009178501C901C0024A1F13003092B53D857
:10083800002303EB830301EB430310F8011FA1F12D
:100848003002092AA3F13003F3D9B3F59A7F28BF00
:100858004FF49A73072B42D9DFED236A1A46F7EE55
:10086800007A083A072A67EEA67AFAD803F007034F
:100878002BB1F2EE046A013B67EEA67AFBD124B3F2
:10088800C7EE276A5DF8044B20EE260A70475378B6
:10089800A3F13001C8B2092802F10102AAD8F2EE88
:1008A800046AF0EE665A07EE901AF8EEE77A12F844
:1008B800013F87EEA66AA3F13001C8B2092866EEA7
:1008C800A56A37EE067AEED994E767EE276AD9E784
:1008D800901C91780124A7E7F7EE007ACFE7F7EEAE
:1008E800007AC5E70000000020BCBE4CB5EEC00A87
:1008F800DFED317AF1EE10FACCBF30EE270A30EE98
:10090800670ADFED2E7A20EE270A30B5FDEEC07AB1
:1009180087B017EE904A054684EAE470002303A9DD
:10092800A0EBE4700193009302932FF05FF9002C81
:10093800ACBF20232D2303A88DF8003030F01CF81D
:10094800012803A924D002282DD0032805BF30236D
:10095800684668468DF8013032F07FF8684630F016
:100968000BF80338C4B222466946284632F0ACF880
:1009780000232B5528462FF0FFFF2E22431C2A5414
:100988000DEB0401E81832F085F8284607B030BDB1
:10099800302368468DF801308DF802308DF8033029
:1009A80032F05BF8DAE7302368468DF801308DF8CD
:1009B800023032F052F8D1E76F12033A00007A445D
:1009C8002DE9F041064615460846B6FBF2F43CB957
:1009D80005FB1464124B1B5D00F8013BBDE8F08178
:1009E800B4FBF2F767B90E4B05FB174705FB146418
:1009F800DA5D00F8012B1B5D00F8013BBDE8F081D2
:100A0800B7FBF2F8B8F1000F02D04046FFF7D8FF65
:100A180005FB1878024B13F8082000F8012BE3E7D0
:100A2800B45803082DE9F04714461D46064600232E
:100A38004FF47A722046294630F048FCDFF84881A6
:100A48004B4A4C4F88FB00310144C31782FB002EF0
:100A5800C3EB611188FB012887FB00278644464ABF
:100A6800C3EBEE2EC1EB011C82FB0E29A0EB8C0C14
:100A78000744424A86F806C0C3EB27474FEAEE7C94
:100A880008EB010ACCEBA90C82FB07824FEAE1785C
:100A98000CEB4C0CC8EB6A18AEEBCC0EC8EB081884
:100AA800DFF8E8C086F804E0A1EB880171718CFBDF
:100AB8000010F917C1EBE21240F2B55101FB1272B6
:100AC800C3EBE050B2F5896F4FEA80073FDA40F296
:100AD800DA239A4243DCB2F5B77FB4BF4FF0000C7B
:100AE8004FF0010C4FEA4C08254B08EB0C0103EBC7
:100AF800C1031FFA8CFE588C224908EB0C0301EB4A
:100B0800C30116310B2301E031F8020D82421BDAD2
:100B1800013BF9D11A4BC44403EBCC0C0123BCF8BC
:100B28000C00B37007F2B2770132121ABE44F270A9
:100B3800A6F800E0204629464FF47A72002330F0E8
:100B4800C5FB3281BDE8F0870133DBB2E9E74FF03E
:100B5800030EF44640F296504FF00608CCE74FF0EB
:100B6800020EF44640F229404FF00408C4E700BFE3
:100B7800C5B3A29107452EC2ABAAAA2A73B06D16B7
:100B8800302B03083C2B030889888888792D0311AA
:100B9800104B2DE93048D3E9004554EA05020BD142
:100BA8000346012200201871587198719A70DA7002
:100BB80018801881BDE83088074B1A6814EB020BBF
:100BC80045F1000C5A466346FFF72CFF0120BDE8AB
:100BD800308800BFD01D0020EC640020F0B40288EB
:100BE8008578164FC37804794179A2F2B27202F07F
:100BF800030606EB4606013D05EB860507EB4505B2
:100C0800013BAE898579008940F2B557920807FB08
:100C18000232931903EB430304EBC303C3EB03133F
:100C280001EB8303C3EB031305EB830300214FF4AC
:100C38007A72C2FB0301F0BC704700BF302B030877
:100C4800FAB170B48E18044603E0101A14D1B142F8
:100C580014D014F8012BA2F14103192B11F8013B10
:100C6800A3F1410598BF2032192D03F12000ECD9DA
:100C7800D01A01D1002BEAD170BC7047002070BC9B
:100C880070471046704700BF4FF0FF32FFF7D8BFDC
:100C9800A0F16103192B98BF20387047A0F14103D8
:100CA800192B98BF20307047202805D00938042810
:100CB8008CBF002001207047012070476138192837
:100CC8008CBF002001207047413819288CBF0020B4
:100CD80001207047303809288CBF00200120704758
:100CE800A0F13003092B07D920F02000413819283A
:100CF8008CBF0020012070470120704730B4026883
:100D08001146531C036011F8024B0160D31C517843
:100D180003609378151D05601B0443EA0123D0780E
:100D2800234343EA006030BC704700BF0368591C86
:100D38001A46016012F8021B0260587841EA002046
:100D4800704700BF03685A1C02601878704700BFDC
:100D580038B504460068154630F07CFD22682A4400
:100D6800226038BD036810B40A0A5C1C04601A705B
:100D780003685A1C026019705DF8044B704700BF85
:100D880003685A1C026010B4197003680A0A5C1CD4
:100D980004601A7003680A0C5C1C04601A7003680B
:100DA800090E5A1C026019705DF8044B704700BFA9
:100DB80003685A1C026019700368090A5A1C026009
:100DC800197070472DE9F047002488B080460F4617
:100DD8001E46A14605AD531C0393117839B3252946
:100DE80033D1931CCDF810900393507830284ED00F
:100DF8004FF0000AA0F13003DBB2092B42D96C286E
:100E080019D0642800F0938024D825281CD063D9F1
:100E1800582876D063281BD131784046B847039AC2
:100E2800531C03931178043601340029D7D1204686
:100E380008B0BDE8F087039B5A1C03921B78642B0B
:100E48007CD02AD8252B54D1252140460134B847D7
:100E5800039AC0E7732833D044D975284FD106F1D7
:100E6800040E30682B4600220A217646FFF7B6F9B1
:100E7800049A0095534639464046FFF7EDF9039A20
:100E88000444A8E704AA03A92EF0F8FDB7E7D31C89
:100E9800039390784FF0010AACE7732B10D05BD91D
:100EA800752B3AD0782B96D1A3F15802B2FA82F278
:100EB800306852092B4610210436FFF78FF9D7E71F
:100EC8003368049A0093394600234046FFF7C4F973
:100ED80004360444039A7EE70028B9D1204608B0B6
:100EE800BDE8F0876E28B3D1039A336804361C60D6
:100EF80071E72AD9582BD7D0632B8DD06BE7782888
:100F0800A6D1A0F15802B2FA82F2306852092B46F3
:100F18001021FFF763F90436AAE706F1040E3068DA
:100F28002B4600220A217646FFF758F9A0E7331D21
:100F3800306829461E46FFF723F999E7331D3068C4
:100F480029461E46FFF71CF992E7002B7FF443AFB2
:100F5800204608B0BDE8F0876E2BC6D03BE700BF3F
:100F68000EB400B584B005AB019053F8042B0649C4
:100F7800039301A8FFF726FF019B00221A7004B013
:100F88005DF804EB03B07047550200080FB430B5A4
:100F980083B006AB0A490B4853F8042B096800686C
:100FA8000193FFF70FFF084C054620680FF06CFA15
:100FB8000028FAD0284603B0BDE8304004B0704796
:100FC800442C0020482C00200C210020DFED2B7A37
:100FD800B4EEE70AF1EE10FA4ADDDFED296A9FED7B
:100FE800297A01E0B0EE670AB4EEC70AF1EE10FA0A
:100FF80070EE667AF6DC9FED247AF4EEC77AF1EEAD
:1010080010FA38D5DFED1E6A9FED207A01E0F0EE88
:10101800407AF4EEC77AF1EE10FA37EEA60AF6D463
:10102800DFED1B7AB4EEE70AF1EE10FA14DDDFED1E
:10103800137A37EEC00A60EE006A9FED166A9FEDDC
:10104800167ADFED167AA6EE867A20EE266AE6EEA6
:10105800877AA6EE270A7047DFED117AB4EEE70A21
:10106800F1EE10FA44BFDFED087A37EEC00AE2E786
:10107800F0EE407ABFE7B0EE670AD1E7DB0F4940F0
:10108800DB0FC940E4CB1641DB0F49C0E4CB16C1E6
:10109800DB0FC93F92E741B99730083C15A82ABE33
:1010A800DB0FC9BF09B909E0194690FBF1F301FB51
:1010B80013030846002BF7D1084670470146FBE7A3
:1010C80007EE901AF8EE677A9FED837A27EE800A8A
:1010D80020EE070AFDEEC07A17EE903A2033402B37
:1010E80000F28C80DFED7D7AB4EEE70AF1EE10FABB
:1010F80040F3E880B0EE407A9FED796ADFED796AD7
:1011080001E0B0EE677AB4EEE67AF1EE10FA77EE27
:10111800467AF6DC9FED747AF4EEC77AF1EE10FAAF
:1011280040F1CD809FED6E6ADFED706A01E0F0EE70
:10113800477AF4EEE67AF1EE10FA37EE867AF6D4CC
:10114800DFED6B7AB4EEE77AF1EE10FA51DCDFED01
:10115800697AB4EEE77AF1EE10FA44BFDFED627A0D
:1011680037EEC77A27EE076ADFED635ADFED637A59
:10117800DFED636A9FED635AE6EE257A67EE065A5D
:10118800E6EE276AF7EE007AA5EEA67AF0EE675A41
:10119800E7EE055AE7EE457A87EEA55ADFED547A71
:1011A80030EE277AFDEEC76A16EE903A2033402BD0
:1011B80029D99FED557AF6EE006AB7EE006AF7EE88
:1011C800004AC4EEA57A0023836143610362C361C8
:1011D80080ED045A67EEA66A27EE866A27EE877ABC
:1011E800C0ED006AC0ED026A80ED016A80ED037A05
:1011F8007047DFED3A7A37EEC77AB3E7B7EE005AB1
:10120800F0EE455ACAE7B4EEE70AF1EE10FA5FDDF0
:101218009FED336ADFED336A01E0B0EE677AB4EE32
:10122800E67AF1EE10FA77EE467AF6DC9FED2E7A42
:10123800F4EEC77AF1EE10FA47D59FED296ADFED93
:101248002B6A01E0F0EE477AF4EEE67AF1EE10FA56
:1012580037EE867AF6D4DFED267AB4EEE77AF1EE49
:1012680010FA27DCDFED237AB4EEE77AF1EE10FA14
:1012780044BFDFED1D7A37EEC77A27EE076ADFED48
:101288001E4ADFED1E6ADFED1E7AE6EE246A67EE7F
:10129800064AE6EE267AB7EE006AA4EEA77AF6EEDC
:1012A800006A36EE476AF8EE007A27EE277A66EE8D
:1012B800266A84E7DFED097A37EEC77ADDE7B0EE14
:1012C800677A3DE7F0EE407A24E7B0EE677AC2E746
:1012D800F0EE477AAAE700BF27D4D236DB0F4940A1
:1012E800DB0FC940E4CB1641DB0F49C0E4CB16C184
:1012F800DB0FC93FDB0FC9BF92E741B99730083C04
:1013080015A82ABEF304353F0000008070B40668B3
:101318008E4217D90139751E002311F8014F082292
:10132800634013F0800F4FEA430318BF83F0D503DF
:10133800013ADBB2F5D18D42EFD1721C02603370F5
:1013480070BC70470023F8E710B44C09012250F82C
:10135800243001F01F0102FA01F10B4340F8243058
:101368005DF8044B704700BF4B0901F01F0150F8AE
:101378002320012303FA01F1114214BF184600206B
:10138800704700BF074A084B10781B78074A83420A
:1013980096BFC31AC3F18003002012681844104492
:1013A800704700BF085F0020845E00206051002065
:1013B800064A074B10781B7883428ABFC3F1800323
:1013C800C01AC018C0F17F00704700BF085F002036
:1013D800845E0020F8B584894FF6FF764FF47A745E
:1013E8002BB311B30F78013101E0B44217D005894E
:1013F800013CAD07A4B2F8D507734FF47A7402E044
:10140800BCB2B4420BD00589ED0704F1FF37F7D51C
:10141800057BEDB20AB115700132013BE0E710F02F
:10142800ADF9003018BF0120F8BDFF27DFE7012024
:10143800F8BD00BF30B5134C237883B01BB9012029
:10144800237003B030BD1049052200230D688DF8C4
:1014580004208DF8053000BFA86810F00FF86A4620
:1014680001A902236868FFF7B5FFA86810F00CF817
:1014780000BF9DF8013003F0010383F001002370E1
:1014880003B030BDA75800209458002070B5064C12
:101498000646256803E023685B1BB34203D8FFF7C1
:1014A800C9FF0028F7D070BDEC640020F0B51F4CD0
:1014B80083B0277800234FF0030E00930E4615469D
:1014C8008DF804308DF800E06FB3030E8DF801300D
:1014D8000DF10203010C020A9870197006205A7067
:1014E800FFF7D4FFE8B100BF114F3B6898680FF0D1
:1014F800C5FF23783A68002B14BF052304236946E7
:1015080050680022FFF766FF3B68324600215868A2
:101518002B46FFF75FFF3B6898680FF0B5FF00BFE9
:10152800284603B0F0BD0DF10103D3E7A65800200B
:101538009458002008B540F2E93300E09BB10289D5
:10154800013B12F0020F9BB2F8D0017340F2E9336D
:1015580000E043B10289013B12F0010F9BB2F8D0C1
:10156800007BC0B208BD10F009F9C0B208BD00BFC9
:1015780038B504460D4600BF80680FF07FFF294646
:101588006068FFF7D7FFA0680FF07EFF00BF38BD87
:101598002DE9F04F89B0B2F1000A0290049103934B
:1015A80040F3C5800B46002201EB8A0153F8040B77
:1015B8008B420244FAD1039B0592002B00F0AF80C6
:1015C800059B002B7CD05E4B059A1B68DFF8889141
:1015D80000920099DAB25118B1F5807F8CBFC2F53C
:1015E8008072009A0192574A92689A4240F2828029
:1015F800554A1178002206928DF81C2002228DF897
:101608001820002960D01A0E8DF819200DF11A0241
:101618001C0C190A9370147051700620FFF736FFDE
:101628000621D9F80000FFF7A3FF484A01231370E9
:1016380000BFD9F8003098680FF020FF424BD9F866
:1016480000201B785068002B06A90CBF0423052333
:101658000022FFF7BFFE0024049D029E019FA346BF
:1016680029684FEA840800220B46013471B1B94257
:101678002DD2D9F8000031684068FFF7ABFE2A6820
:10168800336813443360BF1AC5F800B0A24505F1AA
:10169800040506F10406E3D1D9F8003098680FF084
:1016A800F3FE00BF264B019900981B68421A00926E
:1016B800234A0B441360039A4AB3009A002A88D13C
:1016C800059809B0BDE8F08F0DF11902A0E7029C5A
:1016D800D9F8003054F80810586800223B46FFF744
:1016E80079FE54F808202B683A44DF1B44F8082098
:1016F8002F60D1E70598009C1549164A001B0590F4
:10170800059800230B70137009B0BDE8F08F059B96
:10171800009A9B1A0593059809B0BDE8F08FFFF76A
:1017280089FE00287FF44CAF039B0593C8E7039C10
:101738001CB9FFF77FFE0594C2E700230593BFE7B6
:101748006051002060190020A6580020A7580020EA
:10175800085F0020845E00209458002070B5104D6A
:10176800104E2B7831788B4284B016D00E4A0392F3
:101778001A4402928CBF0C46CA1A04A98CBFC3F142
:1017880080020024012341F8102D02A802220194AE
:10179800FFF7FEFE002333702B7004B070BD00BF4E
:1017A800845E0020085F0020885E0020F0B5124BA0
:1017B8009D6885B00DB905B0F0BDED0A14D00027BD
:1017C80004AE7C196410E00210226946FFF76EFE31
:1017D8000F2809DD6B4653F8042B01320AD1B342B6
:1017E800F9D12546AF42ECDBFFF7B8FF034BED021A
:1017F8001D60E0E7671CF5E76019002060510020D4
:1018080070B5194C194D23782978994284B027D09E
:10181800174A03921A44029234BF0E46CA1A04A900
:1018280034BFC3F180020026002341F8102D02A81E
:1018380002220196FFF7ACFE23781844C0B20306D3
:101848002B7848BF80F080008342207002D00020AF
:1018580004B070BD002301202B70237004B070BD4C
:10186800012004B070BD00BF845E0020085F002026
:10187800885E002010B50C4C45F20820FFF706FEE4
:1018880020680621FFF774FE084B20680122C72153
:101898001A70FFF76DFE06480649074A00230370D1
:1018A8000B70136010BD00BF94580020A75800208B
:1018B800085F0020845E002060510020F0B55B4B7B
:1018C8005B4A97B01968914200AF00F0A38059496C
:1018D800594A00234FF47000C1F888003B607B60D0
:1018E800136843F48033136003E03B68B3F5A04FFB
:1018F80009D0136803F400337B603B6801333B6015
:101908007B68002BF1D04C4B1B6813F4003318BFD5
:1019180001237B607B68012B52D0464C464B474ADB
:10192800E260474A596A11605A6A42F080725A6204
:101938005A6942F4FC025A610025032207F10801A2
:10194800012341F6FF764FF09040FD60BE603A7388
:10195800BB7319F0B5FD4FF6FF7307F1080139485D
:10196800BB6019F0ADFD07F108013748374E19F093
:10197800A7FD07F10801364819F0A2FD07F1080193
:10198800344819F09DFD07F10801334819F098FD16
:1019980007F1080019F0EEFDBB683049304AA1FB99
:1019A800031330499B0CF0204FF0070E5C370B6097
:1019B800566084F823009560C2F800E0BD46F0BD8B
:1019C800294A1D4B122111605A685A605A685A6098
:1019D8005A6842F480625A605A6822F47C125A604B
:1019E8005A6842F4E8125A601A6842F080721A6023
:1019F8001A689201FCD559680F4A21F00301596011
:101A0800596841F002015960536803F00C03082B30
:101A1800FAD182E700221A6062B6144B1B6883F37E
:101A28000888134B1B689847FEE700BFFC9F0020FF
:101A3800EFBEADDE00ED00E0001002400005FA0543
:101A48000066002000040048000800483F19010013
:101A5800000C0048001000480014004883DE1B43B7
:101A680010E000E0F06400200020024000D8FF1FD2
:101A780004D8FF1F70B50F4C0F4DC0EBC00004EB2E
:101A88008004686926693043686182B09209667B80
:101A9800A1600025012101A863618DF804608DF81B
:101AA80005208DF806508DF8071019F0D3FC02B008
:101AB80070BD00BF041A002000100240074BC0EBA5
:101AC800C00030B403EB8000054C056963692B4303
:101AD80063610176427630BC704700BF041A00206B
:101AE800001002402DE9F04F5E4C54F8204083B0BE
:101AF800002C71D0A66D984691465B4B72682265A2
:101B0800A160236004F15E014FF4807304F5AF72A5
:101B18006161A261E36023610746307E2BF034FEE9
:101B2800F068A8B1514B00215A68904203F11C0398
:101B380000F0928001310C29F6D100207A1CD2B233
:101B48000C21FFF7BBFF236DF26862632433E36463
:101B5800B068D8B1454B00215A68904203F11C0384
:101B680078D001310C29F7D100257A1CD2B20B218B
:101B78002846FFF7A3FF2346F27E3D492846FFF794
:101B880079FF236DB268A2632833A36494F85D00DB
:101B98000FF022F8054694F85C000FF01DF818F0D5
:101BA800080F824696F819B01AD0CDB118F0110F67
:101BB8004FF00B0307F1010714BF4E213E21EF71CF
:101BC8005A46AB7128460FF0CBF818F0010F45D0F4
:101BD800636B5BB3A36B4BB3204603B0BDE8F08FD8
:101BE80018F0010F0CBF4FF02E084FF04E0819F0F7
:101BF800020F09D045B10B227B1CAA71EB71284654
:101C08005A4641460FF0ACF819F0010FE0D0BAF18E
:101C1800000FDDD001370C238AF807705A46414679
:101C28008AF8063050460FF09BF8D1E7337FB27E32
:101C38008DF804209B090021012201A88DF80530A8
:101C48008DF806108DF8072019F004FC204603B023
:101C5800BDE8F08FCDB288E7C8B26FE728460FF02D
:101C68000DFCB5E7502C00209C2B0308041A00201B
:101C7800BD05000800B97047F0B595B005462CF0D1
:101C880021F96E4EC368026832600446002B00F0EA
:101C9800C38028460EF0A0FF694B186018B12922AE
:101CA80000238271C371227A664D2E210FF058F8F5
:101CB80030680BF009FC2BF067FD3068624A038836
:101CC80023F001031B041B0C038014A91E232B8083
:101CD80001270F230025138021F84C7D2D23029323
:101CE800ADF80C50ADF80650ADF80E502CF098F841
:101CF800E379ADF8145060229907ADF816500695AF
:101D0800ADF81C50ADF81E50ADF82050ADF822507B
:101D1800049200F1838013F0010F14BF0222002205
:101D28004FF48073ADF81470ADF81C20ADF8203076
:101D3800002304AA6179306806930BF033F8306801
:101D480061792CF04DF83068436C43F400434364E8
:101D580003889BB243F080030380E3799B0768D52F
:101D68006179026A04238B4022EA03020262026A52
:101D7800134303623268354F13889BB243F0010363
:101D88001380207C00222921FFF798FE3049207C0F
:101D980000236022FFF76EFEE068386019F0C6FA8B
:101DA800386803684FF6FE721340036019F0BEFAF4
:101DB80009A819F08DFA33686279264938680A91BA
:101DC80034331344099380221023002509A940F2D3
:101DD8002A3E0E920B934FF400724FF400530D9568
:101DE8001095139511950F921293ADF830E019F0F4
:101DF8007DFA627933680C2A98BF1749D86898BF6A
:101E080031F812503A6815490543DD60136801201E
:101E180043F002031360087015B0F0BD13F0010F12
:101E280014BF08222A460423ADF81E20ADF8163048
:101E38007EE70122617919F089F99BE7445800206F
:101E4800781D00203A5800203858002040580020BB
:101E5800D1040008143A0020B44C03083C58002070
:101E68000348D0F83C3113B100F59A701847704711
:101E7800041A00200348D0F8203113B100F58C7003
:101E880018477047041A00200348D0F804310BB1F2
:101E9800FC301847704700BF041A00200348D0F8E8
:101EA800E8300BB1E0301847704700BF041A002033
:101EB8000348D0F8CC300BB1C4301847704700BF86
:101EC800041A00200348D0F8B0300BB1A8301847E6
:101ED800704700BF041A00200348D0F894300BB1B3
:101EE8008C301847704700BF041A00200248836FDF
:101EF8000BB1703018477047041A00200248C36DB0
:101F08000BB1543018477047041A00200248036C7C
:101F18000BB1383018477047041A00200248436A4A
:101F28000BB11C3018477047041A00200248836818
:101F380003B11847704700BF041A0020F0B53E4CA3
:101F4800059D00EB800004EB80046468002C71D0D0
:101F58003A4E49004FF42040CFB27060A16909049D
:101F680054D46068DFF8E0E047F4903100EA0E00EE
:101F780001434FF420406160706003E0411E002877
:101F880048D00846A1698907F8D54FF42040A262D5
:101F9800706003E0421E00283CD01046A269520639
:101FA800F8D5274A6168DFF8A0E0706042EA03428A
:101FB800174301EA0E0217436760C3B1013BDBB266
:101FC80001332B44A0694FF4204210F0040002F1C1
:101FD800FF3207D1511C26D0A06910F0040002F18D
:101FE800FF32F7D0626A05F8012B9D42EAD14FF41F
:101FF8002040706002E0431E60B11846A3699B064A
:10200800F9D520237060E3610120F0BD411E08B1BD
:102018000846A3E70B4A138801339BB24FF0FF3100
:1020280013807160F0BD074972600B8801339BB261
:102038000B80F0BD2046F0BD5C640020781D0020B8
:10204800002400020C2D0020009800FC2DE9F04F20
:1020580089B090F855300490002B40F06782534BBC
:102068001B7A002B00F0A480049B103305931846BC
:1020780004994A69138823F040031B041B0C13803E
:1020880013889BB223F0380343F038031380138876
:102098009BB243F04003138091F84E201A210FF0B1
:1020A8007FFB0BF081FB04460BF07EFB8442FBD0E8
:1020B800049A5069038823F040031B041B0C038017
:1020C800038823F038031B041B0C038003889BB28E
:1020D80043F040030380137C012B4CD0022B1346A2
:1020E8005BD1936913B11A689B88138540F2E93371
:1020F80002E0002B00F0C9820289013B12F0020FB6
:102108009BB2F6D0C323037340F2E93302E0002BFD
:1021180000F0BB820289013B12F0010F9BB2F6D09E
:10212800037B049B58690627838906AD4FF47A73AD
:102138004FF6FF714FF0FF0E04E0013B9BB28B425C
:1021480000F07A8202899207F7D580F80CE04FF404
:102158007A7303E0A3B28B4200F06E820289D6073D
:1021680003F1FF34F6D5027BD2B20DB12A700135E6
:10217800013FE7D162E292F914001346421C0CD0E9
:1021880002280ADC597D06AB009343220623FFF799
:10219800D5FE002840F05882049BB3F93A305BB270
:1021A800013300F0178209B0BDE8F08F781D0020D8
:1021B8000499BC4C4A69BC4F1388DFF8F8A223F095
:1021C80040031B041B0C138013889BB223F03803B5
:1021D80043F03803138013889BB243F04003103157
:1021E80013800591084680226B210FF0D9FA9623B7
:1021F800AE48DFF8C4C24FF010084FF47A759E4617
:10220800DAF80430C3F30803002B40F07381EFF3CE
:102218001183002B40F06E812168826800BF23681B
:102228009942F9D13E6805FB06F39B1AB3FBF6F316
:1022380005FB013101260391DAF80430C3F30803E2
:10224800002B40F01181EFF31183002B40F00C813B
:102258002368816800BF22689342F9D1D7F800B09B
:1022680005FB0BF2521AB2FBFBF205FB0323039AA0
:102278009B1AB3F57A7FDFD3BEF1010EC0D10322DA
:1022880068210598DFF82CA20FF08AFA9623874870
:10229800DFF824C24FF010084FF47A759E46DAF83A
:1022A8000430C3F30803002B40F00881EFF31183D7
:1022B800002B40F003812168826800BF236899429F
:1022C800F9D13E6805FB06F39B1AB3FBF6F305FB51
:1022D800013101260391DAF80430C3F30803002B17
:1022E80040F0A580EFF31183002B40F0A080236815
:1022F800816800BF22689342F9D1D7F800B005FB86
:102308000BF2521AB2FBFBF205FB0323039A9B1A4A
:10231800B3F57A7FDFD3BEF1010EC0D103226B2162
:1023280005980FF03DFA0BF03FFA04460BF03CFA23
:10233800001B0E28FAD910226A2105980FF030FAEE
:102348000BF032FA04460BF02FFA001B0E28FAD9CC
:1023580000226C2105980FF023FA0BF025FA0446A9
:102368000BF022FA001B0E28FAD9049B059893F863
:10237800502019210FF014FA0BF016FA04460BF04E
:1023880013FA001B0E28FAD918221B2105980FF002
:1023980007FA0BF009FA04460BF006FA001B0E28A0
:1023A800FAD910221C2105980FF0FAF90BF0FCF964
:1023B80004460BF0F9F9001B0E28FAD91022372130
:1023C80005980FF0EDF90BF0EFF904460BF0ECF976
:1023D800001B0E28FAD90122382105980FF0E0F9E0
:1023E8000BF0E2F904460BF0DFF9001B0E28FAD9CE
:1023F800049B5A69138823F040031B041B0C1380A9
:10240800138823F038031B041B0C138013889BB21A
:1024180043F0400313800BF0C7F904460BF0C4F9EE
:102428008442FBD0224A05980123137220E6EFF379
:10243800118988F3128881680368DB0344BFCCF8EC
:10244800006081682368DCF800205FFA89F989F365
:102458001188D7F800901A4405FB09F35B1AB3FBFF
:10246800F9F305FB023351E7EFF3118988F312887A
:1024780081680368DB0344BFCCF800608168236887
:10248800DCF800205FFA89F989F31188D7F8009001
:102498001A4405FB09F35B1AB3FBF9F305FB023396
:1024A800E5E600BFEC640020F064002010E000E0E6
:1024B800781D002000ED00E0E8640020EFF31182B1
:1024C80088F3128886680368D90303D50123CCF8FA
:1024D800003086682368DCF80010D2B282F31188D5
:1024E8003A68194405FB02F39B1BB3FBF2F305FBA7
:1024F8000131EEE6EFF3118288F3128886680368EB
:10250800D90303D50123CCF8003086682368DCF8AA
:102518000010D2B282F311883A68194405FB02F31D
:102528009B1BB3FBF2F305FB013183E61D09013D5B
:10253800052D03F00F0300F29F805D4A32F8150065
:1025480040FA03F2D40740F19780012404FA03F318
:10255800013B18402EF00AFF564B574A5B5D184462
:1025680012EBC00500F0888000232021EB71A971CF
:1025780052F83000514A00F138439B0AD25C02F00D
:102588001F035209022A04FA03F300F08B80032A7E
:1025980000F08380A2427BD0AB88069306A9002373
:1025A800079318F08DFF0499454B41F80C3F2846D6
:1025B80023F0E0F8AB88B3FA83F3C3F11F03581C88
:1025C8003FF44DAD012202FA03F33E490A68134372
:1025D8000B6044E5049B93F9383001337FF4E3AD95
:1025E8000A26322022F094FD4FF4FA750BF0DCF83D
:1025F80004460BF0D9F8001BB0F57A7FF9D3013DFA
:10260800F4D107202BF0BEFC4FF47A750BF0CCF810
:1026180004460BF0C9F8001BB0F57A7FF9D3013DE9
:10262800F4D1013EDDD12849284B2948294A0860C0
:10263800DA6009B0BDE8F08F0FF0A0F8049B9B6941
:1026480013B11A689B8893619DF818409DF81A5039
:102658009DF81B309DF819109DF81C009DF81D2051
:1026680041EA042143EA0523049C1BB242EA002202
:1026780063872187A28792E50499114B41F80C3FA3
:10268800002023F077F801239FE70FF077F848E55B
:10269800114A51690B4353617EE70F4AD1690B43D5
:1026A800D36179E70C4A91690B43936174E700BFE2
:1026B800904C03089C4C030890470020B45403082E
:1026C8003504000800040140FC9F002000ED00E0F4
:1026D800EFBEADDE0400FA0500100240F0B5037C41
:1026E800012B85B0044663D0022B67D1836913B1EF
:1026F8001A689B881385606940F2E93301E0002B72
:102708006CD00289013B12F0020F9BB2F7D0C323B1
:10271800037340F2E93301E0002B5FD00289013BEB
:1027280012F0010F9BB2F7D0037B60694FF0060EE1
:10273800838902AE4FF47A734FF6FF71FF2703E0E7
:10274800013B9BB28B423CD002899507F8D50773B1
:102758004FF47A7302E0ABB28B4232D00289D207CF
:1027680003F1FF35F7D5027BD2B20EB132700136D4
:10277800BEF1010EE8D1A36913B11A689B88936171
:102788009DF80C009DF808609DF809109DF80A5006
:102798009DF80B209DF80D3041EA062143EA0023FD
:1027A80042EA0522012021876287A38705B0F0BD90
:1027B80090F91400431C01D0022805DD002005B063
:1027C800F0BD0EF0DBFFD6E702AB617D009343223C
:1027D8000623FFF7B3FB0028D2D1EFE70EF0CEFFB8
:1027E800A3E700BFF0B5037A012B85B0044663D098
:1027F800022B67D1036913B11A689B881385E068B7
:1028080040F2E93301E0002B6CD00289013B12F061
:10281800020F9BB2F7D0BB23037340F2E93301E008
:10282800002B5FD00289013B12F0010F9BB2F7D059
:10283800037BE0684FF0060E838902AE4FF47A738B
:102848004FF6FF71FF2703E0013B9BB28B423CD060
:1028580002899507F8D507734FF47A7302E0ABB293
:102868008B4232D00289D20703F1FF35F7D5027BBC
:10287800D2B20EB132700136BEF1010EE8D1236931
:1028880013B11A689B8893619DF80C009DF8086045
:102898009DF809109DF80A509DF80B209DF80D3001
:1028A80041EA062143EA002342EA05220120E182A7
:1028B8002283638305B0F0BD90F90C00431C01D05E
:1028C800022805DD002005B0F0BD0EF057FFD6E761
:1028D80002AB617B00933B220623FFF72FFB002806
:1028E800D2D1EFE70EF04AFFA3E700BFB0F1FF3FF8
:1028F80056D0022854DCF0B4324C00EB800004EBD4
:1029080080004468002C5BD02F4E49004FF42040D3
:10291800CDB27060A169090444D460682B4F45F0BA
:102928008071384041F4903101434FF42040616098
:10293800706003E0411E002838D00846A1698F075F
:10294800F8D54FF42040A262706002E0421E68B3DE
:102958001046A2691106F9D562681C4945F0007550
:1029680045F480350A4015434FF420406560706097
:1029780002E0421ED0B11046A2699207F9D54FF481
:102988002040A362706002E0431E78B11846A36934
:102998009B06F9D520237060E3610120F0BC7047E5
:1029A80000207047411E08B10846B3E7084A13885B
:1029B80001339BB24FF0FF3113807160F0BC704758
:1029C8002046FBE75C640020781D0020009800FC8E
:1029D8000C2D00202DE9F04F87B090F8553002906B
:1029E800002B40F0C281029A137C1032012B104652
:1029F800039200F01182022B00F0B281BD4CBE4E52
:102A0800DFF8FC92BD48DFF8FCE24FF0640A4FF0B3
:102A1800100C4FF47A75D9F80430C3F30803002B6F
:102A280040F0F380EFF31183002B40F0EE80216833
:102A3800826800BF23689942F9D1376805FB07F31C
:102A48009B1AB3FBF7F305FB013101270191D9F874
:102A58000430C3F30803002B40F09D80EFF311838B
:102A6800002B40F098802368816800BF2268934259
:102A7800F9D1D6F800B005FB0BF2521AB2FBFBF203
:102A880005FB0323019A9B1AB3F57A7FDFD3BAF1CA
:102A9800010AC0D1029D297C012900F0B4810229D4
:102AA80000F04A81029B012993F8503000F05081D0
:102AB800022900F03B81DFF848929048DFF844E2B1
:102AC8004FF00F0A4FF0100C4FF47A75D9F8043014
:102AD800C3F30803002B40F0B480EFF31183002BFD
:102AE80040F0AF802168826800BF23689942F9D11D
:102AF800376805FB07F39B1AB3FBF7F305FB0131B6
:102B080001270191D9F80430C3F30803002B5FD1E2
:102B1800EFF31183002B5BD12368816800BF226823
:102B28009342F9D1D6F800B005FB0BF2521AB2FB6A
:102B3800FBF205FB0323019A9B1AB3F57A7FE1D3D5
:102B4800BAF1010AC2D1029C237C94F84E20012BD1
:102B580000F06B81022B00F0D780012B00F0DC80A5
:102B6800022B00F0B280012B00F0B980022B00F09C
:102B78009880012B00F09F80022B7ED0012B00F063
:102B88008680022B04D10398012238210EF008FE1A
:102B980007B0BDE8F08FEFF311888CF312888168D5
:102BA8000368DB0344BFCEF8007081682368DEF851
:102BB80000205FFA88F888F31188D6F800801A4454
:102BC80005FB08F35B1AB3FBF8F305FB023359E77F
:102BD800EFF311888CF3128881680368DB0344BF24
:102BE800CEF8007081682368DEF800205FFA88F864
:102BF80088F31188D6F800801A4405FB08F35B1A9D
:102C0800B3FBF8F305FB023395E7EFF311828CF37E
:102C1800128887680368D90303D50123CEF80030EA
:102C280087682368DEF80010D2B282F31188326810
:102C3800194405FB02F3DB1BB3FBF2F305FB01317F
:102C480003E7EFF311828CF3128887680368D903CE
:102C580003D50123CEF8003087682368DEF800101A
:102C6800D2B282F311883268194405FB02F3DB1BE8
:102C7800B3FBF2F305FB013142E71A46372103980B
:102C88000EF08EFD029B1B7C012B7FF47AAF02981D
:102C98003822417D90F91400FFF728FE07B0BDE8FF
:102CA800F08F18221C2103980EF07AFD029B1B7CE2
:102CB800012B7FF461AF029C02233722617D94F9D6
:102CC8001400FFF713FE237C58E718221B210398F2
:102CD8000EF066FD029B1B7C012B7FF447AF029C24
:102CE80018231C22617D94F91400FFF7FFFD237C53
:102CF8003FE700BFEC640020F064002010E000E033
:102D080000ED00E0E86400201A2103980EF048FD69
:102D1800237C012B7FF424AF029C18231B22617DA6
:102D280094F91400FFF7E2FD237C1CE71A461921E9
:102D380003980EF035FDBEE66B21032203980EF0D2
:102D48002FFD297C029B012993F850307FF4B0AE07
:102D580002981922417D90F91400FFF7C7FDAAE6F1
:102D680080226B210EF01CFD48E61D09013D052D52
:102D780003F00F0367D83D4A32F8150040FA03F212
:102D8800D40760D5012404FA03F3013B18402EF060
:102D9800EDFA374B374A5B5D184412EBC00552D049
:102DA80000232021EB71A97152F83000324A00F15A
:102DB80038439B0AD25C02F01F035209022A04FA24
:102DC80003F34ED0032A47D0A24237D0AB880493EE
:102DD80004A90023059318F073FB0299274B41F8C7
:102DE8000C3F284622F0C6FCAB88B3FA83F3C3F144
:102DF8001F02501C3FF4F7AD01239340204A11688D
:102E08000B431360EFE5697D95F9140003236B22EA
:102E1800FFF76CFD297C45E602988023417D90F9F7
:102E280014006B22FFF762FDE8E51346617D94F913
:102E380014001A22FFF75AFD237C8EE6114A5169C5
:102E48000B435361C2E702990C4B41F80C3F002039
:102E580022F090FC0123D1E70A4AD1690B43D361E0
:102E6800B4E7084A91690B439361AFE7904C0308B4
:102E78009C4C030890470020B4540308350400080C
:102E880000040140001002401749184B184A19481D
:102E980010B4D1F8884044F47004C1F888401C6824
:102EA80044F001041C605C6822405A601A6822F0F1
:102EB800847222F480321A601A6822F480221A601E
:102EC8005A6822F4FE025A60DA6A22F00F02DA62C5
:102ED8001A6B002410404FF0006218639C608A60EF
:102EE8005DF8044B704700BF00ED00E000100240A1
:102EF8000CC07FF8CCFC00FF2DE9F04F95B0B0F97D
:102F080008500D81EDB2442D00AF0C46904600F0FC
:102F18001684064632D9812D00F05D8300F2868042
:102F2800542D00F0B38040F2BD806E2D00F0D583A3
:102F3800802D40F0B9806A4B1D780B3D15F0FF05D8
:102F480014D0DFF8C4E100220A262168BEF8003058
:102F5800481C20600E702168FF2B02F10102A8BFF7
:102F6800FF23481CAA4220600B70EEDB01252B468C
:102F7800284654376381BD46BDE8F08F052D00F023
:102F8800CC831FD8022D79D040F20483032D00F0A2
:102F98009B83042D40F08880524920462A46FDF73D
:102FA800D7FE00212046FDF703FF22680021531CAD
:102FB8000125236028462B46543711706381BD468E
:102FC800BDE8F08F242D57D040F29A82282D00F0CA
:102FD8003D83382D68D10A68434B0125511C216077
:102FE80015702268052150192060117022680A2185
:102FF800501920601170226800215019206011704A
:10300800226819785019206011702268597850196F
:103018002060117022689978531923602B4611702B
:10302800284654376381BD46BDE8F08FA02D11D0E6
:1030380040F28582B82D00F04583FE2D34D12B4D0A
:1030480005F1080635F8021B2046FDF7B1FEB5422A
:10305800F8D18BE7264B08461968FDF791FE254BFA
:1030680020461968FDF78CFE234B19682046012578
:10307800FDF786FE2B467BE7204BF6E70422204926
:1030880020460125FDF764FE2B46C9E70B680021A1
:103098005A1C2260197022680125531923602B4697
:1030A8001170BDE7522D80D0214628460EF008FD4C
:1030B800034600287FF45AAF742D00F07E82772DE6
:1030C80024D13268716891421EBF531C3360117855
:1030D8000C4A08BF1946204613F06AFB46E700BFB2
:1030E8006E3F00207E4200206B330020C43F00204A
:1030F800ACF7FF1FB0F7FF1FB4F7FF1FB434002071
:10310800DC580308C95701086C240020F52D01F08C
:10311800AD82472D00F04083292D326801F0668288
:10312800392D01F05082212D01F02D8270680B3D60
:10313800811AEF2D00F28E840FF2040E5EF825F04E
:103148000D4000085D3A00085D3A00085D3A000845
:103158005D3A00085D3A00085D3A00085D3A0008EB
:103168005D3A00085D3A00085D3A00085D3A0008DB
:103178005D3A00085D3A00085D3A00085D3A0008CB
:103188005D3A00085D3A00085D3A00085D3A0008BB
:103198005D3A00085D3A00085D3A00085D3A0008AB
:1031A800993F00085D3A0008773F00085D3A00083B
:1031B8004D3F00085D3A00085D3A00085D3A000896
:1031C800134100085D3A00089D4000085D3A000878
:1031D8006B4000085D3A0008454000085D3A000869
:1031E8003B3F00085D3A0008E33E00085D3A0008EE
:1031F800913E00085D3A00085D3A00085D3A000813
:103208005D3A0008752F00085D3A0008173E00086F
:103218005D3A00085D3A0008934300085D3A0008EB
:10322800394300085D3A00085D3A00085D3A000835
:103238005D3A00082D4300085D3A00085D3A000831
:103248005D3A0008ED4200085D3A00089F42000818
:103258005D3A00085D3A00085F4200085D3A0008E0
:103268005D3A00085D3A00085D3A00085D3A0008DA
:103278005D3A00085D3A0008F14100085D3A00082F
:103288003B4100085D3A00085B4400085D3A0008CD
:10329800AD4300085D3A00084D450008F93D0008B7
:1032A800DD3D00085D3A00085D3A00085D3A000817
:1032B8005D3A00085D3A00085D3A00085D3A00088A
:1032C8005D3A00085D3A00085D3A00085D3A00087A
:1032D8005D3A00085D3A00085D3A00085D3A00086A
:1032E8005D3A00085D3A00085D3A00085D3A00085A
:1032F8005D3A00085D3A00085D3A00085D3A00084A
:103308005D3A00085D3A00085D3A00085D3A000839
:103318005D3A00085D3A00085D3A00085D3A000829
:103328005D3A00085D3A00085D3A00085D3A000819
:103338005D3A00085D3A00085D3A00085D3A000809
:103348005D3A00085D3A00085D3A00085D3A0008F9
:103358005D3A00085D3A00085D3A00085D3A0008E9
:103368005D3A00085D3A00085D3A00085D3A0008D9
:103378005D3A00085D3A00085D3A00085D3A0008C9
:103388005D3A00085D3A00085D3A00085D3A0008B9
:103398005D3A00085D3A00085D3A00085D3A0008A9
:1033A8005D3A00085D3A00085D3A00085D3A000899
:1033B8005D3A00085D3A00085D3A00085D3A000889
:1033C8005D3A00085D3A00085D3A00085D3A000879
:1033D8005D3A00085D3A00085D3A00085D3A000869
:1033E8005D3A00085D3A00085D3A00085D3A000859
:1033F800B33D00085D3A0008973D00086D3D0008A0
:103408005D3A00085D3A00085D3A00085D3A000838
:103418005D3A00085D3A00085D3A00085D3A000828
:103428005D3A00085D3A00085D3A00085D3A000818
:103438005D3A0008F33C00085D3A0008BB3C000810
:103448005D3A0008193C0008FF3B0008513D0008A0
:103458005D3A0008E53B00085D3A0008BD3B0008FE
:103468005D3A00085D3B00085D3A0008053B00082E
:103478005D3A00085D3A0008A93A00087B3A00085E
:10348800673A0008353B00083F3A0008153A00083B
:103498005D3A00085D3A00085D3A00085D3A0008A8
:1034A8005D3A00085D3A00085D3A00085D3A000898
:1034B8005D3A00085D3A00085D3A00085D3A000888
:1034C8005D3A00085D3A00085D3A00085D3A000878
:1034D800F53900085D3A00085D3A00089D39000892
:1034E8005D3A00085D3A00085D3A0008393900087D
:1034F8005D3A00085D3A00085D3A00081F39000887
:10350800202D7FF4D1AD0B68914D591C6A7821604C
:103518001A7023682A78591C21601A702368AA78BF
:10352800591C21601A7029892046FDF741FC23683F
:103538006A79591C21601A702268A97937E5822DA9
:103548007FF4B2AD0B68834A834D1178804A581CCA
:103558002060197011892046FDF72AFC7F4B2268EC
:103568001B88FF2B02F10101A8BFFF232160137004
:10357800A96881F3100189B22046FDF719FC296872
:1035880001F30F0189B22046FDF712FC744B226843
:1035980019780CE5012D7FF487AD0B680022591CC2
:1035A80021601A7023685A1C22601D702268252128
:1035B800531C23602B46117032E5326871689142C2
:1035C8001EBF531C33601178664A08BF194620464F
:1035D80013F0EEF8CAE4644B1E780A3E16F0FF06B4
:1035E8003FF4C4AC614BDFF8A8811E4403F1010924
:1035F8000A2314E0502B00F0B987002529462268D9
:10360800501C206020461370FDF7D2FB2946204647
:10361800FDF7CEFBB1453FF4A9AC19F8013B0A2BE5
:10362800E8D1534A9568116805EB85054FF6FF7296
:103638006D009542A8BF15469142A8BF114625EADC
:10364800E57521EAE171ADB289B2D8E70B68DFF818
:103658004491484E591C022221601A7023684FF089
:1036680006085A1C226083F8008023680A22591C25
:1036780021601A70236801255A1922601D70B9F853
:1036880000102046FDF794FBB9F802102046FDF71C
:103698008FFB23685A19226083F800802368502220
:1036A800591921601A7023680022591921601A706B
:1036B80031882046FDF77CFB71882046FDF778FBB2
:1036C8002B46ADE42C4BD0E40B685A1C0A601D70E5
:1036D8000B685A1C0A601D7067E4204B0A681B8837
:1036E8001D4DFF2BA8BFFF23511C21601370A96833
:1036F80081F3100189B22046FDF75AFB1F4B204683
:103708001988FDF755FB296801F30F0189B2204696
:103718000125FDF74DFB2B4682E40B221849204674
:10372800FDF716FB082217492046FDF711FB012576
:10373800072215492046FDF70BFB2B4670E4002AAB
:103748003FF414AC114B136001252B4668E400BF0D
:10375800A4410020E63F0020B4410020D03F0020D3
:10376800A8380020295801086E3F0020C42B030800
:10377800282400205C24002040450020A438002094
:10378800E4580308F0580308FC5803089D1A010878
:1037980060240020BC600020726835687B62304677
:1037A800551BFDF7ABFA052D38627B6A00F2DD8701
:1037B8008026B346012594E80600521A103AB24210
:1037C800B8BF1FFA82FBC14A396A92683A61521A35
:1037D8009345396A7B622046FA6088BF1FFA82FBEC
:1037E800FDF7CEFA7B6A002B00F09D87002D40F094
:1037F80016872368C7F800D05D71C0B00533C7F8D5
:1038080008D0FB61BBF1000F01F060803B6A3A69A8
:10381800934281F05780AA463E6A7D627C6080258B
:103828005446FB681C1BA94BB4F5807F28BF4FF496
:1038380080749B6832199A4288BF9C1BFDF78EFFE3
:103848002246BC6830462146FDF730FEF969B8616A
:1038580004EB000C0B787B61644530D2DFF8909262
:103868000CF1FF3C04F1FF3E1EF8013F09EB830217
:1038780019F823405688FCB100234FF4004204F1A4
:10388800FF3816424FEA520202D0087828430870DF
:103898006D0806D10AF1010A4D701FFA8AFA013142
:1038A8008025D34505D8E645C0F06686984500F3DF
:1038B800638601339C42E4D1E645D5D1F9617B6A40
:1038C800BA6913449BB2DA457B6206D27B6A3A6ACC
:1038D8001C46D6183B699E42A3D37C68802D1CBF2A
:1038E8000AF101031FFA83FA0AF1020189B220469C
:1038F800FDF75EFA2368796A01255A192260204685
:103908001D70FDF755FA2368534423602B46D7F8FA
:1039180000D0FFF785BB6E4B1B78DB0700F19A8060
:10392800012508F06DFC08F047FE2B46FFF778BB31
:103938003046FDF7FBF93368B8851A46591C3160E3
:1039480012F8021B326087F82E105A7887F82F2059
:10395800DA1C32609A7887F830201A1D3260DA78DB
:1039680087F831205A1D32601B7987F8323007F109
:103978002C000023BB86FDF731F9564A564B1268D6
:10398800801A4FF0010561F10001C3E904012B46DB
:10399800FFF746BB531C336013780F2B5AD8911C82
:1039A8003160C3EBC3034D495078C854D01C306014
:1039B8000B4491785970111D3160D1789970511D5F
:1039C80031601179D970911D316051791971D11D0A
:1039D80031609179597102F108013160D2799A7197
:1039E80001251FF087F82B46FFF71ABB3046FDF775
:1039F8009DF9DFF80081A8F80E003046FDF796F92A
:103A08000125A8F80C002B46FFF70ABB3046FDF746
:103A18008DF9DFF8E480A8F810003046FDF786F944
:103A2800A8F812003046FDF781F90125A8F814001E
:103A38002B46FFF7F5BA1346511C316013F8020BF9
:103A48003360D31C51783360927817F0B5F80028AA
:103A58007FF48CAA4FF0FF352B46FFF7E1BA204BD5
:103A6800204918684E2201252DF0F4FE2B46FFF759
:103A7800D7BA1146531C33601B4B11F8020B187050
:103A8800316051785970D11C316092789A70304603
:103A9800FDF74CF9154B0125D8802B46FFF7C0BA26
:103AA8003046FDF743F9DFF84480A8F800003046B7
:103AB800FDF73CF9A8F802003046FDF737F9012573
:103AC800A8F804002B46FFF7ABBA00BF6019002026
:103AD800673E0020EC640020C01D002054440020F4
:103AE80018420020204E0308C46000209857002088
:103AF800C82B0308CC600020644D0020DFF87493C5
:103B080099F80030002B3FF431AADFF86C830025C8
:103B18003046FDF70BF91FF041FD99F80030A8EC8D
:103B2800010A01359D42F3DBFFF720BA1346511C09
:103B38003160C24913F8020B08703360C0495378EA
:103B48008B70D31C3360BF4B92789A7001252B463B
:103B5800FFF766BA0D297FF47DAF531C33601578E3
:103B6800072D3FF677AFDFF8149330464FF00C0877
:103B7800FDF7DCF808FB05F809EB0805A8803046D6
:103B8800FDF7D4F8E8803046FDF7D0F8336828818F
:103B98001A46591C316012F8021BA97232605B7810
:103BA800EB723046FDF7AAF8012549F808002B46C4
:103BB800FFF736BA531C33601078060600F1778693
:103BC800A14B1B78DD073FF5D1A9032828BF0020AA
:103BD800012508F0F9FA2B46FFF722BA9A4B1B7811
:103BE800D8073FF5C3A9012509F0D0F808F0E4FC8F
:103BF8002B46FFF715BA944B1B78D9073FF5B6A9A2
:103C0800924B4FF4C87201251A802B46FFF708BA69
:103C180009297FF71FAFDFF868821346511CD8F8CF
:103C28000050316013F8021B297033605378AB7071
:103C3800D31C33609378642B02F10401A8BF64237A
:103C48006B713160D378642B02F10501A8BF64233E
:103C5800AB7131601379EB71931D33605379642B29
:103C680002F10701A8BF64232B7231609379EB70CE
:103C780002F108033360D3792B713046FDF756F80B
:103C8800726833686881D11A00290CDD591CD8F88C
:103C980000003160521A002A1978417203DD9A1C1B
:103CA80032605B78437001252BF04AF92B46FFF709
:103CB800B7B9674B1868D31C014621329D1E356081
:103CC80013F8035C0D705D1E356013F8025C4D70CF
:103CD800336013F8015C8D700333934201F10301E3
:103CE800ECD11FF02BFBFFF741B9C1F34705122DAB
:103CF8003FF6B0AEC5B107F1500307F12A0903EB4F
:103D0800450AC846AAF1260A3046FDF70FF828F8F2
:103D1800020FC245F8D14F4B39F8022F23F8022F72
:103D2800C145F9D1112D09D84B4A6B00023B134408
:103D38000021223223F8021F9342FBD1474A012374
:103D48001D461370FFF76CB93F4B1B78DA073FF538
:103D58000DA9434A1378012543F0040313702B4639
:103D6800FFF75EB9531C3F48336001781378002988
:103D780040F0D185042202703B4A9B00138009F071
:103D880013FD3A4B012598612B46FFF749B9DFF837
:103D9800F48000233046C8F80030FCF7AFFF012557
:103DA800C8F800002B46FFF73BB91346511C316099
:103DB80013F8025B3360D31C507833609178002D80
:103DC80000F0D085012D7FF4D1A80FF0BFFA2B4663
:103DD800FFF726B9531C33601378002B00F0A08539
:103DE8004FF4004001250EF07DFE2B46FFF718B971
:103DF800154B1B7813F001017FF42CAE531C336074
:103E0800107801250FF0E4F92B46FFF709B913469E
:103E1800511C3160164913F8025B8D703360557878
:103E28004D7083423FF4A2A8D31C33600F4B9278A5
:103E38001A7201252B46FFF7F3B800BFC8480020C7
:103E4800CC600020DC600020673E002086650020F2
:103E5800184200203A6100203C6100206061002087
:103E6800845100205A5C0020A4380020C01D002086
:103E7800EC6000206E3F0020142D002094430020A9
:103E88001C420020404500200723B1FBF3F3C3EB9D
:103E9800C305491B7FF4DEADDBB203F1FF395FFADE
:103EA80089F9002B3FF462A8DFF808A309F101099A
:103EB8000D46531C336092F90010BE4B4FF00008BA
:103EC80093F902208A4203F1080300F07B8408F189
:103ED8000108B8F1060FF3D1BCE5531C3360137821
:103EE8000E2B3FF6B7AD911C31605578032D3FF688
:103EF800B1ADB148062101FB03F1431802F1030EED
:103F08005D71C6F800E095784554111D3160D1788F
:103F18005970511D316011799970911D3160517935
:103F2800D970D11D316092791A7101252B46FFF79E
:103F380077B8531C3360A14B12785A7501252B466C
:103F4800FFF76EB83046FCF7F1FEDFF89082C8F84C
:103F580000003046FCF7EAFEC8F804003046FCF7DB
:103F6800E5FE0125C8F808002B46FFF759B8DFF829
:103F780070820023C8F800303046FCF7BFFED8F83E
:103F8800003001250343C8F800302B46FFF748B836
:103F9800511C316015783B62132D3FF65BAD911CC7
:103FA800316050787A6212F03DFC00283FF452AD3F
:103FB8007A6A8349007801F82500D01C306001EB4B
:103FC800850590786870101D3060D078A870501DF5
:103FD80030601279EA7001F150003B6A02E0043166
:103FE800884207D00A78002AF9D18D78CA78954294
:103FF800F5D20123734A83F00103012513702B4680
:10400800FFF70EB8704810294FF000020B4628BF82
:104018001023026042608260C2600274002B3EF48A
:10402800A5AF3268411E13440132326012F8010C08
:1040380001F8010F9A42F7D1FEF798BF531C33607D
:1040480015781F2D3FF606AD05297FF403AD3046E0
:10405800FCF754FE5D4B43F8250019F0EDFCFEF724
:1040680085BF5A4D05F140083046FCF75FFE3368BE
:10407800A5F88000591C1A46316012F8021B85F811
:10408800821032605B7885F883300435A845EBD11F
:10409800FEF76CBF531C494D336013782B723046C2
:1040A800FCF744FEA8833046FCF740FE28833046E0
:1040B800FCF73CFE32686883531C33601278EA745C
:1040C8007268D31A032B00F306843368D11A0529C2
:1040D8000EDD5A1C32601B78EB723046FCF70EFE80
:1040E8003368E8605A1C32601B782B743368726836
:1040F800D21A002A7EF73AAF5A1C32601B7885F82C
:10410800213001252B46FEF78BBF531C3360304905
:1041180015780D70C01A00287EF728AF931C3360FD
:104128005378003318BF012301254B702B46FEF747
:1041380077BF1346511C3160DFF8A88013F8021BC3
:1041480088F802103360234953780B70D31C33600E
:10415800214D93782B71131D3360D378092BA8BF99
:1041680009233046AB70FCF7E1FD3368726828809C
:10417800D11A012905DD3046FCF7D8FD336872688D
:10418800E8819A4207D05A1C32601B78003318BF66
:10419800012388F8073008F071F9336872689A4289
:1041A8003EF4E4AE5A1C32601B78EB7001252B46B6
:1041B800FEF736BF9C5900204C450020705900205E
:1041C800B06200209C1B0020A86000206C360020F4
:1041D80078510020C0600020644D00207C2C002015
:1041E800B4340020C8480020C84B1B68002B3EF49C
:1041F800BDAE20F08FFBFF283EF4B8AE3046FCF78A
:1042080095FD3F2840F2B483DFF82883002588F81D
:10421800005033687268A8F80400D21A012A7EF7A1
:10422800A5AE1A46591C316012F8021B88F8021014
:1042380007F15000326000225D7800F8242D20F04C
:104248003BFB97F82C30AB423EF490AE284620F06A
:1042580057FBFEF78BBEAE4B1B78012B3EF686AEA6
:10426800531C11463360DFF8D08211F8023B88F8FE
:104278000230D31CC01A3160012892F801E0336083
:1042880040F385833046FCF751FD0125A8F800006E
:104298002B46FEF7C5BE531C336092F80080B8F178
:1042A800110F3FF6D7AB931C33609A4D537805F83E
:1042B80018303046FCF73AFD40F6CA039842A8BFCA
:1042C800184640F2EE23984205EB4801B8BF18465D
:1042D8000125A0F2EE222B46192092FBF0F24A703B
:1042E800FEF79EBE1346511C8B4D316013F8021B1E
:1042F8002971336053786B713046FCF717FD3368CA
:1043080028805A1C32601B78AB713046FCF70EFDD2
:10431800336868805A1C32601B78EB7101252B4684
:10432800FEF77EBE0125FDF7A5FA2B46FEF778BEFF
:10433800531C3360794B1278DFF800821A7000231F
:10434800C8F800303046FCF7D9FC3368D8F80020AC
:104358007349744D10435A1CC8F8000032601B782A
:104368000B723046FCF7E2FC28603046FCF7DEFCB6
:1043780068603046FCF7DAFCA8603046FCF7D6FCEB
:104388003046FCF7D3FCFEF7F1BD674B02F108019C
:104398000132326012F8010C03F8010F9142F7D193
:1043A800FEF7E4BD3046FCF7C1FC3046FCF7BEFC26
:1043B8003046FCF7BBFC3046FCF7C4FC33685B4D69
:1043C8001946581C2A68306011F8020B82F82C0034
:1043D8003160597882F83610D91C31609B7882F8A0
:1043E80037303046FCF7AEFC3046FCF7ABFC3046C5
:1043F800FCF7A8FC3046D5F80080FCF797FCA8F835
:104408003A003046D5F80080FCF790FC33687268B3
:10441800A8F83800D11A01290ADD591C2A68316028
:104428001B7882F82E303046FCF78CFC33687268B3
:10443800D31A032B0BDD3046D5F80080FCF776FC49
:10444800A8F8320030462E68FCF770FCB086286861
:1044580047E4531C3360354DDFF8E480137888F85F
:1044680005303046D5F80090FCF760FCA9F820002C
:104478003046D5F80090FCF759FC72683368A9F803
:104488001E00D11A072919DD3046FCF74FFCA8F8A1
:104498000A003046FCF74AFCA8F80C003046D5F86C
:1044A8000090FCF743FCA9F822003046D5F80090AC
:1044B800FCF73CFC33687268A9F82400D11A032978
:1044C8000BDD3046FCF732FCA8F80E003046FCF74E
:1044D8002DFC33687268A8F81000D21A002A05DD8E
:1044E800591C2A6831601B7882F8263007F0C6FF0D
:1044F8001BF0BAFA0E4B1B68002B00F01A822868D2
:1045080001251EF083FB2B46FEF78ABD6C3E00207A
:104518009E340020C063002064650020785100208C
:10452800705900207C2C00206F5900201842002070
:104538005C510020703E0020A0340020B4340020DC
:10454800C84800201346511C3160BE4913F8020BBD
:10455800C8703360BC4953784B71D31C3360BB4B74
:104568009278DA7001252B46FEF75ABDD8F8085024
:10457800D8F80010FFF758B8FB697C681A463B7DED
:104588001370FFF7ABB91346511C3160B04D13F8E7
:10459800021B6970336053782B70D31C3360937897
:1045A800AB703046FCF7C2FB33682881591C1A46A9
:1045B800316012F8021B697132605B78AB710125BA
:1045C8002B46FEF72DBD531C336013780A2B00F0E1
:1045D800DF803046FCF7B6FB3046FCF7B3FB01251D
:1045E8003046FCF7AFFB2B46FEF71ABD531C336071
:1045F80013780A2B00F0C680502B7FF4BEAE3046ED
:10460800FCF794FBDFF86482A8F800003046FCF75A
:104618008DFB0125A8F802002B46FEF701BD8D4B46
:104628003A6A9B68D4F800905A449A4240F2BF8094
:104638003A6AA3EB0208FDF791F842464946386A00
:10464800FCF734FF236803442360002D3EF48EAC4E
:10465800B042BEF68BAC002100E0236801305A1C42
:10466800B04222601970F8D1FEF780BC33687268D6
:104678009A4240F0D680784BFF221A704FF0000A19
:10468800764D12F099FD51462022754885F800A014
:104698002EF0DBF987F82CA097F82C30072B00F2C6
:1046A8000481DFF8CC916E4E524697F82C3003EB1C
:1046B800430309EBC3035B7CE3B197F82C3003EBAE
:1046C800430309EBC30320215B699BB197F82C30A6
:1046D80003EB430309EBC303586946F822000CF0C7
:1046E80011FD2B7856F823000CF0CEFE2A78013203
:1046F800D2B22A7097F82C300133DBB287F82C300D
:1047080097F82C30072BD0D92368591C21601A70D0
:10471800B8F1000F3EF42AAC524BC8F8003001251E
:104728002B46FEF77DBC002D7FF479AF5946204615
:10473800FCF73EFB23685A1C22601D70454B266817
:104748009D683B6A0BEB0302AA4200F2FD80FDF76D
:1047580005F85A463146386AFCF7A8FE2368012551
:10476800034423602B46FEF75BBC3046FCF7DEFAB9
:10477800326871687B6A9142834648D106461D4675
:10478800FFF719B83046FCF7D1FADFF8E8803BE7C5
:10479800931C3360344B51781970D11C3160917877
:1047A8005970111D3160D2789A70FEF7DFBBFCF7A3
:1047B800D5FF5A464946386AFCF778FE2368034411
:1047C800236045E70AEBC80B30468BF80210FCF76C
:1047D800ADFA33682AF838001A46591C316012F8C5
:1047E800021B8BF8031032605A788BF80420DA1C0D
:1047F80032609A788BF806201A1D32600135DB7812
:104808008BF80530A9457FF454ABFEF7AFBB511CBC
:10481800316012781D46131C064618BF0123FEF7A7
:10482800CABF5A1C194632600B4811F8022B027095
:1048380031605B784370042A1ED9FF2A7EF4B5AB39
:104848001CE700BFCC600020443E0020DC60002054
:10485800A441002060190020C01D00207B460020D4
:104868003862002049ED01086B3300205C240020E9
:10487800A44C0020BC6000204B490978994205D817
:10488800022A7EF492ABFF2B7EF48FAB23680125BE
:104898005A1922601D70B8F1000F3EF467AB434B04
:1048A800C8F800302B46FEF7BBBB52462CE700F099
:1048B8007F00032828BF002001250EF063FD2B464A
:1048C800FEF7AEBB7D62AA46FFF70EB8DA46C7F818
:1048D80024B0FFF709B83046FCF728FAA884304618
:1048E800FCF724FA33687268E884D11A03297FF741
:1048F800EDAB1A46591C316012F8021BA9773260D9
:104908005B7885F820303046FCF710FA3368726817
:104918006884FFF7DBBB04297EF428ABFFF72CBAC9
:10492800234A1368012523F4004313602B46FEF73E
:1049380077BB20482049214A214B036001250B60A1
:1049480013602B46FEF76CBB3B6AED1AFCF706FFBB
:104958002A463146386AFCF7A9FD236803442360D8
:10496800FEF704BB01251EF075FB2B46FEF758BB6E
:10497800C50800F0070301350133EDB2DFF84880C0
:104988002846194688F8013017F056FD3FE40D4BCC
:1049980091781A88012512FB0EF22B4692FBF1F250
:1049A800A8F80020FEF73CBB6E3F0020B51A0108AE
:1049B80010420020D4550020285600209056002090
:1049C800F50300081C5F0020703E00202DE9F04F21
:1049D8002DED0E8BDFF8F4B097B0DBF804200790CC
:1049E80058469047002800F08E82BBF8A870002136
:1049F8008BF85110002F6DD1BBF93A00DBF8245029
:104A0800DBF82810BBF93860DBF82040BBF93C2004
:104A1800DFF8BCA0401B521ACBF830009BF85210AC
:104A2800CBF83420341B0BF12C00CBF82C401DF0B4
:104A380071FADAF80020910041F17987DBED0C5A20
:104A48001F4CDBED0B7A1F4994ED406AD4ED416AA7
:104A580094ED427AD4F80C2109681B4B0593B8EE03
:104A6800E58ADBED0D5AF8EEE77AF8EEE58A0132D1
:104A780077EE867A38EE268A78EE878A8A42C4EDFF
:104A8800407A84ED418AC4ED428AC4F80C2101F0D1
:104A98004A8393F800E0BEF1140F02F09B870023CD
:104AA800D4F814510693062D01F29784DFE815F027
:104AB8000416161728152917020CC6168A1500BFE2
:104AC800E81D002088510020C03F0020DC4800205D
:104AD800644B0020DE4BDF481A6808934FF47A765F
:104AE800B6FBF2F2C2EB421602EB8602D600DA4BB4
:104AF800DFF8C88344780593B6B2B7421D78B8F991
:104B0800060003F08980DBF87C30BBF93810DBF84D
:104B1800602003F1010E07EE901A0A44BEF1010F5E
:104B2800CBF87CE0CBF86020F8EEE77A03F08180E0
:104B3800DBED1B5ADBED1D6A07EE10EA37EEE56A7E
:104B4800B8EEC75A012F86EE057A37EE257A77EE4A
:104B5800C77A8BED1C7AE7EE866A8BED1B7AF0EE4E
:104B6800667ACBED1E6ACBED1D6A03F00384DBF891
:104B78009030BBF93A10DBF8642003F1010E07EE20
:104B8800901A0A44BEF1010FCBF890E0CBF86420EC
:104B9800F8EEE77A03F06880DBED205ADBED226A55
:104BA80007EE10EA37EEE56AB8EEC75A012F86EE2F
:104BB800057A37EE257A77EEC77A8BED217AE7EE1C
:104BC800866A8BED207AF0EE667ACBED236ACBED20
:104BD800226A03F0A783DBF8A430BBF93C10DBF8AA
:104BE800682003F1010E07EE901A0A44BEF1010F86
:104BF800CBF8A4E0CBF86820F8EEE77A03F04F8012
:104C0800DBED255ADBED276A07EE10EA37EEE56A99
:104C1800B8EEC75A012F86EE057A37EE257A77EE79
:104C2800C77A8BED267AE6EE276A8BED257AF0EEC9
:104C3800667ACBED286ACBED276A03F06683874C4A
:104C4800A8F80600BBF8A820059B013A1D78ABF828
:104C5800A82008990022072D4A608A60CA6040F09F
:104C6800598108F0A1FD059BDFF850821D78079B4C
:104C7800C01A94F82831A8F800000993002B40F0D6
:104C88004F81744A5279002A01F07A81744A127865
:104C9800013AD2B2072D84F8282102F01A820023A3
:104CA8000A93704BD4F83421D3F800A0684B0893CA
:104CB800079B9FED6D6AD4ED4C9A6C49C4F834316A
:104CC8009A1A07EE902AF8EE677AB7EE007AC6EEDF
:104CD800278A0025664BDFF8E891DFF8E881654F01
:104CE80006932E46D1ED006A94ED4BDA9FED629A59
:104CF800DFED62AA9FED62CA9FED62AADFED62BA9C
:104D08009FED62BA77EE69CA6CEEA6CAF4EEC7CA1E
:104D1800F1EE10FA88BFF0EE47CA5D4B99ED008AB4
:104D28002B44D3ED007AF5EE407AF1EE10FA17D065
:104D3800584B2B4493ED007A78EE476AB0EEE66A5A
:104D4800F4EEC67AF1EE10FA08D5F5EEC06AF1EE87
:104D580010FACCBF37EE878A37EE678A83ED008A70
:104D68004D4B1A88930739D0022E37D09AF82E1057
:104D78004A4B07EE901A2B4493ED007A4B42F8EE1B
:104D8800E76A07EE903A26EE877AF8EEE77AB4EE0D
:104D9800E77AF1EE10FA0AD407EE901AF8EE677A7D
:104DA800F4EEC77AF1EE10FA88BFF0EE477A3C4B82
:104DB8003C4903EB460331F91600B3F90C30C31A2A
:104DC80007EE103AB8EEC77AD007E7EE497A41F114
:104DD8007380354B93ED008A27EE888A089B94F8F8
:104DE80068212B4493ED01EA78EE4EDA002A00F0B0
:104DF800F7802E4BD4F86C2107991B688A1A9A42BF
:104E080040F3EE809AF84830022B02F0A181022E7E
:104E180004F04584264B1B68990700F19780254BC1
:104E280087ED00CA1B689342C0F2CA80F7EE007A89
:104E3800F4EEE79AF1EE10FA40F1D28008991E4B91
:104E4800D1ED017A93ED007AF0EEE77A3CE000BF0D
:104E5800544B0020C8480020C03F0020E81D002017
:104E6800C06000201842002000247449E456002045
:104E78000451002010510020CDCCCC3DAE47813FDD
:104E8800000000000000C84200003443610BB63B3C
:104E9800D85600202C1F002014420020381F002064
:104EA800CC600020C4410020C0560020EC560020F1
:104EB800C0410020E8560020F4560020C43F0020DE
:104EC800201F00201C510020F4EEC77AF1EE10FAE2
:104ED80040F18680D1ED027AF0EEE77AB4EEE77A17
:104EE800F1EE10FA7CDDD1ED037AF0EEE77AB4EE5C
:104EF800E77AF1EE10FA73DD0F4B1B689B075FD55D
:104F08000E490F4B43E00F4B0F4C1D780593072DAF
:104F18003FF4A7AE94F828310993002B3FF4B1AEC3
:104F2800013B84F82831012D01F0A88217B0BDECAF
:104F38000E8BBDE8F08F00BFC0410020C4410020A7
:104F4800CC600020C03F0020E81D0020D34BD4498E
:104F5800DFF8C8E331F916C09EED008ADFF8C0E338
:104F680087ED00CA03EB460028EE098AB0F90C0069
:104F7800A0EB0C0007EE900AF8EEE77ADEF80000E6
:104F880027EE888A904278EE4EDABFF64FAFB3F933
:104F98000C20B1F900E0C348AEEB020E00688EEABF
:104FA800EE72A2EBEE7282421ADAB3F90E30B1F960
:104FB8000220D21A82EAE273A3EBE27398420FDD71
:104FC800B94B1A88002384F86831002A43F06A85AF
:104FD800B64AB74B1178186881F001010CF05AFAFB
:104FE800B44B2B4493ED000A069B2DEE000A022ECB
:104FF80020EE2D0AA3EC010A069304F00D83AE4BB4
:10500800D7ED006A93ED007AAC4BD3ED007AAC4B48
:1050180093ED006AAB4B67EE277A2B4427EEAC7A08
:10502800D3ED007A67EE277AF0EE665AEDEEA75ACE
:10503800B1EE467AB4EEE57AF1EE10FA08DCB4EE99
:10504800E56AF1EE10FA8CBFB0EE657AB0EE467AFA
:1050580094ED4C6AF7EE007AB4EEE76AF1EE10FAD6
:10506800ACBF0123002343B1F0EEE66AF0EEC77A45
:10507800F4EEE67AF1EE10FA01D587ED007A022E09
:1050880004F0AC82904A914B52F826001B68B0EEAF
:105098004E0A98478E4A8F4B52F826001B6898474D
:1050A8009AF8373023B18C4B1B88002B00F06B87A4
:1050B800B0EE4C8A894B38EE400A2B4493ED008AB7
:1050C80083ED000A9AF8483030EE480A20EE288A24
:1050D800002B33D0824B1B7813F0010300F0B88605
:1050E800F7EE007AF4EEE79AF1EE10FA94F86831E8
:1050F800C1F2E684002B00F0EB87D4F86C31079AF4
:10510800D31A784A12689A4218DD774BD3ED007AA1
:10511800F0EEEDDAF4EEE7DAF1EE10FA42F129807A
:10512800614B1A88002384F86831002A00F09C86B5
:105138006E494A6912B10A6813604B746C4B94F853
:1051480078212B4493ED000A2DEE000A20EE088A00
:1051580088ED008A32B9069B87ED00CA03ED01CAC3
:1051680088ED00CA0136032E09F1040908F1040884
:1051780007F1040705F104057FF4CFAD059B1A7804
:10518800072A01F0B384012A01F0908700230693CF
:1051980094F88021002A41F07E81DFF888A1554BE0
:1051A800DAF800201968D60491F82C0000F1068777
:1051B800DFF87491504AB9F81A3092ED006A4F4AF4
:1051C8004F4DD2ED005AD5ED036A4E4A84ED646A1C
:1051D80007EE103A4C4B92ED005AD3ED007AD3ED1E
:1051E800013AD3ED024A84ED626AB8EEC77A35EE29
:1051F800C64A012236EEC77A84ED614AC4ED655A83
:1052080084F89821C7EE055A0A8D534206EE103AE3
:105218003E4BDFED3F6A93ED005A3E4B93ED004A5B
:10522800B7EE007AF4EEC75A35EE045AF1EE10FAEA
:1052380088BFF0EE475A35EE275AB8EEC66AF4EE44
:10524800E65AF1EE10FA07EE902AB4EEC65AB8BF45
:10525800F0EE665AF1EE10FAC4ED685AB8EE677AC5
:1052680001F10483B4EEC75AF1EE10FA88BFB0EE2C
:10527800475A264BDFED286AD3ED017A254B93ED8B
:10528800014A77EE847A25EE265A77EEA37AB4EEB1
:10529800E76AF1EE10FA52DC48E000BFCC6000206B
:1052A800C4410020F0560020C4640020C6640020D9
:1052B800C864002094560020D0550020000000202B
:1052C80008570020A0560020D8550020D4550020AB
:1052D8002C5600202856002014420020581F002079
:1052E800673E0020EC560020F8560020CC640020D1
:1052F800AC56002018420020385F0020986000203B
:10530800E83F0020A0570020105100200451002041
:10531800000000001C5100206F12833AC056002084
:10532800E8560020644B002070590020B4EEE77A5C
:10533800F1EE10FA8CBFB0EE676AB0EE476AEC4B3C
:105348004A8DD3ED027A9FEDEB7A534204EE103A80
:1053580074EEA77AB8EEC44A26EE076AF4EEC47A69
:10536800F1EE10FA0AD407EE102AB8EE474AB4EE66
:10537800E74AF1EE10FA88BFB0EE674ADE4ADFED81
:10538800DD7A527824EE274A0AB9B1EE444A002859
:1053980041F0D085B7EE003AD84E3278002A02F0B4
:1053A8004B86D749DFEDD77AD1ED024AD1ED016AB4
:1053B80091ED037A66EE244AE5EE264AE4EE074AC2
:1053C80063EE244AF4EEE74AF1EE10FAB4BFF0EEC9
:1053D800673AF0EE643A98BFF0EE647A012ACDEDB0
:1053E8000E4A02F04E8691ED067AD1ED052AD1EDEE
:1053F800076A26EE077AA5EE227AA4EE267A23EE2D
:10540800077AB4EEE77AF1EE10FAB4EEE37A8CBFDD
:10541800F0EE676AF0EE476AF1EE10FA88BFF0EE38
:10542800676AB4BFF0EE637AF0EE477A022A8DED30
:105438000F7A00F0DE8091ED0A7AD1ED092AD1EDDC
:105448000B3A26EE077AA5EE227AA4EE237A23EE0B
:10545800077AB4EEE67AF1EE10FAB4EEE77A8CBF8A
:10546800F0EE663AF0EE473AF1EE10FA98BFF0EE39
:10547800636AA8BFF0EE477A032A8DED107A00F030
:10548800B88091ED0E7AD1ED0D2AD1ED0F3A26EEC6
:10549800077AA5EE227AA4EE237A23EE077AB4EEF1
:1054A800E67AF1EE10FAB4EEE77A8CBFF0EE663ADF
:1054B800F0EE473AF1EE10FA98BFF0EE636AA8BF33
:1054C800F0EE477A042A8DED117A00F09280D1ED42
:1054D800123AD1ED112A91ED137A66EE233AE5EEF0
:1054E800223AE4EE073A63EE233AF4EEE63AF1EEB6
:1054F80010FAF4EEE73A8CBFB0EE667AB0EE637A53
:10550800F1EE10FA98BFF0EE476AA8BFF0EE637AA2
:10551800052ACDED123A6CD0D1ED163AD1ED152A07
:1055280091ED177A66EE233AE5EE223AE4EE073A71
:1055380063EE233AF4EEE63AF1EE10FAF4EEE73AC7
:105548008CBFB0EE667AB0EE637AF1EE10FA98BFCF
:10555800F0EE476AA8BFF0EE637A062ACDED133A5B
:1055680047D0D1ED1A3AD1ED192A91ED1B7A66EEA2
:10557800233AE5EE223AE4EE073A63EE233AF4EEF4
:10558800E63AF1EE10FAF4EEE73A8CBFB0EE667A3E
:10559800B0EE637AF1EE10FA98BFF0EE476AA8BF52
:1055A800F0EE637A072ACDED143A22D091ED1E7AF7
:1055B800D1ED1D2AD1ED1F3A26EE077AA5EE227A03
:1055C800A3EE847A27EE037AB4EEE67AF1EE10FAC7
:1055D800B4EEE77A8CBFB0EE666AB0EE476AF1EED9
:1055E80010FA8DED157A98BFF0EE466AA8BFF0EE76
:1055F800477A77EEE67AF7EE006AF4EEE67AF1EEAD
:1056080010FAC4ED4C7A43F3D78586EEA77A022ABE
:10561800DDED0F7A67EE244A67EE877ACDED0E4A04
:10562800CDED0F7A2DD0DDED107A67EE877A032A5B
:10563800CDED107A25D0DDED117A67EE877A042A50
:10564800CDED117A1DD0DDED127A67EE877A052A45
:10565800CDED127A15D0DDED137A67EE877A062A3A
:10566800CDED137A0DD0DDED147A67EE877A072A2F
:10567800CDED147A05D0DDED157A27EE877A8DED1C
:10568800157A2149096811F080530A9301F0CB81FA
:10569800F6EE005AC4ED685A002A02F09D8494F987
:1056A80098311A4994ED656AC87894ED645ADAF825
:1056B8000010DFF868E0164FDEED004AB7F906E0A3
:1056C800B9F81A700B9707EE103A124BD4ED616ACD
:1056D8001D78114BD4ED627A1B780893BDEEC66A2B
:1056E80001F4805316EE10CABDEEC56A0D9317E09B
:1056F800045100206F12833A785100206E3F002039
:10570800105700200000000090600020C0420020D8
:1057180092710020673E0020884D00200C57002021
:1057280001F4800301F01007B8EEC77A0C9305F076
:10573800010816EE101A002840F06487002F41F087
:10574800D582D34D9DED0E5A95ED006AD14825EED0
:10575800866AA5EE076AB0EE675AA6EE265ABDEE2F
:10576800C56A16EE10EA16EE107AE645A8BF674637
:105778007145C8BF0F4606EE107AB8EEC66A012A10
:1057880080ED006A00F0DC8095ED046A9DED0F5A0B
:1057980025EE866AA5EE076AB0EE675AA6EE265A87
:1057A800BDEEC56A16EE10EA16EE107AE645A8BFF9
:1057B80067467145C8BF0F4606EE107AB8EEC66A4E
:1057C800022A80ED016A00F0BB8095ED086A9DED24
:1057D800105A25EE866AA5EE076AB0EE675AA6EE5D
:1057E800265ABDEEC56A16EE10EA16EE107AE645A0
:1057F800A8BF67467145C8BF0F4606EE107AB8EED7
:10580800C66A032A80ED026A00F09A8095ED0C6A58
:105818009DED115A25EE866AA5EE076AB0EE675A25
:10582800A6EE265ABDEEC56A16EE10EA16EE107AF6
:10583800E645A8BF67467145C8BF0F4606EE107A11
:10584800B8EEC66A042A80ED036A79D095ED106A2D
:105858009DED125A25EE866AA5EE076AB0EE675AE4
:10586800A6EE265ABDEEC56A16EE10EA16EE107AB6
:10587800E645A8BF67467145C8BF0F4606EE107AD1
:10588800B8EEC66A052A80ED046A59D095ED146A07
:105898009DED135A25EE866AA5EE076AB0EE675AA3
:1058A800A6EE265ABDEEC56A16EE10EA16EE107A76
:1058B800E645A8BF67467145C8BF0F4606EE107A91
:1058C800B8EEC66A062A80ED056A39D095ED186AE1
:1058D8009DED145A25EE866AA5EE076AB0EE675A62
:1058E800A6EE265ABDEEC56A16EE10EA16EE107A36
:1058F800E645A8BF67467145C8BF0F4606EE107A51
:10590800B8EEC66A072A80ED066A19D095ED1C6ABA
:105918009DED155A65EE865AE7EE055AE6EEA57A2C
:10592800FDEEE77A17EE905AAC45A8BFAC46A942FF
:10593800D8BF614607EE901AF8EEE77AC0ED077A0D
:10594800B8F1000F00F06C87534A1268002A40F043
:105958007487524A127892B1307868B14D4FDFF8A7
:105968005C810025E8B2D8F80030B7EC010A984706
:10597800307801358542F5DB494A12689047059B26
:105988001A78072A01F0A1800026DAF800205305CA
:1059980000F1D187434B1B78BBB1434AB9F81A30A1
:1059A800B2F906209A4210DC404B1B78012B01F01B
:1059B8009583192B01F092830E2B06D0082B04D067
:1059C8003B4D0023AB60C4F8403194F8AA5125B18F
:1059D800384B1B889F0741F02F8394F8B021002A89
:1059E80040F0488799F81E70002F00F02984022F94
:1059F80001F0D582032F41F0CE8299F82030C3EB15
:105A0800431103EB8101C90089B299F81F300233B1
:105A1800DBB2002A00F05585002900F0528526489F
:105A28000768B1FBF7F10FB2A4F8E071002B03F09F
:105A3800438007EE907AF8EEE77AF7EE006A86EE92
:105A4800A77A1B4D012BD4ED7D6AD5ED007A77EE50
:105A5800E67A67EE877AC4ED797A3BD0D5ED017A9C
:105A6800D4ED7E6A77EEE67A022B67EE877AC4ED8C
:105A78007A7A2FD0D5ED027AD4ED7F6A77EEE67A7E
:105A8800032B67EE877AC4ED7B7A23D018E000BF3A
:105A98001057002038510020CC550020B05000206D
:105AA800844D00209C1B002092710020785100201A
:105AB800E83F0020144200205C5100207C4D00206B
:105AC800D5ED037AD4ED806A77EEE67A67EE877AC9
:105AD800C4ED7C7A05990978092903F0ED81002F36
:105AE80040F3B4839BB394ED7D7AD4ED797A77EE65
:105AF800877A012BC4ED7D7AC5ED007A21D094ED2B
:105B08007E7AD4ED7A7A77EE877A022BC4ED7E7AA4
:105B1800C5ED017A15D094ED7F7AD4ED7B7A77EED6
:105B2800877A032BC4ED7F7AC5ED027A09D0D4EDCC
:105B3800807A94ED7C7A77EE877AC4ED807AC5ED29
:105B4800037A013B022BB8BF0223DBB20993099BFE
:105B5800002A18BF02239E46C84BDFEDC96A1A689F
:105B6800059B91781878137807EE903AF8EEE77A63
:105B7800B0EE007A67EEA67AF4EEC77AF1EE10FA84
:105B880040F35F86DFEDBF6A37EEC77AB0EE676A2B
:105B9800A7EE266AF0EE466A95ED007A9FEDBA6A9E
:105BA80027EE066AF0EEC65A84ED546AC4ED575AD9
:105BB80099B107EE101AB8EEC75A9FEDB17A66EEA2
:105BC800064A25EE075AB7EE007A37EE457A64EEB4
:105BD800A54AA4EE857A26EE076A9FEDAC7A53793A
:105BE80026EE877A27EE067ACBB1DFEDA56A9FED20
:105BF800A86A65EEA65A06EE903AF8EEE66A65EEF1
:105C0800A65AF4EEC65AF1EE10FA01F38981B7EEFE
:105C1800006A76EE655AC6EE256A27EE267A0C28C3
:105C28009FED9C8ADFED9C6A00F02487B4EEC87A69
:105C3800F1EE10FA98BFB0EE478AB4EEE68AF1EEBC
:105C480010FAB8BFB0EE668A84ED4E8ABEF1000F36
:105C580000F0DD80B0EE007AF4EEC77AF1EE10FACB
:105C680005DD37EEC77ADFED876AE7EE267A95ED30
:105C7800017ADFED856A27EE267AF0EEC75A84EDC1
:105C8800557AC4ED585A99B106EE901A9FED7C6A80
:105C9800F8EEE66A27EE075A66EE866AB7EE006AFD
:105CA80036EE666A25EE255AA5EE266A27EE067AAE
:105CB800DFED766A937967EEA67A67EE877AABB1FD
:105CC80007EE103AB8EEC77A9FED6D6ADFED706A9D
:105CD80027EE257A27EE067AB4EEE67AF1EE10FA88
:105CE80041F31081DFED6D6A67EEA67A0C2800F0AB
:105CF800A186DFED686A9FED687AF4EEE67AF1EE48
:105D080010FA88BFF0EE667AF4EEC77AF1EE10FA70
:105D1800B8BFF0EE477ABEF1010FC4ED4F7A76DDD9
:105D28005378DFED576A07EE903AF8EEE77AB0EE6F
:105D3800007A67EEA67A537AF4EEC77AF1EE10FA93
:105D480005DD37EEC77ADFED4F6AE7EE267A95ED87
:105D5800027ADFED4D6A27EE267AF0EEC75A84ED17
:105D6800567AC4ED595A9BB106EE903A9FED446AB3
:105D7800F8EEE66A27EE075A66EE866AB7EE006A1C
:105D880036EE666A25EE255AA5EE266A27EE067ACD
:105D9800DFED3E6AD37967EEA67A67EE877AFBB1C4
:105DA80007EE103AB8EEC77A9FED356ADFED386A2C
:105DB80027EE257A27EE067AB4EEE67AF1EE10FAA7
:105DC80001F39C80B5EEC07AF1EE10FA02F1FE8282
:105DD800B7EE006A36EE477AC6EE076A67EEA67A2D
:105DE8000C2800F06586DFED2B6A9FED2B7AF4EE28
:105DF800E67AF1EE10FA88BFF0EE667AF4EEC77A2A
:105E0800F1EE10FAB8BFF0EE477AC4ED507A0928DF
:105E180000F0FC8599F82150002D40F0B185002351
:105E280084F8B0311E4B1B7823B91E4DAA78002A7E
:105E380041F0C180059B1D78072D7FF474A807F0F9
:105E4800B3FC194B059A801B1578D880FFF76BB8FF
:105E580094F86821002A3FF471A9144A84F868313B
:105E68001288002A7FF464A9114A124B1178186825
:105E780081F001010BF00EFBFFF760B91C42002016
:105E88000AD7233CD7A368416F12033B000048435D
:105E9800A4707D3F00C0F94400C0F9C40000C842A6
:105EA8005D420020A0340020C43F0020C4640020CC
:105EB800C6640020C864002094ED577AB1F9000048
:105EC800D4ED586AB1F902E0E24AF4EEC76A80EA12
:105ED800E0738EEAEE71A3EBE073F1EE10FAA1EB3A
:105EE800EE71B8BFF0EE476A8B42B8BF0B4607EEBB
:105EF800103A1378B8EEC77A27EE097A002B40F0EB
:105F0800B880D54B93ED006AB4EEEA6AF1EE10FA68
:105F180041F14C80F7EE005A75EEC65A3BEEC77A4F
:105F280065EE8B5ACD4BA7EE256A93ED007A26EEE7
:105F3800076AB5EEC06AF1EE10FA40F27085CAEE53
:105F4800065AB7EE007AB0EE476AA6EEE56AF0EEBA
:105F5800466AF4EEC76AF1EE10FA88BFF0EE476AB7
:105F6800F5EEC06AF1EE10FAB8BFF0EE4C6ABC4B21
:105F780093ED007A67EE877AA7EEA68AFEF72EBF22
:105F88000122FEF787BEB74BB74A2B4493ED007A40
:105F9800D2ED007AB54B67EE277AF7EE006AF4EE99
:105FA800E67AF1EE10FA93ED007A88BFF0EE667AA1
:105FB80067EE877A27EE888AFFF77CB8AC4BDFF864
:105FC800EC921A78D5075CBFB9F81820A4F88C2190
:105FD800A84AA94D1288D5ED037A07EE102AB8EE23
:105FE800C77AF4EEC77AF1EE10FA41F2C587A34DED
:105FF8002B8807EE103AB8EEC77AF4EEC77AF1EEBE
:1060080010FAC1F277809E4A9E4D92ED006AD5ED56
:10601800006A94F99821C4ED646A76EE665A012AFA
:10602800C4ED626AC4ED615A84ED656A01F0EE85DB
:10603800079BC4F89C31002537EEC77AFCEEE77A57
:10604800914E84ED687A17EE902AA4F88C210122EB
:1060580096ED005A84F898218C4A954241F2798746
:106068008B4BD3ED007AD3ED013AD3ED024AFFF71B
:10607800C9B87A4B93ED005AB5EEC05AF1EE10FA52
:1060880040F3CD84834BD3ED004AF5EEC04AF1EEE0
:1060980010FA40F3C48434EEC77A66EECA5A87EE23
:1060A800246AC5EE856AB7EE007AB4EEC76AF1EEE7
:1060B80010FA88BFB0EE476AB5EEC06AF1EE10FA82
:1060C80076EE876AB8BFB0EE4C6A66EE266A40E79D
:1060D800714AD2ED007AB0EEC87AB4EEE77AF1EE02
:1060E80010FA7FF72BA86D4AD2ED007AB0EEED7A60
:1060F800B4EEE77AF1EE10FA7FF720A8684AD9EDF6
:10610800007A92ED007AF0EEE77AF4EEC77AF1EED3
:1061180010FA7FF513A801220799C4F86C1184F8C6
:106128006821FEF7EEBF07EE102A1978DFF88081A4
:10613800C4F80C71B8EEC77AF7EE006A132986EE38
:10614800879AB8F90400B4F810619BED070A01F0CA
:10615800E984544A544992ED001AD2ED053A92ED79
:10616800122A92ED173AD2ED091AD2ED0E4A92EDA3
:10617800016A92ED064A92ED0A7AD2ED0F5AD2EDF3
:10618800132AD2ED186A92ED045AD2ED030A67EE8B
:10619800897A69EE288A29EE088AE1EE273A01EB26
:1061A80086070025A2EE283AC4F80051C4F8045125
:1061B800E1EE884AA6EE274AE7EE085A92ED167AEB
:1061C80092ED0D6A92ED021AD2ED0C1AC7ED003A63
:1061D800E2EEA86A25EE635A27EE437A92ED0B2A7F
:1061E800D2ED152AC7ED204AA0EEE34A26EE646AEE
:1061F800D2ED143A82ED054AA1EE275AF0EE477A1D
:10620800E1EEE45AA2EE086AE2EEC36AE3EEA87A87
:1062180082ED065AC2ED0E5A82ED0F6A87ED403ABA
:10622800C2ED176AC2ED187AC4F80851721C02F060
:106238001F02A4F81021A8F80400059BFEF729BC4A
:10624800A4F8E071002A3FF4EDAD0B4D4FF0020EBB
:1062580082E400BFCC560020D4560020C856002047
:10626800C4560020441F0020BC560020B856002009
:10627800673E0020A4570020E83F0020A6570020D2
:106288009860002090570020AC5700208FD0030062
:1062980010510020D0560020FC560020F85600204F
:1062A8000057002018540020AC51002070590020DD
:1062B800C43F0020BC4A1178D4F81871BB4B9FED3D
:1062C800BC7AFE009A1982ED007A002979D0B94883
:1062D800B0EE476AF0EE476A0022F0EC017A01322C
:1062E80067EEA77A05EE902AB4EEE77AF1EE10FA97
:1062F800F8EEE55AB8BFB0EE677A8A4276EEA76A3A
:10630800A7EEA56AE9D1F5EEC06A9A19F1EE10FA7E
:1063180082ED007A55DDC6EE265AA74AA7490988B4
:10632800F7EE007A75EEE75AD2ED007A65EEA77AB5
:10633800FDEEE77A17EE902A812A42F353808A42CB
:10634800A8BF0A4607EE902AF8EEE77A9C4AF019A9
:1063580002EB800292ED057AD2ED003A92ED066AE0
:1063680092ED014AD2ED046AD2ED034A92ED025A47
:10637800A3EEA77AA4EE276A66EEC76AA7EE646A58
:10638800BDEEC77AE5EE276A17EE100A812882ED7E
:10639800056AC2ED066A42F322808142A8BF01461F
:1063A80007EE901AF8EEE77AFCEEE77ACDED087A78
:1063B800BDF8202099198A801FB9BEF1130F02F089
:1063C800E786BEF1150F41F0ED801E44DFF810821C
:1063D800B28828F81720D4F814517A4A013582FB7C
:1063E80005325119EA17C2EBA102C2EBC202AD1A7B
:1063F800C4F814517448D4F81C11079B734D0268F3
:106408002D78C4F81C31591A0A440260002D64D151
:1064180007EE901A6E4EDFF8E0916E4FB8EEE78AFD
:1064280006F5F07506F51378F6EC017A9BED070A88
:10643800DBF80832F8EEE77A284627EE800A984714
:10644800A5F1E000DBF828319847A5F17000DBF8EA
:1064580098319847D6F8EC00DBF8AC309847D7ED80
:10646800007AA9EC010AE0EE087A2435A845E7ECA1
:10647800017AD9D1059B1D78FEF749BD564B574A7D
:1064880019681288564BC96919805A8017B0BDEC33
:106498000E8BBDE8F08F534B534E1A7812F0010F54
:1064A800327840F03983002A00F03E8592004F4947
:1064B8004F48DFF848A1DFF848912BF0CBF9FFF7F8
:1064C80043BAB4F8E071013F3FB2002FA4F8E0717D
:1064D8007FF7B8AE474DFFF705BB07EE901A3C4D66
:1064E800454BDFF8FC80DFF8EC900694F8EEE78A7D
:1064F80005F5B87600271C46CDF82480059BDBED12
:10650800077A1B78172B00F0A08195ED007AB8EE7A
:10651800C78A082B28EE278A07D1B0EE480A0893C5
:106528002BF0D8FA089BA8F80000DAF800209200AF
:106538000BD5002F03F00281B0EE480ADBF80832D1
:1065480006F170009847B0EE408AB0EE480ADBF8D2
:106558002831A6F170009847DBF898313046984703
:10656800059B1B78032BB0EE408A00F07A81D5F8A2
:10657800F000DBF8AC30B0EE480A9847D9ED007A65
:10658800A4EC010AE0EE287A0137032F06F124066D
:1065980008F1020805F10405E9EC017AAED1059B82
:1065A800069C1D78FEF7B3BC8E5100208454002051
:1065B80000000000E81D0020905100208C510020B0
:1065C800AC5300209324499228650020855100206F
:1065D800084900202C650020543E0020102D002082
:1065E800C43F0020673E00206E3F0020142D00208D
:1065F80038510020E83F0020584B0020644B002011
:1066080070590020002F00F09186B8F1000F42F079
:10661800A982089BCD4D002B42F0F68095ED006ACB
:106628009DED0E5ACA4825EE866AFDEEE44AA5EEAF
:10663800076AB0EE675AA6EE265A14EE901ABDEE17
:10664800C56A16EE10EA16EE107AE645A8BF674648
:106658007145C8BF0F4606EE107AB8EEC66A012A21
:1066680080ED006A00F0DF8095ED046A9DED0F5A19
:1066780025EE866AA5EE076AB0EE675AA6EE265A98
:10668800BDEEC56A16EE10EA16EE107AE645A8BF0A
:1066980067468E45B8BF0F4606EE107AB8EEC66A52
:1066A800022A80ED016A00F0BE8095ED086A9DED32
:1066B800105A25EE866AA5EE076AB0EE675AA6EE6E
:1066C800265ABDEEC56A16EE10EA16EE107AE645B1
:1066D800A8BF67468E45B8BF0F4606EE107AB8EEDB
:1066E800C66A032A80ED026A00F09D8095ED0C6A67
:1066F8009DED115A25EE866AA5EE076AB0EE675A37
:10670800A6EE265ABDEEC56A16EE10EA16EE107A07
:10671800E645A8BF67468E45B8BF0F4606EE107A15
:10672800B8EEC66A042A80ED036A7CD095ED106A3B
:106738009DED125A25EE866AA5EE076AB0EE675AF5
:10674800A6EE265ABDEEC56A16EE10EA16EE107AC7
:10675800E645A8BF67468E45B8BF0F4606EE107AD5
:10676800B8EEC66A052A80ED046A5CD095ED146A15
:106778009DED135A25EE866AA5EE076AB0EE675AB4
:10678800A6EE265ABDEEC56A16EE10EA16EE107A87
:10679800E645A8BF67468E45B8BF0F4606EE107A95
:1067A800B8EEC66A062A80ED056A3CD095ED186AEF
:1067B8009DED145A25EE866AA5EE076AB0EE675A73
:1067C800A6EE265ABDEEC56A16EE10EA16EE107A47
:1067D800E645A8BF67468E45B8BF0F4606EE107A55
:1067E800B8EEC66A072A80ED066A1CD095ED1C6AC9
:1067F8009DED155A65EE865AE7EE055AE6EEA57A3E
:10680800FDEEE77A17EE905AAC45A8BFAC46A94210
:10681800D8BF614607EE901AF8EEE77AC0ED077A1E
:10682800002A3FF491A892004A4949482BF012F8EF
:10683800494A1268002A3FF48CA81BF08FFDFFF725
:1068480088B8F0EE676AFFF7A7B995ED007A0BEB09
:106858004702B8EEC78A128FA8F8002028EE278AC8
:1068680063E62BF037F9A8F8000080E6B0EE465A48
:10687800FEF7FFBC39493A4BD1F8EC101B6844F6D7
:1068880020608142A8BF0146B1F57A7FB8BF4FF4B6
:106898007A7189B213F0100FA4F8B211DAF8003047
:1068A80000F02384DB0441F1A1852E4BD3F800E0EE
:1068B800BEF832707F082C4D2C48D4F8B431D5ED91
:1068C800037AA0FB01018809642191FBF0F11429E6
:1068D800BDEEE77A04EB4305A8BF142101338B42D0
:1068E800C4F8B43117EE10CAA4BF0023C4F8B431F9
:1068F80004EB4303A5F8B8C1B3F9B83107EE103A71
:10690800B8EEC77A77EEC77AFDEEE77ACDED067A6C
:10691800BDF9181081EAE173A3EBE173BB4201F3FF
:106928002D8713494FF07E530B60FFF75BB8114B6F
:106938000593114C5EE5DBF80830002B3FF42AA8DC
:106948000E49A1F14C009847FFF724B810570020D2
:1069580038510020142D0020CC550020540F002061
:106968009060002018420020E83F0020D34D6210BC
:1069780000000020C03F0020E81D0020284900201A
:106988001E21CE48FAF7F0FC00283FF448AACC4B69
:106998001B8858063FF543AA94F80432AB4242F0EC
:1069A8001C82C84BD4ED827AD3ED016A94ED505A1B
:1069B800DFEDC55A9FEDC56A27EEC57A68EE277ADE
:1069C800A8EE267AE5EE267AB4EEE57AF1EE10FA2C
:1069D80088BFB0EE657AB4EEC67AF1EE10FAF4EE3E
:1069E800E57AB8BFB0EE467AF1EE10FA88BFF0EE5D
:1069F800657AF4EEC67AF1EE10FAB8BFF0EE467A90
:106A080084ED4E7AC4ED507AFFF709BAFDEEC87AE4
:106A1800AF4A17EE903A9780D380FFF7FBB9DFEDC6
:106A2800AD6AFFF7A4BADAF8001049023EF530AEB5
:106A3800FEF732BE9FEDA47ADFEDA46AA449F4EE16
:106A4800C77AF1EE10FA98BFB0EE677AFDEEE77AF2
:106A5800B4EEE67AF1EE10FA17EE903AB8BFB0EE5F
:106A6800667ABEF1010F84ED4F7A4B803FF758A943
:106A7800FFF7D0B9B4EEC87AF1EE10FA98BFB0EECD
:106A8800478ABDEEC77AB4EEE68ADFF844C2F1EE73
:106A980010FA17EE103AB8BFB0EE668A84ED4E8A47
:106AA800ACF80030BEF1000F7FF4D4A8FFF7B2B9FC
:106AB800BDEEE77A864B17EE102A9A80FFF793B956
:106AC800002B3EF43BABFEF718BB06F06DFE059BB2
:106AD8007F491A78069B072AA0EB030088807EF47A
:106AE80053AF06F061FE0646FEF74FBF06F05CFEA8
:106AF800059BDFF8DC811A780A9B012AA0EB0300CA
:106B0800A8F8020000F0D482072A7EF43FAB06F012
:106B18004BFE0690FEF73CBB002A00F00582D4ED40
:106B2800583A94ED574AD4ED627A6B4994ED617AFC
:106B380091ED005AD4ED555A94ED546A674D684862
:106B4800F4EEC43AF3EE046AF1EE10FA77EEA64AD0
:106B580000F11E8395ED026A26EE656AB0EE674A7B
:106B6800A6EE074AB4EEE44A34EE666AF1EE10FA8D
:106B780048BFB0EE456A012A80ED006A00F0D48172
:106B880095ED066A26EE656AB0EE674AA6EE074AF4
:106B9800B4EEE44A34EE666AF1EE10FA48BFB0EE9D
:106BA800456A022A80ED016A00F0BE8195ED0A6A05
:106BB80026EE656AB0EE674AA6EE074AB4EEE44AE6
:106BC80034EE666AF1EE10FA48BFB0EE456A032A61
:106BD80080ED026A00F0A88195ED0E6A26EE656ADE
:106BE800B0EE674AA6EE074AB4EEE44A34EE666AA7
:106BF800F1EE10FA48BFB0EE456A042A80ED036A48
:106C080000F0928195ED126A26EE656AB0EE674A49
:106C1800A6EE074AB4EEE44A34EE666AF1EE10FADC
:106C280048BFB0EE456A052A80ED046A00F07C8111
:106C380095ED166A26EE656AB0EE674AA6EE074A33
:106C4800B4EEE44A74EE666AF1EE10FA48BFF0EE6C
:106C5800456A062AC0ED056A00F06681D5ED1A6A14
:106C680066EEE56AB0EE674AA6EE874AB3EE046AB6
:106C7800B4EEE44A74EE466AF1EE10FA48BFF0EE5C
:106C8800456A072AC0ED066A00F04E81D5ED1E6AF6
:106C9800DFF850A0DFF8509066EEE55AE5EE877A07
:106CA800F4EEE74A77EEC67AF1EE10FAC8BFF0EED6
:106CB800457AC0ED077AFEF747BE00BF9060002016
:106CC800144200200000002000C0F94400C0F9C4AC
:106CD800C43F0020000000000C570020105700207F
:106CE80038510020644B002070590020B8F1000F83
:106CF80041F00282DB4D9DED0E5A95ED006ADA48AF
:106D080025EE866AA5EE076AB0EE675AA6EE265A01
:106D1800BDEEC56A16EE10EA16EE107AE645A8BF73
:106D280067467145C8BF0F4606EE107AB8EEC66AC8
:106D3800012A80ED006A3FF476AD95ED046A9DED79
:106D48000F5A25EE866AA5EE076AB0EE675AA6EED8
:106D5800265ABDEEC56A16EE10EA16EE107AE6451A
:106D6800A8BF67467145C8BF0F4606EE107AB8EE51
:106D7800C66A022A80ED016A3FF455AD95ED086AAE
:106D88009DED105A25EE866AA5EE076AB0EE675AA1
:106D9800A6EE265ABDEEC56A16EE10EA16EE107A71
:106DA800E645A8BF67467145C8BF0F4606EE107A8C
:106DB800B8EEC66A032A80ED026A3FF434AD95ED59
:106DC8000C6A9DED115A25EE866AA5EE076AB0EEAB
:106DD800675AA6EE265ABDEEC56A16EE10EA16EEFA
:106DE800107AE645A8BF67467145C8BF0F4606EE4C
:106DF800107AB8EEC66A042A80ED036A3FF413AD30
:106E080095ED106A9DED125A25EE866AA5EE076A81
:106E1800B0EE675AA6EE265ABDEEC56A16EE10EA1F
:106E280016EE107AE645A8BF67467145C8BF0F46FB
:106E380006EE107AB8EEC66A052A80ED046A3FF4B9
:106E4800F2AC95ED146A9DED135A25EE866AA5EE0F
:106E5800076AB0EE675AA6EE265ABDEEC56A16EE68
:106E680010EA16EE107AE645A8BF67467145C8BF16
:106E78000F4606EE107AB8EEC66A062A80ED056A55
:106E88003FF4D1AC95ED186A9DED145A25EE866A4B
:106E9800A5EE076AB0EE675AA6EE265ABDEEC56A99
:106EA80016EE10EA16EE107AE645A8BF6746714559
:106EB800C8BF0F4606EE107AB8EEC66A072A80EDFC
:106EC800066A3FF4B0AC95ED1C6A9DED155A65EE67
:106ED800865AE7EE055AE6EEA57AFDEEE77A17EE52
:106EE800905AAC45A8BFAC46A942C8BF8C4607EE2D
:106EF80090CAF8EEE77AC0ED077A91E4DFED5B6AB5
:106F0800FEF76CBFB5EEC07AF1EE10FA01F15A82C5
:106F1800B7EE006A36EE477AC6EE076AFEF7E4BEB9
:106F2800DFED526AFEF779BEDFF878A1DFF87891D5
:106F3800FEF70ABD4E494A79002A3EF42BAA4D4A6B
:106F48001278002A3EF426AA0B784B49DFED4B4A0B
:106F580007EE903A0B88B8EE677A07EE902A06EEAD
:106F6800903AF8EEE77AF8EE666A67EE277AB7EEB7
:106F7800007A87EEA63AB4EEE43AF1EE10FA88BF4A
:106F8800B0EE643AB4EEC73AF1EE10FAB8BFB0EE1C
:106F9800473AFEF701BA3A4B5988FEF736BDB4F8BE
:106FA800B21101F57A7189B2FEF72FBD354B93ED19
:106FB800006AFEF7BEBF344F3B78013B0D2B24D847
:106FC800DFE813F0F506BB07E606CB06230023002F
:106FD800A4078F0734070E0067075B0786070207B9
:106FE8002A4B1B78002B02F0F5801A2027F046FF69
:106FF800002842F0EF80264B1B78002B42F0EA80F5
:1070080009233B7024F0DEFAAA78012A00F0638590
:107018002B79012B01F05985022B7EF40BAF3B78BD
:10702800012B7EF407AF1A4B1B78002B7EF402AFBE
:1070380023F092FFFEF7FEBE164B9FED177AD3EDB5
:10704800087AF4EEC77AF1EE10FA00F2F9849FEDAF
:10705800137A134DD5ED037A77EE877AC5ED037A67
:10706800FEF7BBBC10570020385100200000C84272
:10707800A4410020E63F0020D03F0020713DAA3FF8
:10708800A8420020C85600209E3400207A510020D3
:10709800095F0020006500208FC2753C00000000D9
:1070A800E83F0020644B002070590020DFF8708210
:1070B80006F07AFB9049D4F87C2109680690821A78
:1070C800511AC4F87C01A8F80420A8F80610FEF7A5
:1070D8005FB806F069FB0A90FDF7E3BD874B9B7B21
:1070E800002B3EF46DACFEF770BCDD003FF5DAAB6B
:1070F800FEF778BCB4F88C51954240F2028594F8BA
:10710800A451002D40F06E877D4A7E4E92ED007AA4
:10711800D6ED007A94F99821C4ED647A77EE676A1F
:10712800012AC4ED627AC4ED616A84ED657A02F0E1
:107138003D80079BC4F89C31734A9FED747A92EDA9
:10714800005A84ED687A012284F89821FEF784BFFA
:107158006F4B1B88002B40F0E8856E4A6E4B117808
:1071680018680AF097F9D4F86C21079B9A1AFDF76A
:107178004EBE6A4BD9ED007A93ED007AF0EEE77ACD
:10718800F4EEC77AF1EE10FA7DF7D8AFFDF7C8BF75
:10719800D5ED015A65EEC65AB0EE674AA5EE874AA4
:1071A800B4EEE44A74EE665AF1EE10FA48BFF0EE17
:1071B800455A012AC0ED005A3FF4B6AED5ED055A3E
:1071C80065EEC65AB0EE674AA5EE874AB4EEE44AC1
:1071D80074EE665AF1EE10FA48BFF0EE455A022AEC
:1071E800C0ED015A3FF4A0AED5ED095A65EEC65A76
:1071F800B0EE674AA5EE874AB4EEE44A74EE665AE2
:10720800F1EE10FA48BFF0EE455A032AC0ED025AD3
:107218003FF48AAED5ED0D5A65EEC65AB0EE674A10
:10722800A5EE874AB4EEE44A74EE665AF1EE10FA17
:1072380048BFF0EE455A042AC0ED035A3FF474AE35
:10724800D5ED115A65EEC65AB0EE674AA5EE874AE3
:10725800B4EEE44A74EE665AF1EE10FA48BFF0EE66
:10726800455A052AC0ED045A3FF45EAED5ED155ACD
:1072780065EEC65AB0EE674AA5EE874AB4EEE44A10
:1072880074EE666AF1EE10FA48BFF0EE456A062A17
:10729800C0ED056A3FF448AED5ED196A66EEC66AD8
:1072A800B0EE674AA6EE874AF3EE045AB4EEE44A13
:1072B80074EE656AF1EE10FA48BFF0EE456A072AE7
:1072C800C0ED066A3FF430AED5ED1D6ADFF854A074
:1072D800DFF8549026EEC66AE6EE077AF4EEE47A12
:1072E80077EEE57AF1EE10FAB8BFF0EE457AC0ED28
:1072F800077AFEF729BB00BF5C510020C04600207A
:107308009860002090570020AC5700200000000033
:10731800C4640020C6640020C86400200057002010
:10732800C43F0020644B002070590020089BD94DB1
:10733800002B41F08D8095ED006A9DED0E5AD648E0
:1073480025EE866AFDEEE44AA5EE076AB0EE675AB6
:10735800A6EE265A14EE901ABDEEC56A16EE10EA8D
:1073680016EE107AE645A8BF67467145C8BF0F46B6
:1073780006EE107AB8EEC66A012A80ED006A3EF47D
:10738800DFAA95ED046A9DED0F5A25EE866AA5EEF3
:10739800076AB0EE675AA6EE265ABDEEC56A16EE23
:1073A80010EA16EE107AE645A8BF67468E45B8BFC4
:1073B8000F4606EE107AB8EEC66A022A80ED016A18
:1073C8003EF4BEAA95ED086A9DED105A25EE866A30
:1073D800A5EE076AB0EE675AA6EE265ABDEEC56A54
:1073E80016EE10EA16EE107AE645A8BF67468E45F7
:1073F800B8BF0F4606EE107AB8EEC66A032A80EDCB
:10740800026A3EF49DAA95ED0C6A9DED115A25EE8F
:10741800866AA5EE076AB0EE675AA6EE265ABDEE52
:10742800C56A16EE10EA16EE107AE645A8BF67465A
:107438008E45B8BF0F4606EE107AB8EEC66A042A23
:1074480080ED036A3EF47CAA95ED106A9DED125A10
:1074580025EE866AA5EE076AB0EE675AA6EE265AAA
:10746800BDEEC56A16EE10EA16EE107AE645A8BF1C
:1074780067468E45B8BF0F4606EE107AB8EEC66A64
:10748800052A80ED046A3EF45BAA95ED146A9DED29
:10749800135A25EE866AA5EE076AB0EE675AA6EE7D
:1074A800265ABDEEC56A16EE10EA16EE107AE645C3
:1074B800A8BF67468E45B8BF0F4606EE107AB8EEED
:1074C800C66A062A80ED056A3EF43AAA95ED186A5E
:1074D8009DED145A25EE866AA5EE076AB0EE675A46
:1074E800A6EE265ABDEEC56A16EE10EA16EE107A1A
:1074F800E645A8BF67468E45B8BF0F46FEF7FEB9FA
:10750800664ED4ED017A94ED006A3188726977EE9F
:10751800A77AF0EE006AB0EE677AA6EE267A4E1EDB
:1075280004EBC601D6EE267A08391032F6EE003A98
:1075380027EE237A67EEA37A84ED207AC4ED217AC8
:10754800574C274604F1800091ED027A91ED036AC9
:10755800D7ED036AD7ED027A52ED014A12ED025ACD
:1075680037EE674A76EEC65A77EE277AE4EE845A03
:10757800013EA1F10801E5EE047A07F1080702F1DE
:10758800080236EE267A00F10800E4EE877AE5EE86
:10759800475A67EEA37A25EEA37AC0ED007A80ED0C
:1075A800017AD1D1BEF1140F7EF417AF06F0FCF8C2
:1075B800069BDFF80081C01AA8F80200D4F814511D
:1075C800FEF70BBFD4F81831B4F810C1354ACCF126
:1075D80020095FFA89F90CEB431702EB87075FEA8A
:1075E800990201F0F285013216012F482F4907EB65
:1075F800060807F1100212ED024A12ED035A12EDC5
:10760800016A12ED047A50ED024A50ED035A50ED2A
:10761800016A50ED047A64EE244A65EE255A66EE56
:10762800266A67EE277A1032904541ED024A41ED0D
:10763800035A41ED016A41ED047A00F1100001F1AD
:107648001001D8D11A48A6F110010F4400EB010827
:10765800214419F0030209D0B7EC017AF8EC017A59
:1076680067EE277A013AE1EC017AF5D1BCF1000F17
:1076780041F03180BEF1140F7EF4AFAE06F094F8FD
:10768800069BDFF83080D4F81451C01AA8F802001D
:10769800FEF7A3BE10570020385100209451002057
:1076A800E81D0020AC5100203C530020F81D0020AC
:1076B8002C530020C43F0020D04E318873684FEA15
:1076C80051094FEA89005FEAD10C04EB000204EB90
:1076D800810500F0A18000F110010CF1010CC84FE8
:1076E80002EB0C1C2944103203F1100E05F11000B6
:1076F80050ED032A50ED043A17ED043A17ED032A2A
:1077080050ED026A10ED016A17ED021A57ED010AF1
:1077180011ED044A11ED035A52ED044A52ED035A91
:1077280012ED027A52ED017A51ED021A11ED010AB9
:1077380073EE238A32EE228A47ED048A07ED038A24
:1077480071EE268A30EE868A47ED028A07ED018AB5
:1077580074EE848A35EE858A42ED048A02ED038A46
:1077680077EE218A37EE808A42ED028A02ED018A9D
:1077780073EE633A75EE655A1EED035A32EE623ABD
:1077880074EE644A25EE638A1EED044A23EE052A48
:1077980064EE652AA3EE048A1032944524EE843AF6
:1077A800A3EE842A07F110070EF1100EA5EE853A14
:1077B80000F1100001F11001E4EE852A00ED078ABE
:1077C80000ED082A01ED073A41ED082A5EED055A59
:1077D8001EED065A71EE666A30EEC66A31EEC77A59
:1077E80070EE677A26EE253A65EEE63A25EE674AA8
:1077F80067EE054AE6EE053AA6EE853AA7EE254A73
:10780800E7EEA54A00ED063A40ED053A01ED064AD5
:1078180041ED054A7FF46CAF1FFA89F91A464946CB
:1078280078481EF007F87268494628461EF002F8A4
:10783800059B1A78142A7FF4C1AEB7E6D4F818511C
:1078480071497248724BEA00114415448A881968D4
:1078580000EE102A643AC82AA8BFC822782AB8BFFE
:10786800782207EE902AB8EEC07AF8EEE77A00EBB5
:10787800850577EE670A77EE876A67EE877A20EEE6
:10788800A67AB8EE400AC7EE870A2846D5F81490BB
:10789800D5F81880EF692E6A1EF09AFC059BC5F88A
:1078A800149093F800E0C5F81880BEF1140FEF614A
:1078B8002E6201F0A484D4F81821564BD4F8145140
:1078C800013283FB0213A3EBE27303EB4303D31AE6
:1078D8000135C4F81831C4F8145175E6474E4948C3
:1078E800B268B18928F0E8FF059B93F800E0BEF183
:1078F800140F01F09184D4F814510135C4F81451CF
:10790800FFE5454E31785FEA910C01F0AC85434FB5
:107918000CF101094FEA491907EB090807F12002A0
:10792800A7F1700012ED076A52ED056A12ED037AAD
:1079380052ED017A52ED025A12ED084A52ED064A0A
:1079480012ED045A26EE066A66EEA66A27EE077A54
:1079580067EEA77AA4EE046A20329045E4EEA46AA2
:1079680000F11000A5EE057AE5EEA57AF1EEC65A0B
:10797800B1EEE66AF1EEC76AB1EEE77A40ED085A71
:1079880000ED076A40ED066A00ED057ACAD1A9F153
:1079980020023A4404EB0C1711F0030018BF083218
:1079A8000FD052ED017A12ED027A67EEA77A01380C
:1079B800E7EE077A02F10802B1EEE77AA7EC017A5E
:1079C800EFD1BEF1140F01F00A840135C4F8145147
:1079D800FEF772BC05F0E8FE059B069093F800E000
:1079E800BEF1140F05BFDFF83880D4F81451D4F86D
:1079F8001451A8F80050FDF756B800BF9451002064
:107A0800F81D0020E81D002084540020E84A0020CA
:107A1800544B0020565555558E510020681E0020A5
:107A2800C43F0020306E99BC2716983DA40DC93F6D
:107A3800843459BEDB0F4940D06D393A000000004C
:107A4800F0EEE76AB7EE005A35EE665A1FED0B4ABC
:107A58005FED0B5A1FED0A6A1FED0C7A94ED6B0A65
:107A6800F1EEC54AE6EE845AF5EEC07AA6EEA56AAE
:107A7800F1EE10FAA6EE867A48BF5FED127A27EE8D
:107A8800247A48BF37EEC77A27EE000A2AF022F890
:107A9800B0F5617F00F38D8607EE900AF8EEE76A8D
:107AA8005FED1B7A66EEA76A07EE905ABDEEE67A9E
:107AB800F8EEE77A17EE103A2033402B41F2818432
:107AC8001FED220A2AF006F800B207EE900AB8EE77
:107AD800E77AFFF7BEBAC249C24B89681B68994268
:107AE8003FF696AA3B780C3B022B7EF6A3A9BE4C28
:107AF8003A702378002B3EF49DA900232370FEF7EB
:107B080099B9BA4A02F1500503E00432954200F0EF
:107B180069821378262BF8D19678D3789E42F4D2CE
:107B2800FFF7EDBAB24DB34F95ED004A95ED057AE2
:107B3800D5ED014A95ED066AD5ED046A95ED035A2F
:107B4800D5ED025A67EE897A07EB8602A4EE277A0A
:107B5800A4EEA76A66EEC76AA5EE476AE5EEA76ACD
:107B680020EE070A85ED056AC5ED066A82ED007A02
:107B780029EE088A29F0AEFF69EE288AD5ED0E5A5B
:107B8800D5ED176A95ED091AD5ED121A95ED0F5A2C
:107B980095ED187A95ED0A2AD5ED132A95ED0D6A1B
:107BA800D5ED167A95ED0C3AD5ED0B3A95ED154ACB
:107BB800D5ED144AE1EE085A002207EB8601E8EEFB
:107BC800A16A00B2C4F80021A2EE085AC4F8042140
:107BD800C4F80821A8EEA27A26EE656A67EEE67A6E
:107BE800A3EE655AA3EE886AA6EEC47AE8EEA47AF4
:107BF80085ED0E5AC1ED205A85ED0F6AC1ED406A38
:107C080085ED177AC5ED187AFEF710BBD4F89C51AC
:107C1800079B5D1BFEF710BABBF93820CBF8201084
:107C280007EE902A0121F8EEE77ACBF86020CBF82E
:107C38007C100022012FCBED1C7ACBED1B7ACBF800
:107C4800742001F09D82B7427CF491AFBBF93A20D1
:107C5800CBF8642007EE902A00210122F8EEE77A9B
:107C6800CBF82410CBF890200022012FCBED217AFD
:107C7800CBED207ACBF8882001F08682B7427CF4DD
:107C8800AAAFBBF93C20CBF8682007EE902A002168
:107C98000122F8EEE77ACBF82810CBF8A4200022CE
:107CA800012FCBED267ACBED257ACBF89C207CF4FE
:107CB800C6AF9FED518A032D49D04CB107EE904ACB
:107CC800F8EEE77AF4EEC87AF1EE10FA01F1D08313
:107CD8004A4A4B4C1168DBF86820A8F8060094F86B
:107CE800200102EB560292FBF6F60022CBF8286040
:107CF8008A620A63CA6228B1424A126832F480630F
:107D08007CF4A0AF404A126812F4003241F030828D
:107D18003E481146835C012B02F10C0200F0778388
:107D280001311829F6D1FCF78DBF39494B69002B71
:107D38003DF46DA83748384B008893FBF0F00B688A
:107D48004FF0010E186081F811E0FDF760B8B0EE51
:107D5800480A29F0BFFE00B2AFE711F05FFC2F4AD6
:107D68000292A2F10C03252101930091A2F10A03CA
:107D78005021163A492019F091F8A8B9284BAA7849
:107D880018604FF0FF31596007233B70FFF73DB98A
:107D9800DFF88C8011F042FC224AD8F804301268CF
:107DA80064339342C1F07C83AA78FFF72EB91E4B47
:107DB8001B78D90701F16A831F2027F05FF8002894
:107DC800F2D00C233B70EFE71F20069227F056F8FD
:107DD800069A00287FF419A901233B70FFF715B90B
:107DE8006019002060510020095F0020B062002067
:107DF80018540020AC51002000000000543E002020
:107E0800E81D00201042002040450020D04A030809
:107E1800CC640020E464002020A10700323003086D
:107E28009C600020EC640020673E00201A2027F0A8
:107E380025F800283FF4E6A89B4B1B88002B7FF40D
:107E4800E1A89A4B4520D3F8008022F059FF0E2074
:107E580022F056FF404623F049F8DDF81C804046E2
:107E680023F044F8924A934B12681A6040460A235A
:107E78003B7023F0E5F8FFF7C5B8012A01D1F9F7FF
:107E8800F9FC0D2313203B700EF0FEFAAA78FFF7D9
:107E9800BCB8894B89495B680968C8338B4205D3EC
:107EA80011F0E0FBAA7800283FF4AFA8032A93D189
:107EB800DFF84082D8F800000DF0EAFD804B1B780F
:107EC8000022022BC8F8002001F00384AA7883E777
:107ED800012A01F0D4820E2313203B700EF0D4FA4D
:107EE80062E711F09BFB23F0A3FB00283FF45CAF93
:107EF80011F0B8FB00283FF457AF6D4A6D4B12687C
:107F08001A600A233B70AA78FFF77FB811F086FB46
:107F18006C4B002105208DE80300A3F108020291B3
:107F2800532018F0BBFF00287FF43EAF624BAA78BD
:107F3800186008233B70FFF768B8604B5E491B6800
:107F48004B60614800230B60032103603970FFF721
:107F58005CB8DFED5E7A5E4B94ED687AC3ED007A2B
:107F6800C3ED017AC3ED027A5A4BF0EE674AF0EEA0
:107F7800673A1968FDF746B9574A584DD2ED006A75
:107F8800574A95ED006A1278C4ED646A84ED656A13
:107F9800002A00F01F8276EE665A94F99821C4ED03
:107FA800615A0132C4ED626A00F08985079BC4F802
:107FB8009C31002537EE677AFCEEE77A494E84ED6E
:107FC800687A17EE902AA4F88C21FF2296ED005AC1
:107FD80084F89821FEF740B8434B1D7805F0010856
:107FE800FDF7AEBC3C4A3D4DD2ED007A3C4A95EDDA
:107FF800007A1278C4ED647A84ED657A002A00F07C
:10800800658377EE676A94F99821C4ED616A013255
:10801800C4ED627A00F0DB86079BC4F89C3100252A
:108028009FED2A7A2F4E84ED687AFF2296ED005A4A
:1080380084F89821FEF710B82C49DFED2D7A0968ED
:10804800C4ED4C7A11F080530A9340F0A683DAF815
:10805800001011F480030A9300F0CF8100230A93E3
:10806800B6EE007A67EE877AF4EEE57AF1EE10FA6A
:10807800C8BFF0EE675A40F39083C4ED685AFDF725
:108088000BBB73EEE77AB7EE007AF4EEC77AF1EE3F
:1080980010FAC4ED4C7A41F38F8084EEA77A8DED07
:1080A8000E7AFDF7EEBA00BF105F00200C5F0020CB
:1080B800205F0020185F00209C600020EC640020F6
:1080C80058510020E03103085C3500200000000012
:1080D8001051002018420020385F002094570020DB
:1080E800884D0020A8570020673E0020906000209F
:1080F8000000008060350020D14D0D9B9DED0E5A8B
:1081080095ED006A002B00F01B8725EE866ACD48A6
:10811800A5EE076AB0EE675AA6EE265ABDEEC56A06
:1081280016EE10EA16EE107AE645A8BF67467145C6
:10813800C8BF0F4606EE107AB8EEC66A012A80ED6F
:10814800006A3DF401AC95ED046A9DED0F5A25EEE9
:10815800866AA5EE076AB0EE675AA6EE265ABDEE05
:10816800C56A16EE10EA16EE107AE645A8BF67460D
:108178007145C8BF0F4606EE107AB8EEC66A022AE5
:1081880080ED016A3DF4E0AB95ED086A9DED105A6B
:1081980025EE866AA5EE076AB0EE675AA6EE265A5D
:1081A800BDEEC56A16EE10EA16EE107AE645A8BFCF
:1081B80067467145C8BF0F4606EE107AB8EEC66A24
:1081C800032A80ED026A3DF4BFAB95ED0C6A9DED84
:1081D800115A25EE866AA5EE076AB0EE675AA6EE32
:1081E800265ABDEEC56A16EE10EA16EE107AE64576
:1081F800A8BF67467145C8BF0F4606EE107AB8EEAD
:10820800C66A042A80ED036A3DF49EAB95ED106AB8
:108218009DED125A25EE866AA5EE076AB0EE675AFA
:10822800A6EE265ABDEEC56A16EE10EA16EE107ACC
:10823800E645A8BF67467145C8BF0F4606EE107AE7
:10824800B8EEC66A052A80ED046A3DF47DAB95ED6B
:10825800146A9DED135A25EE866AA5EE076AB0EEFC
:10826800675AA6EE265ABDEEC56A16EE10EA16EE55
:10827800107AE645A8BF67467145C8BF0F4606EEA7
:10828800107AB8EEC66A062A80ED056A3DF45CAB42
:1082980095ED186A9DED145A25EE866AA5EE076AD3
:1082A800B0EE675AA6EE265ABDEEC56A16EE10EA7B
:1082B80016EE107AE645A8BF67467145C8BF0F4657
:1082C80006EE107AB8EEC66A072A80ED066A3DF413
:1082D8003BAB95ED1C6A9DED155A65EE865AE5EEA9
:1082E800075AE6EEA57AFDEEE77A17EE902A94454E
:1082F800A8BF94468A42A8BF614607EE901AF8EED6
:10830800E77AC0ED077AFDF71FBBBEF1010F7FF7D3
:10831800D0AC07EE103AB8EEC77AC7EE876AB1EE6E
:10832800E68AC8E4BEF1010F40F32E8707EE103A43
:10833800B8EEC77AC7EE876AB1EEE68A032D13D086
:108348004CB107EE904AF8EEE77AF4EEC87AF1EE0F
:1083580010FA01F18D80DBF8642002EB560292FBE3
:10836800F6F2CBF8242089E4B0EE480A29F0B2FBF3
:1083780000B2E5E7BEF1010F40F3028707EE103ABD
:10838800B8EEC77AC7EE876AB1EEE68A032D13D036
:108398004CB107EE904AF8EEE77AF4EEC87AF1EEBF
:1083A80010FA01F16580DBF8602002EB560292FBBF
:1083B800F6F2CBF8202046E4B0EE480A29F08AFB12
:1083C80000B2E5E7F7EE006AFDF78EBCF7EE006A4B
:1083D800FDF704BD76EEC65AF0EE466ADDE5822268
:1083E800FDF7E8BFDFED187AFDF7B0BF174BD3F8FC
:1083F80000E0BEF93270FEF75EBAB6EE007AF4EE2F
:10840800C75AF1EE10FA3FF72BAEFDF745B9D4F88D
:1084180024614A003EB1551800EB850576786D78E1
:10842800B542BCF40FAC0A4400EB82000022C4F849
:108438002401A4F81022C4F81422FCF703BC00BFDE
:108448001057002038510020000002431842002035
:1084580095ED006A9DED0E4AE34825EE866AFDEE2D
:10846800E43AA4EE076AB0EE674AA6EE264A13EE8F
:10847800901AB4EEC45AF1EE10FAB0EE446A88BF0E
:10848800B0EE646ABDEEC66A16EE10EA16EE107A11
:10849800E645A8BF67467145C8BF0F4606EE107A85
:1084A800B8EEC66A012A80ED006A3DF449AA95ED46
:1084B800046A9DED0F4A25EE866AA4EE076AB0EEBF
:1084C800674AA6EE264AB4EEC45AF1EE10FAB0EEA8
:1084D800446A88BFB0EE646ABDEEC66A16EE10EA5A
:1084E80016EE107AE645A8BF67468E45B8BF0F4618
:1084F80006EE107AB8EEC66A022A80ED016A3DF4EB
:108508001FAA95ED086A9DED104A25EE866AA4EE2D
:10851800076AB0EE674AA6EE264AB4EEC45AF1EEF0
:1085280010FAB0EE446A88BFB0EE646ABDEEC66A5F
:1085380016EE10EA16EE107AE645A8BF67468E4595
:10854800B8BF0F4606EE107AB8EEC66A032A80ED69
:10855800026A3DF4F5A995ED0C6A9DED114A25EEE8
:10856800866AA4EE076AB0EE674AA6EE264AB4EE1B
:10857800C45AF1EE10FAB0EE446A88BFB0EE646AED
:10858800BDEEC66A16EE10EA16EE107AE645A8BFEA
:1085980067468E45B8BF0F4606EE107AB8EEC66A33
:1085A800042A80ED036A3DF4CBA995ED106A9DED90
:1085B800124A25EE866AA4EE076AB0EE674AA6EE6E
:1085C800264AB4EEC45AF1EE10FAB0EE446A88BFF7
:1085D800B0EE646ABDEEC66A16EE10EA16EE107AC0
:1085E800E645A8BF67468E45B8BF0F4606EE107A27
:1085F800B8EEC66A052A80ED046A3DF4A1A995ED96
:10860800146A9DED134A25EE866AA4EE076AB0EE59
:10861800674AA6EE264AB4EEC45AF1EE10FAB0EE56
:10862800446A88BFB0EE646ABDEEC66A16EE10EA08
:1086380016EE107AE645A8BF67468E45B8BF0F46C6
:1086480006EE107AB8EEC66A062A80ED056A3DF491
:1086580077A995ED186A9DED144A25EE866AA4EE71
:10866800076AB0EE674AA6EE264AB4EEC45AF1EE9F
:1086780010FAB0EE446A88BFB0EE646ABDEEC66A0E
:1086880016EE10EA16EE107AE645A8BF67468E4544
:10869800B8BF0F4606EE107AB8EEC66A072A80ED14
:1086A800066A3DF44DA995ED1C6A9DED154A65EEE7
:1086B800865AE7EE045AE6EEA57AB4EEE75AF1EEEA
:1086C80010FAC8BFF0EE647AFDF72AB977EEC76AE8
:1086D800F0EE477A97E4454A4FEA89075FEA9C0932
:1086E800384402EBC313274437D009F101094FEA94
:1086F800091903EB090803F1100200F1100607F14C
:10870800100112ED024A12ED035A12ED016A12ED40
:10871800047A56ED024A56ED035A56ED016A56EDB3
:10872800047A64EE244A65EE255A66EE266A67EEF8
:10873800277A1032904541ED024A41ED035A41ED46
:10874800016A41ED047A06F1100601F11001D8D151
:10875800A9F110094B4448444F441CF0030C3EF463
:1087680089AFB3EC017AF0EC017A67EE277ABCF1B5
:10877800010CE7EC017AF4D1FEF77CBFBEF8343087
:108788009FED1B7A07EE903AF8EEE77A194B67EE01
:10879800877AC3ED007AFDF725B9B7EE007A77EE50
:1087A800677AF4EEE75AF1EE10FA88BFF0EE675AEE
:1087B80063E407EE905ADFED106AF8EEE77A66EEAA
:1087C800A65A9FED0E5A9FED0E6A9FED0E7AA5EE02
:1087D800856A26EEA55AA5EE867AE5EE076A26EEA4
:1087E800A70AFFF76FB900BF38510020AC5100202D
:1087F8006F12833A0000002084F9223F92E741B9C2
:108808009730083C15A82ABE95ED006A9DED0E4AE2
:10881800CC4825EE866AFDEEE43AA4EE076AB0EE8F
:10882800674AA6EE264A13EE907AB4EEC45AF1EEE1
:1088380010FAB0EE446A88BFB0EE646ABDEEC66A4C
:1088480016EE10EA16EE101AE645A8BF61467745FF
:10885800C8BF394606EE101AB8EEC66A012A80ED7E
:10886800006A3DF4E0AF95ED046A9DED0F4A25EEF0
:10887800866AA4EE076AB0EE674AA6EE264AB4EE08
:10888800C45AF1EE10FAB0EE446A88BFB0EE646ADA
:10889800BDEEC66A16EE10EA16EE101AE645A8BF37
:1088A8006146BE45B8BF394606EE101AB8EEC66A2C
:1088B800022A80ED016A3DF4B6AF95ED086A9DED98
:1088C800104A25EE866AA4EE076AB0EE674AA6EE5D
:1088D800264AB4EEC45AF1EE10FAB0EE446A88BFE4
:1088E800B0EE646ABDEEC66A16EE10EA16EE101A0D
:1088F800E645A8BF6146BE45B8BF394606EE101A20
:10890800B8EEC66A032A80ED026A3DF48CAF95ED95
:108918000C6A9DED114A25EE866AA4EE076AB0EE50
:10892800674AA6EE264AB4EEC45AF1EE10FAB0EE43
:10893800446A88BFB0EE646ABDEEC66A16EE10EAF5
:1089480016EE101AE645A8BF6146BE45B8BF3946BF
:1089580006EE101AB8EEC66A042A80ED036A3DF4E2
:1089680062AF95ED106A9DED124A25EE866AA4EE77
:10897800076AB0EE674AA6EE264AB4EEC45AF1EE8C
:1089880010FAB0EE446A88BFB0EE646ABDEEC66AFB
:1089980016EE10EA16EE101AE645A8BF6146BE4567
:1089A800B8BF394606EE101AB8EEC66A052A80ED39
:1089B800046A3DF438AF95ED146A9DED134A25EE2F
:1089C800866AA4EE076AB0EE674AA6EE264AB4EEB7
:1089D800C45AF1EE10FAB0EE446A88BFB0EE646A89
:1089E800BDEEC66A16EE10EA16EE101AE645A8BFE6
:1089F8006146BE45B8BF394606EE101AB8EEC66ADB
:108A0800062A80ED056A3DF40EAF95ED186A9DEDD6
:108A1800144A25EE866AA4EE076AB0EE674AA6EE07
:108A2800264AB4EEC45AF1EE10FAB0EE446A88BF92
:108A3800B0EE646ABDEEC66A16EE10EA16EE101ABB
:108A4800E645A8BF6146BE45B8BF394606EE101ACE
:108A5800B8EEC66A072A80ED066A3DF4E4AE95EDE5
:108A68001C6A9DED154A65EE865AE7EE045AE6EE55
:108A7800A57AB4EEE75AF1EE10FAC8BFF0EE647AC0
:108A8800FDEEE77A17EE901A8C45A8BF8C468F4208
:108A9800D8BF674607EE907AF8EEE77AC0ED077A16
:108AA800FDF7BEBE28494A69002A3CF499AA0A681B
:108AB80013604B74FCF794BA244DFDF70BB8D4F847
:108AC8009C51079B5D1BFFF775BA214B1B78DA0792
:108AD80004D41BF0EFF9002840F068851D4DD4F848
:108AE8000C222B689A423EF69AAA3B78012B3DF459
:108AF800A1A9194C2278002A3DF49CA90B2B19D85E
:108B080001229A4040F6030112EA01087EF4F5AF0B
:108B180012F4C06F0ED0093B012B0BD8452022F070
:108B2800EFF8FF2022F0ECF80C4822F05FF84046FE
:108B380022F0E6F80A4B2A685A600B233B70FEF7CE
:108B4800DCBF00BF38510020CC640020E83F002083
:108B5800673E0020EC640020095F002008590308E4
:108B68009C6000200D9B002B00F07183E34D9DED70
:108B78000E4A95ED006A089B25EE866AA4EE076A00
:108B8800B0EE674AA6EE264AB0EE446A33B1B4EEB8
:108B9800445AF1EE10FAC8BFB0EE646AFDEEE44A3A
:108BA800BDEEC66A14EE907A16EE101A8F4214EED5
:108BB80090EA00F3F3846145A8BF614606EE101AF7
:108BC800CF48B8EEC66A012A80ED006A3CF4BCAE14
:108BD80095ED046ADDED0F4A089B25EE866AA4EE42
:108BE800876AF0EE674AE6EE264AB0EE646A002B22
:108BF80000F0CA84B4EEE45AF1EE10FA40F3C484EB
:108C080039466145A8BF614606EE101AB8EEC66A35
:108C1800022A80ED016A3CF497AE95ED086ADDED15
:108C2800104A089B25EE866AA4EE876AF0EE674A2A
:108C3800E6EE264AB0EE646A002B00F09B84B4EEA0
:108C4800E45AF1EE10FA40F3958439466145A8BF1D
:108C5800614606EE101AB8EEC66A032A80ED026A6B
:108C68003CF472AE95ED0C6ADDED114A089B25EED9
:108C7800866AA4EE876AF0EE674AE6EE264AB0EE08
:108C8800646A002B00F06C84B4EEE45AF1EE10FA3A
:108C980040F3668439466145A8BF614606EE101A5E
:108CA800B8EEC66A042A80ED036A3CF44DAE95ED31
:108CB800106ADDED124A089B25EE866AA4EE876AE3
:108CC800F0EE674AE6EE264AB0EE646A002B00F042
:108CD8003D84B4EEE45AF1EE10FA40F33784394695
:108CE8006145A8BF614606EE101AB8EEC66A052AA5
:108CF80080ED046A3CF428AE95ED146ADDED134A64
:108D0800089B25EE866AA4EE876AF0EE674AE6EECF
:108D1800264AB0EE646A002B00F00E84B4EEE45AE2
:108D2800F1EE10FA40F3088439466145A8BF614660
:108D380006EE101AB8EEC66A062A80ED056A3CF4FB
:108D480003AE95ED186ADDED144A089B25EE866A98
:108D5800A4EE876AF0EE674AE6EE264AB0EE646A49
:108D6800002B00F0E083B4EEE45AF1EE10FA40F381
:108D7800DA8339466145A8BF614606EE101AB8EE97
:108D8800C66A072A80ED066A3CF4DEAD95ED1C6ADA
:108D9800DDED154A089B65EE865AE4EE875AE5EE46
:108DA800A67A002B00F0B783F4EEC57AF1EE10FA3C
:108DB80040F1B1833A466245A8BF6246964607EE3F
:108DC80090EAF8EEE77AC0ED077AFCF7BDBDD4F873
:108DD8009C51079B5D1BFFF723B907EE905ADFED07
:108DE800496A9FED497A84F80452F8EEE77A67EE0B
:108DF800A67A77EE876ABDEEE66A16EE103A203359
:108E0800402B40F29782DFED416A414BBDEEE77A95
:108E1800C3ED016A17EE103A2033402B00F260824E
:108E28009FED3C7AF4EEC77AF1EE10FA40F3CA836C
:108E3800DFED395A9FED396A01E0F0EE477AF4EE3A
:108E4800C67AF1EE10FA37EEE57AF6DCDFED347A21
:108E5800B4EEE77AF1EE10FA40F1B183DFED2E5A65
:108E68009FED306A01E0B0EE677AB4EEC67AF1EEB3
:108E780010FA77EE257AF6D49FED237AF4EEC77AC6
:108E8800F1EE10FA40F3E3829FED227A77EE677AEB
:108E980067EEA75A9FED245A9FED246A9FED247A26
:108EA800A5EE856A27EEA55AA5EE867AE5EE077A3D
:108EB800C4ED827AFDF77ABD95ED000A0893069213
:108EC80028F008FE1B49DFF870E0D1F8EC10DFF855
:108ED8006CC0069AACF800008EFB013EC917C1EBC6
:108EE800AE1107EE901AF8EEE77A089BFDEEE77AE6
:108EF80017EE901AACF80210FCF7F1BD10570020DD
:108F08003851002035FA8E3CDB0FC93F00000000C5
:108F180000000020DB0F4940DB0FC940E4CB1641BD
:108F2800DB0F49C0E4CB16C192E741B99730083C42
:108F380015A82ABE540F0020D34D6210C43F00204C
:108F480025EE866AA5EE076AB0EE675AA6EE265A9F
:108F5800BDEEC56A16EE100A814200F36C816045C9
:108F6800A8BF604606EE100A0A9BB8EEC66A002B38
:108F780000F0FF83DC48012A80ED006A3CF4E4AC91
:108F880095ED046A9DED0F5A25EE866AA5EE076AEF
:108F9800B0EE675AA6EE265ABDEEC56A16EE107AEE
:108FA800B94200F346816745A8BF674606EE107AC6
:108FB8000A9BB8EEC66A002B00F09883022A80ED5F
:108FC800016A3CF4C1AC95ED086A9DED105A25EE96
:108FD800866AA5EE076AB0EE675AA6EE265ABDEE77
:108FE800C56A16EE107AB94200F32D816745A8BF0D
:108FF800674606EE107A0A9BB8EEC66A002B00F0A8
:109008009383032A80ED026A3CF49EAC95ED0C6ACA
:109018009DED115A25EE866AA5EE076AB0EE675AED
:10902800A6EE265ABDEEC56A16EE107AB94200F3CE
:1090380008816745A8BF674606EE107A0A9BB8EE16
:10904800C66A002B00F06683042A80ED036A3CF4AC
:109058007BAC95ED106A9DED125A25EE866AA5EE59
:10906800076AB0EE675AA6EE265ABDEEC56A16EE36
:10907800107AB94200F3E3806745A8BF674606EE59
:10908800107A0A9BB8EEC66A002B00F0B182052A56
:1090980080ED046A3CF458AC95ED146A9DED135AC2
:1090A80025EE866AA5EE076AB0EE675AA6EE265A3E
:1090B800BDEEC56A16EE107AB94200F3BE80674568
:1090C800A8BF674606EE107A0A9BB8EEC66A002B60
:1090D80000F01683062A80ED056A3CF435AC95ED60
:1090E800186A9DED145A25EE866AA5EE076AB0EE59
:1090F800675AA6EE265ABDEEC56A16EE107AB94230
:1091080000F3A3806745A8BF674606EE107A0A9B5E
:10911800B8EEC66A002B00F07582072A80ED066A51
:109128003CF412AC95ED1C6A9DED155A65EE865A15
:10913800E7EE055AE5EEA67AFDEEE77A17EE902AF5
:10914800914203DC6245A8BF6246114607EE901AB9
:109158000A9BF8EEE77A002B7FF435AE0C9B002BC8
:109168007FF431AE0B9B9E45B8BFF0EE647A2AE6D9
:109178005E4A1278032A00F015820022FEF7C8BD65
:109188009FED5B8AFFF702B99FED598AFFF7D6B8C2
:109198009FED580ADFF8708125EE800A28F09AFCC6
:1091A800D4F81451A8F80600FDF717B9D4F89C5163
:1091B800079B5D1BFDF7C0BF4F49096811F080533D
:1091C8000A937EF44DAFFEF742BF4C484C498046A7
:1091D800FEF73FBA079821F033FFFDF713BF04F0FD
:1091E800E3FA059BDFF8208193F800E0069B3178CD
:1091F800D4F81451C01AA8F80400FEF7E6BB04F02E
:10920800D3FA059BDFF8008193F800E0069BC01AAB
:10921800A8F80200FEF74FBB04F0C6FA059BDFF87A
:10922800E88093F800E0069BC01AA8F80200FEF751
:1092380062BB0F46BAE6084694E60F4642E70F4679
:109248001DE70F46F8E60F46D3E60F465DE70EA981
:10925800BDEEE46A01EB820290462A48089A224D44
:109268000A9B089416EE107A05E04145A5EC016AC0
:1092780000F1100031D090ED006AB1EC014A25EE02
:10928800866AA7EE046AB0EE674AA6EE864AB0EE92
:10929800446A32B1B4EE445AF1EE10FAC8BFB0EEE7
:1092A800646ABDEEC64A06EE107A14EE104AA7426A
:1092B80006DC14EE104A6445A8BF644606EE104A60
:1092C800B8EEC66A002BD0D10C9C002CCDD10B9CDB
:1092D800A645B8BFB0EE646AC7E7089CFCF734BB84
:1092E800DFED037AE4E500BF38510020A8380020FC
:1092F800000000000000C842906000202C530020AD
:10930800E81D002010570020C43F002092E741B913
:109318009730083C15A82ABEE4CB1641DB0FC9409C
:10932800E4CB16C1DB0FC93FDB0F4940DB0FC9BFD8
:10933800DB0F49C0F4EEC77AF1EE10FA40F355811D
:109348005FED0A5A1FED0C6A01E0F0EE476AF4EE91
:10935800C66AF1EE10FA36EEE57AF6DC5FED0C6AD5
:10936800B4EEE67AF1EE10FA40F12F815FED155A6E
:109378001FED156A01E0B0EE667AB4EEC67AF1EE3A
:1093880010FA77EE256AF6D41FED1A7AF4EEC76A5A
:10939800F1EE10FA40F3B3801FED1D7A77EE666A9E
:1093A80066EEA65A1FED275A1FED276A1FED277A8A
:1093B800A5EE856A26EEA55AA5EE867AE5EE076A39
:1093C80023E51FED277AF4EEC76AF1EE10FA40F3B1
:1093D8008A815FED2E5A1FED306A01E0F0EE476A90
:1093E800F4EEC66AF1EE10FA36EEE57AF6DC5FEDD9
:1093F800306AB4EEE67AF1EE10FA40F171815FED71
:10940800395A1FED396A01E0B0EE667AB4EEC67AD1
:10941800F1EE10FA77EE256AF6D41FED3E7AF4EEF7
:10942800C76AF1EE10FA05DD1FED417A77EE666A3C
:10943800FFF7C5B91FED437AF4EEC76AF1EE10FAEB
:1094480044BF1FED457A77EE666AFFF7B8B91FED9E
:10945800497AF4EEC77AF1EE10FA44BF1FED4C7A60
:1094680077EE677A14E5C84F07F18002FEF794BAE1
:10947800A8F80600ABF8A860C34CFBF7EABBF7F7FF
:10948800D9FF00283EF490ACFEF725BD802026F0D9
:1094980041FD08B10CF028FB17F054FEFEF78CBC18
:1094A800402010F093F800287EF47EACD8F8003005
:1094B800DFF814A3DFF814B34FF040090EE021F0F1
:1094C8001FFCDBF80020D8F80030013A0133B9F16D
:1094D8000109CBF80020C8F8003079D01AF8033019
:1094E8001846002BEBD100234FF0FF32C8F80030AC
:1094F8000423C8F804203B70AA78FDF786BD9FEDC9
:10950800A37AF4EEC76AF1EE10FA44BF9FEDA07A91
:1095180077EE666A44E7FDEEE77A17EE902ABA42DC
:10952800FFF64DAC47E4BDEEC66A16EE101AB94216
:10953800BFF620AC394620E4BDEEC66A16EE101A16
:10954800B942BFF6F2AB3946FFF7F2BBBDEEC66AC9
:1095580016EE101AB942BFF6C3AB3946FFF7C3BBC4
:10956800BDEEC66A16EE101AB942BFF694AB39467C
:10957800FFF794BBBDEEC66A16EE101AB942BFF6E5
:1095880065AB3946FFF765BBBDEEC66A16EE101A25
:10959800B942BFF636AB3946FFF736BB14EE901A20
:1095A800FFF70CBB0CF054FFFBF74CBB794B1B6867
:1095B80003F59C530833C4F80C32FDF730BDF0EEC8
:1095C800477A59E4B0EE677A40E4F0EE476ADBE6A2
:1095D8001AF80330002B7EF4E7AB84E794F878316F
:1095E800002B7BF4CBADFBF7B6BDB0EE667AB5E6E3
:1095F8000C9B002B7FF44BAD0B9B9E45B8BFB0EE88
:10960800646A44E50C9B002B7FF487AD0B9B9E4559
:10961800B8BFB0EE646A80E55F4A604B10681B68AB
:1096280098475F4BD7ED006A93ED007A5D4BD3ED19
:10963800007A5D4B83ED020A5C4B67EE277A2B4478
:1096480027EEAC7AD3ED007A594B67EE277AF0EE25
:10965800665AEDEEA75A93ED006AB1EE467AB4EE7B
:10966800E57AF1EE10FA08DCF4EEC65AF1EE10FADB
:109678008CBFB0EE467AB0EE657A4E4B1B78012B64
:1096880002D0192B7BF4E4ACDFED4B7AF4EEE7DA89
:10969800F1EE10FACCBF01230023FBF7E4BC474BE3
:1096A800D3ED007AB1EE677AF4EEC7DAF1EE10FA8C
:1096B80013D4F4EEE7DAF1EE10FA88BFF0EE67DAC9
:1096C8003F4B87ED00CA1B689342BBF6AFABFBF775
:1096D80013BC0CF017FEFEF7F9BBF0EE47DAEFE724
:1096E800F0EE476A99E6B0EE667A80E60C9B002BAE
:1096F8007FF464AC0B9B9E45B8BFB0EE646A5DE432
:109708000C9B002B7FF4E6AC0B9B9E45B8BFB0EEDC
:10971800646ADFE40C9B002B7FF496AC0B9B9E45A0
:10972800B8BFB0EE646A8FE40C9B002B7FF469AC81
:109738000B9B9E45B8BFB0EE646A62E4132B05D15B
:10974800B0EE480A28F0C6F9099B1880B0EE480A1E
:10975800DBF808321B489847059B1B78132BB0EEA3
:10976800408A7CF4F2AE28F0B5F9099B5880FCF7E2
:10977800ECBE0C9B002B7FF4FDAB0B9B9E45B8BF4A
:10978800B0EE646AFFF7F6BBE81D0020DB0FC9BF27
:10979800DB0F49C0EC6400207C5600209056002066
:1097A80000000020D055002004510020A0560020C1
:1097B8000857002034550020000096420457002026
:1097C800E8560020E84A0020CC2F03085C3500202A
:1097D8002DE9F04F2DED068BA04BA14A1C7897B0D0
:1097E80000F59C41203181460B911160002C00F05E
:1097F800EA869C4A1268904240F283809A4A06920E
:1098080016689A499A4A0591013C1C70994B049232
:1098180006F480560893002E40F08180964B1B7802
:10982800022B01F08081042B01F06F81012B01F0E4
:109838002381924B9945089B9B7800F29585002BD4
:1098480040F096858E4B0793069B1E6816F480574A
:1098580040F08786DFF860A2049BB3F90610059BE9
:109868005D8BA942B4BF00250125864B1B6813F008
:1098780080535ED0079A127812F001025FD00598E3
:10988800408C884241F3A482002D5ED17E4C94F82E
:109898008C10002959D17D487D49006890F82D0029
:1098A80000240C604C608C607A4900284ED1087006
:1098B800002A4FD0F0064DD5774A1278D10649D400
:1098C800002F47D1002B45D1720243D4734B1B782C
:1098D800002B02F07F81724B9B78002D42F023828F
:1098E8003BB1704A704B12681B689B1A002BC2F27E
:1098F80045821020644C0CF0C7FD012384F88D309C
:1099080028E0594B06931E68594B584A049306F4AD
:109918008056584B05920893002E3FF47FAF0021E4
:109928005848F7F721FD00287FF478AF0DF080FC48
:1099380074E774029ED4079A127802F00102524C1E
:10994800002184F88C10002DA5D052490120087000
:10995800002AAFD1554B1A78002A40F0BD800599EE
:10996800049C488BB4F90070898BB4F90240B84262
:10997800B4BF8026002646F04003B942D8BF33461C
:109988009B0843F08006A042B8BF3346049F43F0CB
:109998004006A142C8BF33469B08B7F90440B7F94F
:1099A800066043F08007A042B8BF3B4643F040073B
:1099B800A142C8BF3B469B0843F08007324C864211
:1099C800C8BF3B4643F0400794F88EE08E42B8BFCC
:1099D8003B469E4501F03684A4F8902084F89220F6
:1099E8002E4984F88E300E78002E01F037835F2BD5
:1099F80001F0AA836F2B01F0E983079B1B78DE0730
:109A08006AD494F89210002966D1B4F99030322BB8
:109A180062DD94F88E200120572A84F892004DD0F8
:109A2800069B1B685D0741F185825A2A41F08282B4
:109A380094F89430002B42F0518194F8963083F0DA
:109A4800010384F89630002B42F051810C200CF071
:109A58001BFD174B174D099341E000BFF05C002038
:109A6800F85B0020EC5C0020644B0020705900205B
:109A780092710020C04200205A5C0020404B4C00EC
:109A8800673E00209060002004200020184200203B
:109A980010510020601F0020845100209C1B0020D2
:109AA800EC600020EC640020603300202F4300208D
:109AB8001C4200201442002000630020874B884A83
:109AC80019684FF47A73B3FBF1F3C3EB431103EB5B
:109AD8008103DB00A2F8A830824B834D0993069BD3
:109AE8001B685F0700F1A5860DF150097F4E0A95A6
:109AF8000022C9F804203446149240F6330B4FF084
:109B0800190840F28337049D02E00434544520D0FC
:109B1800A178E378994218FB0170F6D26178043194
:109B280018FB037335F911105945A8BF5946B1F50B
:109B3800617FB8BF4FF461718142E6DD9942E4DC90
:109B480021782729E1D848460434F7F7FDFB544526
:109B5800DED1674A0A9D1378664A99E8030082E8CD
:109B68000300002B40F0F285634B1A78002A00F0BE
:109B78006C8501215F48F7F7F7FB002840F0E78282
:109B8800089BDB78002B40F0E2825C4B0A932B8821
:109B98001FB227F001071FFA87F84345A5F8008090
:109BA80000F0F087564F4FF002090E204FF0140ACC
:109BB8004FF0FF0B87F8009087F801A087F802B0F4
:109BC8000CF062FC49464B48B5F80080F7F7CCFB2F
:109BD800002841F0888228F002039BB243452B807D
:109BE8000BD0474B02201421FF2218700E20597009
:109BF8009A700CF049FCB5F80080424B424A19783B
:109C080050680B9318F0030F08BF81F00201C1F3ED
:109C180040010C9207F03EFC24213648F7F7A4FBDC
:109C280030B9079A13785F0744BF23F00403137011
:109C38000A9B1B6813F00A0F11D006212D48F7F76D
:109C480093FB002801F09B802B88580641F1138272
:109C580007212848F7F788FB002840F0B6870C2131
:109C68002448F7F781FB2A88002800F0518342F442
:109C780080739A422B8009D0214B022214211A703A
:109C88000E20FF2259709A700CF0FEFB1F4B1B78B8
:109C9800082B00F049830E2B00F04683069BD3F86F
:109CA800008018F4806F6BD0194B1B79002B00F0E3
:109CB800308214210F48F7F757FB002840F02E8216
:109CC80010F0D2FB01200CF0E7FA002855D0DFF89D
:109CD80044A000274FF0CC0BA14620E0544B0020B5
:109CE800DC4800201C42002014420020B062002002
:109CF800884D0020906000205D420020C041002077
:109D08007C460020B4640020B8640020785100200C
:109D1800D83F00209C6E0020DFB2022F2CD80BFB0E
:109D280007F87B1C5AF80840002CF5D1032290F95B
:109D3800023002940192C278E24951F8222000923E
:109D480018462246234601210BF0E6FE034607EBA0
:109D5800470000EB00100A9353B121460AEB80003C
:109D6800CC2228F072FE0A9B4AF808300137FFB26D
:109D78001CF0E4FD0028D0D14C46069BD3F80080A7
:109D8800079B93F800A0D04B1AF0010A00F041821B
:109D980001221A70099B04991B68B1F906105A89A7
:109DA800CA4801279142077080F21982C84B4FF0C8
:109DB8007E521A60059BC74FB3F81890049B97F919
:109DC8000420B3F90030387897F801C0002AA3EBD3
:109DD800090714BF01224FF0FF32002FB8BF7F429E
:109DE800B7F5FA7FA8BF4FF4FA77B84280F2F4814A
:109DF8003F1A07EE907AF8EEE77AB74F4B45C7ED72
:109E0800007A03DAF1EE677AC7ED007A049BB3F9BA
:109E180002E0AEEB0903002BB8BF5B42B3F5FA7F53
:109E2800A8BF4FF4FA73984280F2D3811B1A07EE49
:109E3800903AF8EEE77AF145C7ED017A03DDF1EEE5
:109E4800677AC7ED017A049BB3F90400A0EB090314
:109E5800002BB8BF5B42B3F5FA7FA8BF4FF4FA7383
:109E68006345CCBFA3EB0C03002302FB03F207EE10
:109E7800902AF8EEE77A4845C7ED027ABCBFF1EEC2
:109E8800677AC7ED027A18F4805800F07F81B1F53F
:109E9800FA6F924BA8BF4FF4FA61B1F57A7F1A783E
:109EA800B8BF4FF47A71A1F57A71002A41F00B819D
:109EB8008B4ADFF844E282FB0130CB17C3EB601317
:109EC800581C6FF0630C3EF910003EF913E00CFBD0
:109ED8000313A0EB0E0003FB00F382FB0312DB1756
:109EE800C3EB62139E440FFA8EFE07EE90EAB8EEBB
:109EF800E78A87ED038AB8F1000F40F059842B8870
:109F08005A0640F1FB807749774A91ED018AD2EDF4
:109F1800019A92ED026A91ED034A92ED030A91EDDE
:109F2800029A92ED007AD1ED005AD7ED011A97ED19
:109F3800002A6E4A6E4938EE445A79EEC63A77EEF0
:109F4800007A65EE233A75EEC96A75EE890A37EE2E
:109F5800401A66EEA76AB0EE633AA0EE813A13F0B3
:109F68000303B0EE665A78EE044A79EE867AA0EEDC
:109F7800815AF0EE638AA4EEA73AD4EEA78AA4EE3B
:109F8800E75A33EE263AF0EE687AF0EE674AF6EED4
:109F9800008A35EE88AAE0EEC14A28EEC33A35EECB
:109FA800635A77EE293A77EEE67AAAEE233A25EE57
:109FB800285A76EE403A34EE49AAE0EE817A74EEF9
:109FC800A64AAAEE235A34EE094A37EE697A64EEB5
:109FD800A84A63EE036AE4EE074A75EEC85A36EEFD
:109FE800006A67EEA87AB0EE667A95EE057AE5EE35
:109FF800056AE5EE867AB1EE648AF0EE665AF0EE0E
:10A00800476AB1EE674AE8EE246A63EE270A67EE0C
:10A01800A43AE4EE275AB1EE450AB0EE606AB0EE13
:10A02800631AA4EE277A23EE244AE7EEA76AA5EE80
:10A03800246AA0EE031AE8EE245AB0EE448A31EE00
:10A04800A19AE0EE240AA5EE278A66EEA16A72EECE
:10A05800028AE5EE033A61EE211A26EE096AA4EEB9
:10A06800A47AA0EE274A0CBFD7ED022ADFED212AF9
:10A0780082ED005AA2EE256AE8EEA06AE2EE081A1E
:10A0880073EEA33A27EE227A34EE044AF0EE005A31
:10A09800E3EEA26AA2EE846AA1EEA57AC7ED016A90
:10A0A800C1ED366A81ED356A87ED006A81ED377A50
:10A0B80082ED013AC2ED027AC2ED034AF3B987EDA7
:10A0C800027A1BE038450308683E0020981F0020EC
:10A0D800141F0020C4600020E83F00209C240020BA
:10A0E8001F85EB51E0000020541B00208C1B002032
:10A0F80004200020000000006C650020BAF1000F69
:10A1080040F0258125F00CF917B0BDEC068BBDE8B1
:10A11800F08F079B1B78D9077FF5D2AD4FF40F70EE
:10A1280025F0F8FE00283FF428AE0BF0DDFC4FF4D4
:10A138000F7025F091FE00283FF41FAE0BF0D4FC01
:10A148004FF40F7025F088FE0028EED115E69B4BE2
:10A158000A931B689B077FF51AADB5F8008018F0C5
:10A16800010F7FF438AD48F0010398452B803FF488
:10A1780032AD934B022214211A700E20FF2259701F
:10A188009A700CF081F9B5F8008024E5059B5A8B8C
:10A198009142C0F2F484B1F5FA6FD4BFC2EB010169
:10A1A800C2F5FA614FF47A7303FB01F1854803782D
:10A1B800C2F5FA62B1FBF2F1002B3FF479AE4378B5
:10A1C800814A01FB03F182FB0123C917C1EB63112B
:10A1D8006EE6DFED7E7A2EE6DFED7C7A0DE6B1F5F0
:10A1E800FA6F80F2C584187A8B1A03FB00F3C2F564
:10A1F800FA6293FBF2F3C3F1640307EE903AF8EEC8
:10A20800E77A9FED737A734B67EE877AC3ED007A2E
:10A21800D0E51B780693002B7FF4BCAD6E4A12681C
:10A22800002A3FF4B7AD6D4A079212F8030CDFF825
:10A23800E4B11146D71E24F0F7FD9BF80090079A69
:10A24800002800F01E86069BB9F1000F41F06D84CE
:10A2580007F10801787924F0E7FD002841F0968499
:10A268005F49B87A24F0E0FD002800F01D86B9F1B6
:10A27800020F41F087845B49F87B24F0D5FD002864
:10A2880041F07C845849387D24F0CEFD002800F048
:10A298001D86B9F1040F41F06D845449787E24F08D
:10A2A800C3FD002841F062845149B87F24F0BCFD09
:10A2B800002800F01D86B9F1060F41F053844D497E
:10A2C80097F8230024F0B0FD002841F047844A495C
:10A2D80097F8280024F0A8FD002800F01D86B9F1A1
:10A2E800080F41F03784454997F82D0024F09CFD6C
:10A2F80000283FF44FAD0922134602EB82021744AF
:10A308003F4A7878B9788BF800301070517041E581
:10A3180022F480739BB29A422B807FF4ADAC394B08
:10A328001B78082B7FF4B7AC2A8822F040039BB235
:10A338009A422B803FF4B2AC214B022214211A70AE
:10A348000E20FF2259709A700CF09EF8A6E40B9B21
:10A3580019780C9B01F00101186807F09BF817B0F9
:10A36800BDEC068BBDE8F08F13B9089A01239370F2
:10A37800254B089A1D7892F8214007931B2024F05A
:10A388007DFD012C05F00108814600F0F68605F0F8
:10A398000205089A1D4E92F82030DFF87CA01C4F69
:10A3A80009959346052B00F28B87DFE813F0BF0071
:10A3B800B5003700FD00FF00F20000BFC0410020DB
:10A3C8007C4600209C2400201F85EB5100000000E3
:10A3D8000AD7233C141F00206C3E0020364600207C
:10A3E80040460020454600204A4600204F460020AF
:10A3F80054460020594600205E460020634600204F
:10A40800703E002078510020673E002064650020DF
:10A4180010420020080000209C1B0020012C04BFD3
:10A4280005238BF82030B8F1000F12D0059B308837
:10A43800B3F918100022134661F30F0260F31F42AC
:10A4480061F30F03049861F31F4303600323426021
:10A458000993BF4DDBF814102A68914280F0EE850D
:10A4680047F230510322CBF81C108BF82020022031
:10A4780008F038FB0CF0DCFE2968DBF81C200A44E5
:10A488000421CBF818208BF82010012C40F06987A4
:10A498002A68DBF81810914280F012879AF80000B9
:10A4A80020B924F0EBFC002840F00A873A6822F033
:10A4B80002023A602A687388642101FB03234FF47F
:10A4C80080600022CBF810308BF820208BF8032016
:10A4D80008F0D8FA9BF8203064E724F0D5FC01286E
:10A4E80007D19B4D72882B68642101FB0233CBF89E
:10A4F8001030B9F1000F02D0B379002B4BD1012CE9
:10A5080000F0DE86924DDBF810102A689142C0F008
:10A518001D8701238BF82030012C3AD0F379012BC9
:10A5280046D024F03FFC9BF820303BE7B8F1000F01
:10A53800D3D1099D4FF48060B9F1000F00F0428338
:10A5480008F0B8FA089A00231361002D3FF47CA99B
:10A5580028460BF099FF069B1E6816F480573FF4B7
:10A5680079A91D217B48F6F7FFFE00287FF472A920
:10A57800794B03F1500A03E004339A4500F0A686AC
:10A588001A78262AF8D19978DA789142F4D2FFF726
:10A5980063B96F4D8EE724F005FC03224FF47A73FC
:10A5A8008BF82020CBF81C30694D60E7684D6CE7CC
:10A5B80024F0F8FB032240F6B8338BF82020CBF8C0
:10A5C8001C30634D53E7654F3B78002B01F019822F
:10A5D800634BDFF89881DFF898B1DFF898A105930D
:10A5E80045465E46049099460EE019F804109847CF
:10A5F800032C28DC88B93B782AF8020F01349C42E6
:10A6080005F1040580F23A81072CE1B23046DBF807
:10A618000430EADD984700B2EDE738F824206B886B
:10A62800801A4FF47A719B1A01FB00F040F6CA02B7
:10A6380090FBF3F00844904240F2EE23A8BF104686
:10A648009842B8BF184600B2D5E7DFF82C91DFF87A
:10A658002CA1444F0A9209F15A084FF0010B4946C0
:10A6680019F8010C24F0E0FB00B399F8040099F8FC
:10A67800023099F803E000EB400107EB8101013B50
:10A68800D1F8A02003EB4303534493420ED097F82C
:10A69800CC20C1F8A0300BFA00F022EA00000A9B97
:10A6A80081F89CE0C1F8A43087F8CC0009F10609CC
:10A6B800C145D4D12C4B264A1B780A93099BDFF855
:10A6C800C0A012681B680B93AAF19C094FF0000BFD
:10A6D8009046DAF8043083B31F7877B3DAF80820A5
:10A6E800A8EB0202002A0CDB99F8CC20012101FA20
:10A6F8000BF122EA010208F5FA7189F8CC20CAF8B0
:10A7080008100A9ACAB19AF8002059780432D2B2CD
:10A71800002940F0A18305990498098B30F912208B
:10A7280001F1C800824240F3E38599F8CC109A7889
:10A7380041FA0BF3D80740F16D860BF1010BBBF121
:10A74800040F0AF10C0AC4D1FFF713BA024B1DE03B
:10A75800EC64002090600020B06200207463002048
:10A768007059002004200020E93700208C63002065
:10A77800A8420020022000204D4500200032030896
:10A78800A02000200433A3423FF4EEA9197823291E
:10A79800F8D19878DA789042F4D2A548F6F7E4FD33
:10A7A80000283FF4E1A914200BF06EFEFFF7DCB996
:10A7B8001D219F48F6F7D8FD28B100F05BBD04368F
:10A7C800A6423FF49CAB31782629F8D1B278F378C9
:10A7D8009A42F4D2089BDB78002B7FF490AB944824
:10A7E800F6F7C2FDDFED937A002801F00E8138EE0E
:10A7F800678A914A9149FDEEC87ACDED047ABDF990
:10A8080010301B0382FB0302DB17C3EBA212C9F54E
:10A818007A731BB203FB02F343F30F334B4407EE87
:10A82800903AF8EEE77A0123C7ED037A0B70FFF749
:10A8380066BB834C94F896305BB1079B1B78DE07A8
:10A8480007D5049BB3F90620059B5B8B9A4200F35E
:10A85800D38511217648F6F787FD002800F0A682F7
:10A8680094F89A302BB994F8943013B93223A4F899
:10A878009830012384F89A30FFF736B9DDF8109044
:10A88800704A06926C49126842F2010AA1FB091B40
:10A8980012EA0A0A4FEA9B1B00F085826A4D6B4850
:10A8A8006B4C6C492E780078267008701EB1694987
:10A8B8000E7886F00106624C0F2184F82410002BD4
:10A8C80000F0E183059D644BB5F826C0B5F824E097
:10A8D800059D109318462D8B0078604B129594F8BF
:10A8E800255009955E4D0495A3FB00535B0803EBC7
:10A8F8004303C31ADBB20F90CDF834C002F4805280
:10A908000C9304F128000BF59673CDF8449097F852
:10A918000080DDF82490DFF858C10994504C0E915E
:10A92800139200210A930896CDF81CE0089B002B8F
:10A9380000F02683099B079D33F911201FFA82FE38
:10A94800AE454FEA410303D30D9DAE4540F25D830A
:10A958005CF82120934580F01D83E25EBAF1000F78
:10A9680040F0328301314145E25200F10600DDDB5F
:10A978000E9A099C3B4B84F824200F2A49460CBFA9
:10A9880001220022DDF8449084F825101A7000F0A6
:10A998008183354B2D492F4ADFF8D8B008931C46E0
:10A9A800042001230B70137008F09CF8DBF80030CA
:10A9B800A1686268E3605B1A934284BF002384F84D
:10A9C8002130069B3C781E68002C01F07B80059A9C
:10A9D800264DB2F824E0178B214916F480562846F4
:10A9E80040F0948332460EE0437803EB830303EB95
:10A9F800830303F2EE239BB20132A24221F8023B09
:10AA080000F102000ED015F81230002B00F001837F
:10AA1800022BE9D001320B8821F8023BA24200F157
:10AA28000200F0D1109A137801331370FEF7F3BEC9
:10AA38009060002000007A44D34D62108C1F0020E3
:10AA480004200020644B0020D45B002070190020F3
:10AA5800E93700207119002065620020ABAAAAAA74
:10AA6800927100204E430020C0420020C0630020A5
:10AA780068620020EC640020D84CD4F88830A9EB38
:10AA88000303002BFEF6D5AED54AD64B527C05996A
:10AA980033F812308A7DDFEDD46A9FEDD46AC97D20
:10AAA8009BB207EE102A07EE903AB8EEC77AF8EE96
:10AAB800E77A27EE267A67EE867A0B9AC4F888201A
:10AAC800C7EE876A40F2FF32FCEEE67ACDED077AF0
:10AAD800BDF81C30934228BF134609B1D31A9BB264
:10AAE800C348C44D0178C44C35F81160226825F874
:10AAF8001130921B13440131C04D236001F00F0245
:10AB08001B0902702B80FEF794BE02F04DFEBC4B71
:10AB1800BC4A1B68C31A93427EF78BAEB74B002220
:10AB28001A80FEF786BE059A0499537DD27D013BB3
:10AB380031F913301AB1C3F53B6308331BB2A3F5DF
:10AB48007A7307EE903A9FEDB07AAC4AF8EEE77A5E
:10AB580040F2FF3167EE877AFCEEE77ACDED077AAF
:10AB6800BDF81C308B4228BF0B461380FEF761BE30
:10AB78001B7AC3F1640307EE903AFFF740BB4146E6
:10AB8800FFF714BB0221A148F6F7EEFB00283FF4BB
:10AB980022A82F8018F0020F7FF42FA848F0020394
:10ABA80043452B803FF429A8994B022214211A709F
:10ABB8000E20FF2259709A700BF066FCB5F80080E1
:10ABC800FFF71BB807F05EFFBCE4924AB2F9003009
:10ABD800002BB8BF5B42B3F5E17FBFF640A8B2F9DE
:10ABE8000230002BB8BF5B42B3F5E17FBFF637A850
:10ABF800894B93ED096AD3ED076A93ED057AD3ED96
:10AC0800037A76EE866A77EE877A76EEA66AB7EEEC
:10AC1800007A37EE666A77EEA77AB0EEC66AF0EE8B
:10AC2800E75AB4EEE56AF1EE10FAB4BFB0EE655A31
:10AC3800B0EE465AB5EE405AF1EE10FA40F0AD8348
:10AC48009FED767AB4EEE56AF1EE10FA44BF9FED17
:10AC5800746A36EE477AB7EE006AF4EEC66AF1EE29
:10AC680010FAC8BFDFED6F6AF5EEC07AC8BF36EEDE
:10AC7800C77AF1EE10FA48BFB1EE477AF6EE007ADD
:10AC880027EE677ADFED667A77EE276ABDEEE66A29
:10AC980016EE103A2033402B40F23086DFED626A20
:10ACA800624ADFED617AC2ED006AFDEEC76AC2ED65
:10ACB800017A16EE903A2033402BC2ED027A49D839
:10ACC800DFED587AB4EEE77AF1EE10FA40F37887C0
:10ACD8009FED576ADFED576A01E0B0EE677AB4EE90
:10ACE800E67AF1EE10FA77EE467AF6DC9FED527AC4
:10ACF800F4EEC77AF1EE10FA40F1EA879FED4C6A5C
:10AD0800DFED4E6A01E0F0EE477AF4EEE67AF1EE16
:10AD180010FA37EE867AF6D4DFED417AB4EEE77AA8
:10AD2800F1EE10FA40F33E86DFED3E7A37EEC77A51
:10AD380027EE076ADFED425ADFED426ADFED427A1D
:10AD4800E6EE256A67EE065AE6EE267AA5EEA77ABB
:10AD5800F0EE477A3D4BC2ED037A1B6813F40033DB
:10AD680040F018863A491A46C85C0A2803F10C03D1
:10AD780000F051850132182AF6D1FEF770BF2A88F3
:10AD880022F040039BB29A422B803EF461AF204BE5
:10AD9800022214211A700E20FF2259709A700BF0AB
:10ADA80073FBFEF755BF2B490E787FE594F8943076
:10ADB800002B3EF499AE079B1B7813F001037EF439
:10ADC80093AE012284F8943084F89520FEF78CBE67
:10ADD800024C012184F88C10FEF7B7BD0420002036
:10ADE80034640020546400200000C84200008044FD
:10ADF8005B5C0020605C00205C5C0020A4380020C4
:10AE0800D81D002060E316006F12833F9060002079
:10AE18007C460020C4410020641B0020A7DFA83422
:10AE2800DB0FC93FDB0F494000000000E0000020B5
:10AE3800DB0FC940E4CB1641DB0F49C0E4CB16C198
:10AE480092E741B99730083C15A82ABE4045002032
:10AE5800D04A0308E9370020012900F0038599F852
:10AE6800CC20012303FA0BF30BF1010B1343BBF1C5
:10AE7800040F89F8CC300AF10C0A7FF42AACFEF7EB
:10AE880078BE511D787923F0CFFF00283FF4E8A958
:10AE9800B9F1010F40F07A8607F10D01B87A23F075
:10AEA800C3FF002840F06E86B549F87B23F0BCFF4D
:10AEB80000283FF4E7A9B9F1030F40F05F86B149D4
:10AEC800387D23F0B1FF002840F05486AE49787EE3
:10AED80023F0AAFF00283FF4E7A9B9F1050F40F0D5
:10AEE8004586AA49B87F23F09FFF002840F03A869C
:10AEF800A74997F8230023F097FF00283FF4E7A914
:10AF0800B9F1070F40F02A86A24997F8280023F0E4
:10AF18008BFF002840F01E869F4997F82D0023F0EC
:10AF280083FF00283EF436AFB9F1090F3EF432AF83
:10AF3800FFF7E1B95D2A00F029855B2A00F06F82EE
:10AF48005E2A00F0CD85562A00F0DA85972A00F0AF
:10AF5800F285A72A00F0BA85904D2B889B0740F010
:10AF68007585A2F1B703072B00F28B82DFE813F097
:10AF78007D028902890289027102890265026502DD
:10AF8800079B002B3FD05CF8212093454FEA4103F3
:10AF9800FFF4E3AC824A824DD25C05EB030E002A33
:10AFA80000F09480022A47D19EF8012002EB820229
:10AFB80002EB820202F2EE2292B2032933DD12B2D0
:10AFC800BAF1000F3FF4CEAC0C9D20F81520B9F172
:10AFD800000F03D10F9D022D7FF6C4ACB0F802908C
:10AFE8000288B0F804E04A4496446E4A0FFA8EFE8E
:10AFF80082FB0E526C4DA2EBEE7225F803E012B202
:10B008004FF00109AEE41A464B000A9D4CF8215056
:10B01800A4E4D3B2022B04D9032B7FF4FBAC734610
:10B02800EAE43B46E8E4012505FA01FE0E9D25EA1F
:10B038000E0512B20E9591E4E25ABEE75B4A127809
:10B04800002A7FF40DAAB8F1000F3FF409AA012CD9
:10B0580040F036819BF82030FFF7A4B931465448B8
:10B06800F6F782F9002800F0C98084F893600CF0A4
:10B078000DFDFEF7C2BC43F0400293422A807FF4E4
:10B0880086AEFEF7E5BD4B4B4B4A109201221A7073
:10B098004A4B04931B214648F6F766F900287FF4CB
:10B0A80078AC474BDFF820B108931946DBF800303D
:10B0B800CA688B609B1AC82B00F2F584069B1E6831
:10B0C80006F48056AEE45B78FFF77AB8CAB2022A73
:10B0D80040F2BC83032AAFD1129A139D079E002D1C
:10B0E80008BF324669E728F0010292B242452A8039
:10B0F8003FF450AD0E2087F8009087F801A087F83C
:10B1080002B00BF0C1F9B5F8008043E500220FE06A
:10B11800437803EB830303EB830303F2EE239BB231
:10B128000132A24221F8023B00F102003FF47AAC5E
:10B1380015F812301BB1022BEAD00B88F0E7D3B216
:10B14800032BFAD83B46EBE7B2F5FA7FFEF6C4AC20
:10B1580094F89230002B7EF4BFAC079B1B78012239
:10B1680013EA020584F8922000F0B9830CF060F825
:10B17800144B0A4D0993FEF7B2BC0025FFF709B935
:10B18800454600204A4600204F46002054460020ED
:10B19800594600205E4600206346002014420020E5
:10B1A800C06300205655555574200020501F0020BC
:10B1B800906000204E4300206562002092710020BC
:10B1C800C04200201C420020EC640020B2F5FA7F47
:10B1D800FEF682AC94F89230002B7EF47DAC079A90
:10B1E80012780121D70784F8921000F103840CF03B
:10B1F8004DFCC24BC24D0993FEF771BC079BC14A77
:10B208001B781060DB077EF5FCABBF4B1B78002B6F
:10B218003EF462AC089BDB78002B7EF45DAC94F8BE
:10B2280093300133DBB2032B84F893307EF654ACB1
:10B23800B64B5B7813B9002D7EF44EAC0BF0F8FFDB
:10B24800FEF7DBBBB24AB3491068B4F99020C6696F
:10B2580081FB06018911F617701A00F5FF407F304F
:10B2680082423EF7BDAB891B0A4412B2A4F8902073
:10B27800FEF7B6BB089BDB78002B7FF4A4AADFEDB2
:10B28800A67AA44938EE678AC9F5FA63FDEEC87A4A
:10B298001BB2CDED047ABDF91020120381FB020127
:10B2A800D217C2EBA11203FB02F343F30F334B4453
:10B2B80007EE903AB8EEE78A87ED038AFFF783BA7C
:10B2C800099D002D3EF4C0AAFFF742B9934A059B99
:10B2D800D588049A1B8BB2F906105A1B914240F389
:10B2E80088802B449942B4BF00250125FEF7BDBADA
:10B2F800C8398A4242DA99F8CC109A7841FA0BF3A5
:10B30800D9073FF51AAA524201200C920BF0A2F974
:10B318007B1E0C9A162B00F24781DFE813F01A0205
:10B328002E020102530242026702EC01D701C20158
:10B33800AD0198014501530285016702EC01D7016F
:10B3480070015C01480135011F01DA0023F02AFD74
:10B35800032140F6B8328BF82010CBF81C20FFF7F9
:10B3680086B8AB460899DBF80020CB69099D1344E1
:10B378008B61002D3EF468AAFFF7EAB899F8CC3043
:10B38800012202FA0BF223EA020308F5FA7289F89D
:10B39800CC30CAF80820FFF7D0B9B4EEE56AF1EE70
:10B3A80010FA8CBFB0EE654AB0EE464AC4EE054AC4
:10B3B8009FED5B2A9FED5B5ADFED5B1ADFED5B2AA1
:10B3C8009FED5B3ADFED5B3A9FED5B4AA4EE825A54
:10B3D800E4EEE12AA4EE857AA4EEA23AB0EE475A4A
:10B3E800B0EE637AA4EE837AA4EE874A84EE057AF7
:10B3F80028E40125FEF739BA00215048F5F7B4FFD3
:10B4080000287FF426AA322384F89600A4F89830FE
:10B41800FFF71FBA002A0CBF0120022075E7484B2E
:10B42800012202204749484C0B60344B2270344DAE
:10B4380009930BF00FF9FEF752BB304A424B0992C1
:10B448001146424A0A6002225A7023F079FDFEF73B
:10B4580046BB2A4A3C4B099211463D4A0A600022E3
:10B468005A7023F06DFDFEF73ABB244A364B099219
:10B478001146384A0A6001225A7023F061FDFEF72E
:10B488002EBB792A00F017847A2A00F00B849E2AB2
:10B4980000F000849D2A00F0F683AE2A00F0EC83C9
:10B4A800AD2A00F0E283EF2A00F0DC83FD2A00F0E9
:10B4B800A183FB2A00F07483FE2A00F03184F72A66
:10B4C80000F059847B2A00F065830C4B0993FEF742
:10B4D80006BBD9F8D000204B90F836109B78114461
:10B4E8006429A8BF642121EAE17180F83610002B95
:10B4F80040F04C8417F022FFB1E400BF1C4200204A
:10B508001442002064330020E9370020EC6000205A
:10B51800543E0020D34D621000007A449857002012
:10B5280099FB243F69A2163E39094E3DE3B59E3E7C
:10B5380088FA163E45FE7F3FA7DFA83490600020BA
:10B54800CE33002018420020784200209C42002080
:10B558008442002090420020A0340020D9F8D00076
:10B56800BC4B90F837109B781144FE29A8BFFE21E8
:10B5780021EAE17180F83710002BBBD0162023F0A8
:10B58800C5FCD9F8D000B5E70B98B24B4178114407
:10B59800B1F5967FA8BF4FF4967121EAE171417029
:10B5A8009B78002B40F0AB83D9F8D000A2E7D9F8FC
:10B5B800D000A84B81781144C829A8BFC82121EA26
:10B5C800E17181709B78002B94D0142023F09EFCAD
:10B5D800D9F8D0008EE7D9F8D0009E4B41781144B5
:10B5E800C829A8BFC82121EAE17141709B78002BC6
:10B5F80080D0132023F08AFCD9F8D0007AE7D9F854
:10B60800D000944B01781144C829A8BFC82121EA69
:10B61800E17101709B78002B3FF46CAF122023F08E
:10B6280075FCD9F8D00065E78A4B0B989B7841796F
:10B6380011446429A8BF642121EAE1714171002BFA
:10B64800B2D00E2023F062FCD9F8D00052E7D9F826
:10B65800D000804B017A9B781144C829A8BFC82123
:10B6680021EAE1710172002B3FF444AF0B2023F073
:10B678004DFCD9F8D0003DE7D9F8D000754BC17919
:10B688009B781144C829A8BFC82121EAE171C1717A
:10B69800002B3FF42FAF0A2023F038FCD9F8D00054
:10B6A80028E7D9F8D0006B4B81799B781144C829D9
:10B6B800A8BFC82121EAE1718171002B3FF41AAFBC
:10B6C800092023F023FCD9F8D00013E7D9F8D000DB
:10B6D800604B417993F802E01144C829A8BFC821FA
:10B6E80021EAE1714171BEF1000F40F02883112F6A
:10B6F8007FF460AFFEE6D9F8D000564B017993F895
:10B7080002E01144C829A8BFC82121EAE1710171EA
:10B71800BEF1000F40F0FA82102F7FF45FAFE9E628
:10B728000B994C4B0F790C931744642FA8BF6427CF
:10B7380027EAE7770F7123F003FC0C9B9B78002B1B
:10B748003FF432AF0320394623F0E0FBD9F8D000AC
:10B75800D0E60B983F4B01781144FA29A8BFFA218B
:10B7680021EAE17101709B78002B3FF41DAF0120A5
:10B7780023F0CCFBD9F8D000BCE60B98354B817888
:10B7880011446429A8BF642121EAE17181709B7882
:10B79800002B3FF409AF022023F0B8FBD9F8D00002
:10B7A800A8E60B982B4BC1799B78114481F30801CB
:10B7B800C171002B3FF4F8AE052023F0A7FBD9F8A0
:10B7C800D00097E60B98234B817993F802E0114457
:10B7D8006429A8BF642121EAE1718171BEF1000FDB
:10B7E80040F0B7820D2F7FF420AFDDE6D9F8D00006
:10B7F800184BC17893F802E01144C829A8BFC821A2
:10B8080021EAE171C170BEF1000F40F0AA820F2F4A
:10B818007FF4F8AE6EE61048D0F800E05300BEF1B1
:10B82800000F08D09F1801EB87079EF801E07F788A
:10B838007745BEF414AA1A44084F094B01EB82015C
:10B84800002201603A801A60FEF709BA129AFFF7DF
:10B85800B4BB00BFA03400200C1F0020F81F00203C
:10B86800FC1F002004999B7831F91220B2F5617F02
:10B878004FF4966191FBF3F3C0F2A18040F63301D7
:10B888009142A8BF11460C2FA1F5617191FBF3F10C
:10B8980000F05E81182F7FF4E2AAC9B2C8290B46CE
:10B8A800A8BFC823D9F8D020D77DD8B2B8423FF472
:10B8B800D6AADF1BD14BD07548BF0737FF109B783E
:10B8C8000137FFB23BB9002F3FF4C9AA38460AF046
:10B8D800C1FEFFF7C4BA182023F018FBF3E70F20C6
:10B8E8000AF0D2FDB4F8903084F89250FA3BA4F8EC
:10B8F8009030C34BC34D0993FEF7F1B8B4EEE77A25
:10B90800F1EE10FA40F36381DFEDBF5A9FEDBF6A95
:10B9180001E0F0EE676AF4EEC66AF1EE10FA76EE30
:10B92800E57AF6DCDFEDBA6AF4EEE67AF1EE10FAC3
:10B9380040F14A81DFEDB45A9FEDB66A01E0F0EEBE
:10B94800667AF4EEC67AF1EE10FA77EEA56AF6D4C6
:10B95800DFEDB17AF4EEE76AF1EE10FA40F3C48055
:10B96800DFEDAE7A77EEE66A66EEA65A9FEDAC5A40
:10B978009FEDAC6ADFEDAC7AA5EE856A26EEA55A96
:10B98800E5EE867AE5EE276AFFF78AB9A74B00222B
:10B99800012047E5A64B1B78032B00F0D580002338
:10B9A800FFF7E0B9DFEDA37AB4EEE77AF1EE10FA2B
:10B9B80044BFDFED977A37EEC77AFFF7B9B90C2F96
:10B9C80040F0AD80002739469B4B0D915B78BB4218
:10B9D8003FF445AA894B0C93384607F0D3FC0C9BDF
:10B9E8000D999B781BB1C9B20C2023F08FFA01374F
:10B9F800FFB268E7914A834D1360814B0993FEF7C4
:10BA08006EB88F4A0592FEF73BBF38EE678A8D4BBA
:10BA18008D491870FDEEC87AC9F5FA63CDED047A40
:10BA2800BDF91020120381FB0201D217C2EBA1124B
:10BA38001BB203FB02F343F30F334B4407EE903A78
:10BA4800F8EEE77AC7ED037AFEF759BA0023BB2A66
:10BA580014936DD0B72A00F03781BE2A00F03C81DC
:10BA6800BD2A7FF40EAD4FF6FE71784A6448D68938
:10BA78000990908933440144D38191811CF00EFCD4
:10BA8800F4F7E0FD1CF0F2FB00F096FD01200AF04F
:10BA9800E1FDB4F890300022FA3BA4F8903084F825
:10BAA8009220FEF71CB86A4A069B1E68136823F0AA
:10BAB80004031360089A012306F4805682F82130A3
:10BAC800FEF7B0BF06F48056FEF7ACBF614A4D4D95
:10BAD800137843F004031370494B0993FDF7FFBF34
:10BAE8005D4B022203209DE4DFED527AF4EEE76A13
:10BAF800F1EE10FA44BFDFED467A77EEE66A33E7F7
:10BB08001CF0CCFBF4F79EFD1CF0B0FB00F054FDDC
:10BB180001200AF09FFD94F88E20FFF717BA182F1E
:10BB28007FF49DA900210B46BCE61A46FEF7E5BB4B
:10BB38001946022399E7494B324D4FF4C8721A80CF
:10BB48002F4B0993FDF7CBBF0AF082FCFEF787B8AD
:10BB5800CFB239E708221346FEF7CFBB07221346B8
:10BB6800FEF7CBBB06221346FEF7C7BB05221346DA
:10BB7800FEF7C3BB04221346FEF7BFBB03221346DE
:10BB8800FEF7BBBB02221346FEF7B7BB01221346E2
:10BB9800FEF7B3BB4FF4FA61022007F019FB94E4F7
:10BBA8000021022007F014FBB4F89030144A0992DF
:10BBB800963B0022A4F8903084F89220FDF78FBFBE
:10BBC800F0EE477AFFF792B8F0EE676AC0E6F0EE5B
:10BBD800667AA7E6002D3DF48CAE214C94F88D30A2
:10BBE800002B3DF4B7AE0AF033FC002384F88D3007
:10BBF800FDF7B0BE00210120D4E700BFA03400202B
:10BC08001C42002014420020DB0FC940E4CB16413F
:10BC1800DB0F49C0E4CB16C1DB0FC93FDB0F49403E
:10BC280092E741B99730083C15A82ABE8033002016
:10BC3800A8380020DB0FC9BF7842002064330020F9
:10BC4800705900208C1F0020D34D6210CC6000205A
:10BC580010420020845100201C34002086650020FA
:10BC680004200020002108469CE7FF2100200FF057
:10BC7800CDFE94F88E2016E4012100200FF0C6FEB8
:10BC880094F88E200CE40021FF200FF0BFFE94F8FA
:10BC98008E2002E4002101200FF0B8FE94F88E20D7
:10BCA800FFF7F8BB3B4A3C4B0993137A43F0010377
:10BCB8001372FDF714BF374A374B0993137A23F0F1
:10BCC80001031372FDF70BBF19464FF6FE73CCE65E
:10BCD800B0EE677AFFF720B80221C6E62E4B84F84B
:10BCE800941084F895002D4D0993FEF7A3BD0B2001
:10BCF8000AF0CAFB284B294D0993FDF7F0BE152021
:10BD080023F004F9D9F8D000FFF7F4BB10200D9305
:10BD18000C9223F0FBF8D9F8D0000D9B0C9AFBE4A9
:10BD2800002103203EE7002B3FF457AF1C491D4A72
:10BD380009684FF47A7000FB031313604DE7112074
:10BD48000D930C9223F0E2F8D9F8D0000D9B0C9AD1
:10BD5800CDE40D200D930C9223F0D8F80D9B0C9A8E
:10BD680040E50F200D930C9223F0D0F8D9F8D000BD
:10BD78000D9B0C9A4BE50021042013E70A4C0BF0AD
:10BD880057FA002384F88D30FDF7E4BD172023F01F
:10BD9800BDF809E4344300201C420020144200206E
:10BDA800EC640020603300200420002038B50B4CE0
:10BDB80023688BB15A68821A002A054604DA0CE017
:10BDC8005A68AA1A002A07DB9A68226018461A6875
:10BDD80090472368002BF3D138BD38BDF45C0020B0
:10BDE8000B4B002210B4027203F1B404042102E0E8
:10BDF800072A09DC9979890702D519798154013212
:10BE08009C4203F11403F3D15DF8044B704700BF63
:10BE1800BC54030810B40D4C04232146002200E052
:10BE28008B7913F0010301F1140106D101320A2ABA
:10BE3800F6D103705DF8044B704702EB820204EB05
:10BE480082025DF8044B137903707047BC540308F1
:10BE580010B4012302241521222204724170C270F9
:10BE6800037083705DF8044B704700BF2C220223D7
:10BE780002704370704700BF2DE9F0478C4B1B7868
:10BE8800DB07074644D58B4B8B4D1C788B4E012C1A
:10BE980059D01CD3022C07D189498A4A09881288AB
:10BEA800914201D901241C70EB7AE3B12B89D3B1FB
:10BEB800854B1B78BBB107F087FA002800F09B8000
:10BEC8002B7B83422CBF0121002131700CE07C497F
:10BED8007E4A098810886A7B801A8842E2DAEB7AFF
:10BEE8000024002BE2D131782A79632A06D8022C63
:10BEF800774E00F0BA803378002B5DD1754AAB7A63
:10BF08008C4238BF0C461470002B4CD1BDE8F0872A
:10BF18006B4B694D19885B88E878CB1A83EAE37222
:10BF28008142A2EBE3721DD32B788B421AD3614B6B
:10BF38001C78E01E012861D96749097802294FD089
:10BF4800012C5E4EA5D15F4A5D491288687B09883D
:10BF5800121A914239DD5D4A12888A42A4D200241D
:10BF68001C70A1E7B1EB400FE1DC524B1C78E11EDD
:10BF7800012940F29480022ADEDC57494F4E0878A6
:10BF8800DFF84481DFF844C1DFF838E100210324F9
:10BF9800022834701C7088F80010ACF80010AEF855
:10BFA800001081D11FE0012C71D0022C0BD1072089
:10BFB800BDE8F0470AF068BA7068381A474B9842EB
:10BFC80058DD72709AE7BDE8F08702241C706BE7B1
:10BFD800022AD2DD4049097802294FF0040464D1CD
:10BFE8003949364E09783E48022ACCBF0022012240
:10BFF800C28081804BE70221317075E7022A9BDC01
:10C0080095F800C091FBFCFC0CF1010CBCF1080F89
:10C01800DFF8B4A0304EA87895F801E096F80080D3
:10C028002A4CDFF8A090254EA8BF4FF0080C8AF8DC
:10C0380000C01FFA8CFA10FB0AF01EFB0AFE80B241
:10C04800DFF88CA02080A9F800E000244FF0640EEF
:10C05800B8F1020F34701C70CAF804408AF801E085
:10C068007FF439AF0FFA8CF1BDE73078A0B901231E
:10C0780077603370C2F164021A4B00FB02F083FB55
:10C088000023C017A0EBA3506430707036E7082077
:10C09800BDE8F0470AF0F8B97368F81A8EE7032C80
:10C0A80096D10D49097802299AD0044EFCE600BFC2
:10C0B800673E002094240020A4410020A4240020EE
:10C0C800D03F002098240020E63F0020962400203E
:10C0D8009C240020A8380020C03F00207F969800AC
:10C0E800C43F00206BCA5F6B2DE9F0470569C36840
:10C0F8001D4028D00F4606464FF000484FF0000973
:10C10800B5FA85F328FA03F2D2431B3B3261154096
:10C11800042B16D8DFE803F03129211903007B6AC4
:10C12800002B32D003F1FF3A1FFA8AFAC7F824909D
:10C138003C6A34B123682046514698476468002C0D
:10C14800F8D1002DDCD1BDE8F0873868716B036841
:10C1580089B29847002DD3D1F5E77868B16B0368A9
:10C1680089B29847002DCBD1EDE7B868F16B036829
:10C1780089B29847002DC3D1E5E7F868316C0368A8
:10C1880089B29847002DBBD1DDE7F36A1FFA83FA1D
:10C19800CEE700BF08B50121022005F0AFF9094B31
:10C1A8001B7803F00503052B08D00021012005F0BA
:10C1B800A5F90021084605F0A1F9FEE717F002FBF2
:10C1C800F3E700BF4C2C0020022828BF022010B43F
:10C1D800084C094B207000EB8002C0EBC2020749F3
:10C1E8005DF8044B013003EB4203C0B20B600AF068
:10C1F80031BA00BF78420020803300201842002066
:10C2080008B51CF04BF8F4F71DFABDE808401CF01F
:10C218002DB800BF2DE9F04F013085B0C3B20393AC
:10C228008E4D8F4F8F4C904E0A2302933220DFF8A9
:10C23800409218F06DFF4FF4FA7A4FF0100C4FF45B
:10C248007A70D9F80430C3F30803002B40F0C88093
:10C25800EFF31183002B40F0C3802968A26800BF68
:10C268002B689942F9D1D7F800E000FB0EF39B1A2E
:10C27800B3FBFEF300FB01314FF0010E0191D9F839
:10C288000430C3F30803002B40F08E80EFF31183D2
:10C29800002B40F089802B68A16800BF2A68934270
:10C2A800F9D1D7F800B000FB0BF2521AB2FBFBF23F
:10C2B80000FB0323019A9B1AB3F57A7FDFD3BAF107
:10C2C800010ABED1039B002B40F0C4804FF47A7A58
:10C2D800DFF89C9150464FF0100CD9F80430C3F3A6
:10C2E8000803002B40F09980EFF31183002B40F0F6
:10C2F80094802968A26800BF2B689942F9D1D7F8C1
:10C3080000E000FB0EF39B1AB3FBFEF300FB0131C8
:10C318004FF0010E0191D9F80430C3F308033BBB79
:10C32800EFF3118323BB2B68A16800BF2A689342EF
:10C33800F9D1D7F800B000FB0BF2521AB2FBFBF2AE
:10C3480000FB0323019A9B1AB3F57A7FE3D3BAF172
:10C35800010AC2D1029B013B02937FF467AF4349B4
:10C36800434B4448444A0860DA6005B0BDE8F08FA2
:10C37800EFF311888CF31288A1682368DB0344BFAC
:10C38800C6F800E0A1682B6832685FFA88F888F37D
:10C398001188D7F800801A4400FB08F35B1AB3FB36
:10C3A800F8F300FB0233CDE7EFF311888CF3128822
:10C3B800A1682368DB0344BFC6F800E0A1682B68C6
:10C3C80032685FFA88F888F31188D7F800801A4431
:10C3D80000FB08F35B1AB3FBF8F300FB023369E7D1
:10C3E800EFF311828CF31288D4F808E02368D9039C
:10C3F80003D501233360D4F808E02B683168D2B242
:10C4080082F311883A68194400FB02F3A3EB0E0388
:10C41800B3FBF2F300FB01312EE7EFF311828CF34B
:10C428001288D4F808E02368D90303D501233360C0
:10C43800D4F808E02B683168D2B282F311883A68E0
:10C44800194400FB02F3A3EB0E03B3FBF2F300FB6A
:10C4580001315DE7184621F095FD37E7EC640020CF
:10C46800F064002010E000E0E8640020FC9F002059
:10C4780000ED00E0EFBEADDE0400FA0538B5434B31
:10C488005A899989914224BF00225A81198ADA89E6
:10C49800914224BF0022DA81DA788AB3072A2FD0A2
:10C4A8003B493C4D91F85300012400210A282C7087
:10C4B8009C70D9713DD00C2865D0DFED377A8ABBE6
:10C4C800364C9FED370AA278002918BFF0EE407A63
:10C4D800062A04D8334901EB820191ED000A21793B
:10C4E80059B3013A032A4DD8F7EE007A87EE800A4D
:10C4F80025F0F0FA2388984228BF1846208038BDD6
:10C50800D97921B198780428B8BF042098702048B8
:10C5180090F853000A280CD00C28CED1DFED227AEF
:10C52800002ACDD0072ACBD00A282CD1DFED1F7ADC
:10C53800C6E70A20DFED1E7AC1E79B78154A07EEA9
:10C54800103A1178B8EEC77A27EE277A07EE901AD4
:10C55800F8EEE77A67EE877AB4EEE70AF1EE10FABA
:10C5680010DDC0EE077AFDEEE77A17EE903A102B51
:10C57800A8BF1023012BB8BF0123DBB28B4238BF01
:10C588000B46137038BDDFED0B7A99E7C8480020D9
:10C59800DC480020C06000206F120339644D002081
:10C5A8006F120338483203080AD7A3390F506E3A7E
:10C5B8005304E9386F12833A2DE9F047AA4FAB4E7E
:10C5C8001BF06CFEBE421ED2DFF81C83DFF81C9302
:10C5D8004446258862197DB14A450DD2052D0BD9EF
:10C5E80033886188C3F30B03994200F0E280144654
:10C5F80025886219002DEFD171683046143605F090
:10C608000AFABE42E4D39A4A1378A3F11701022921
:10C618000FD9984911F83300002840F0F680D80067
:10C628000144497829B1944911F83330002B00F0BE
:10C638001481924B5A78022A40F2E18000229049F4
:10C648005A701A788F48022A016000F2D48002EBEF
:10C6580082018D4BC2EBC10203EB4203998C5A8CC9
:10C668008A4C9142236001D300225A84884B9A78DD
:10C67800042A00F0E98032B91A88B2F5F07F84BF45
:10C688004FF4F0721A80834DFFF7F8FE2B68824A48
:10C698001A40002A00F0E480D80700F1D08059043D
:10C6A80000F1C8801A0700F1C0809B0400F1B68031
:10C6B80019F0A0FE10B9794809F088F8802005F033
:10C6C800E1F94FF4007005F0DDF94FF4802005F032
:10C6D800D9F94FF4001005F0D5F94FF0007005F0C6
:10C6E800D1F94FF0806005F0CDF94FF0006005F00A
:10C6F800C9F922F025FC00213022694826F0A5F965
:10C70800206816F0C3FC674B276803F1500102E06C
:10C71800043399426DD01A78002AF9D19C78D878D8
:10C728008442F5D26049614B0D79614961480A70CC
:10C73800614E624C0460C822642111FB052100226D
:10C7480059609A60DA601A615A619A61DA6183F80D
:10C75800202083F82120376015F05AFC584B9FEDB4
:10C76800595A1B88584A9FED596A5079584906EE1C
:10C77800903AF8EEE66A1388C5EE265A07EE103AA4
:10C7880053881279C1ED005A07EE903AB8EEC77A8D
:10C79800504BF8EEE77A18725A7227EE067A67EE6F
:10C7A800867ABDE8F04783ED017AC3ED007A1BF085
:10C7B8005DBD63799B077FF41AAF716894F804A094
:10C7C800304605F028F93388BAEB133F04D0143605
:10C7D800BE42FFF4FDAE16E773887068AA1FC3F364
:10C7E8000B039A4204F10601A8BF1A4625F032F855
:10C7F800EDE7012296E700221A70234B2EE7204925
:10C8080002EB420201EB82011BE7D8000C186468B6
:10C81800002C7FF405AF1724147001E72E4805F0AB
:10C8280031F9402005F02EF942E72C4805F02AF9A5
:10C838002B683AE72A4805F025F92B6832E729489A
:10C8480005F020F92B682AE79A8AB2F57A7FBFF4B7
:10C858001AAF4FF47A729A8215E718231370E8E634
:10C8680043F400532B6017E7008D0308A0880308E2
:10C878007851002084550308704E03087842002040
:10C88800844200201C4200208033002018420020EF
:10C89800644D0020B4340020096000029C59002037
:10C8A800A0200020B062002064650020C042002063
:10C8B8009C1B0020E4200020D4200020D26000200F
:10C8C800901F0020C0C9FB48C41D002017B7D138ED
:10C8D800941F002048650020094000020160000202
:10C8E800092000020860000202F0030800000408A2
:10C8F80008B51BF0D3FCF3F7A5FE1BF0B7FCFFF758
:10C908005BFE0120BDE8084009F0A4BE2DE9F04710
:10C91800B54C82B0636820469847002800F0BF8075
:10C92800B24B1B780122042B84F83C2000F0BA801B
:10C93800B4F91610B4F91820B4F91A3021636263F7
:10C94800A363AB4B1B88002B69D0AA4DD4ED0C7A9E
:10C95800D5ED004A95ED050A95ED015A95ED067A53
:10C96800D5ED035A95ED026AF8EEE76AD5ED047A3B
:10C97800A4EEA60AA5EE267A67EEC07AA5EEC07ADE
:10C98800E6EE267A85ED057AC5ED067A25F0A2F859
:10C99800D4ED0D6AD5ED094A95ED0E0A95ED0A5AC2
:10C9A80095ED0F7AD5ED0D7AD5ED0C5A95ED0B6A0C
:10C9B8002063F8EEE66AA4EEA60AA5EE267A67EEEC
:10C9C800C07AA5EEC07AE6EE267A85ED0E7AC5ED38
:10C9D8000F7A25F07FF8D4ED0E6AD5ED124A95ED61
:10C9E800170A95ED135A95ED187AD5ED167AD5ED07
:10C9F800155A95ED146A6063F8EEE66AA6EEA40A85
:10CA0800A6EE857A67EEC07AA0EE657AE6EE867ABB
:10CA180085ED177AC5ED187A25F05CF8A063764F96
:10CA2800A17F764815F076FA3B88002B7CD1744EAE
:10CA38003568744B1B685B0742D4B5F90070216BED
:10CA4800636BA06B704A714E92ED026AD2ED006A78
:10CA5800D2ED015AC91B2163B5F90270DB1B636370
:10CA6800B5F904703568C01B07EE900AB8EEE75AAE
:10CA780007EE901AB8EEE77A07EE903AF8EEE77A02
:10CA880036EE056A36EE877A77EEA57A0135A06329
:10CA980082ED026A82ED007AC2ED017A356002B059
:10CAA800BDE8F0875A4BB4F91600B4F91810B4F978
:10CAB8001A2018802063598061639A80A26340E736
:10CAC800544F3B88322B7ED0002B5BD152480378E1
:10CAD800002BB2D0DFF848E1F169326A8EFB0173AE
:10CAE8000027C9170770C1EB23118EFB0203D21769
:10CAF800C2EB2312736A29806A80A08A47498EFB99
:10CB080003E2DB17C3EB22131B1AAB80CF601BF0C9
:10CB1800C5FBF3F797FD1BF0A9FBFFF74DFD0120BF
:10CB280009F098FD356888E7354E226B3568B3F50E
:10CB3800C87F4FF0000323632B80398818BF7068C3
:10CB4800B7F8008008BF0020B1F5C87F18BFB368E8
:10CB5800616B02440B440020B8F5C87F60637260C3
:10CB6800B36068803AD0D4F838E0F168A0637144C3
:10CB7800B8F1010FA880F16054D008F1FF38A7F888
:10CB8800008056E7F169226B002323632B80B7F8F6
:10CB980000E00A44BEF1320F616B63636B80F2619F
:10CBA800A26B6BD0706A0190306AA363014401984C
:10CBB80031620244BEF1010FAB80726263D00EF1A4
:10CBC800FF333B8082E7154B2988D8686A88AB8891
:10CBD8003182B0617282B3820021D4E7A36BF36023
:10CBE800A063A880C9E700BFCC410020C03F002057
:10CBF800C0540020C454002086650020FC41002059
:10CC0800E4200020644B00203C65002038650020AB
:10CC1800C43F00209C20002099200020CC600020E8
:10CC28001F85EB51DFF80CC1DFF8F8E0C8328CFB48
:10CC380002A9C833D217C2EBE9128CFB03A9DB1790
:10CC4800C3EBE913C8316B802A808CFB013CA28AB4
:10CC5800CB17C3EBEC139B1AAB80CEF80C001BF080
:10CC68001DFBF3F7EFFC1BF001FBFFF7A5FC4046AB
:10CC780009F0F0FCB7F8008035687EE7A3633162FD
:10CC88007262AB809BE7234A2348126823490370EA
:10CC980012F4003281F800E032D113462049C85C12
:10CCA8000B2803F10C030ED00132182AF7D1338A6E
:10CCB8002B80728A1B4B6A80B18AB269A980B7F847
:10CCC80000E0DA607BE71848D0F800C05300BCF1F8
:10CCD800000F09D003EB020E01EB8E0E9CF801C089
:10CCE8009EF801E0E645E2D21344DFF84CE00F4A33
:10CCF80001EB830100230160AEF800301360D6E732
:10CD08000B4A1278032A01D01A46C7E709F0A0FB9C
:10CD18003568CCE7404500209E2000209820002060
:10CD2800D04A0308CC6000200C1F0020FC1F002004
:10CD3800A83800201F85EB51F81F002038B50C4C8F
:10CD48000C4DAC4206D261682046143404F063FEF0
:10CD5800AC42F8D3084A094B094C1460002209492F
:10CD68001A705A7008480860BDE8384010F064BE70
:10CD7800A0880308008D030818420020784200208C
:10CD8800803300201C4200208442002008B5FFF7B1
:10CD9800D5FF1BF083FAF3F755FCBDE808401BF0FC
:10CDA80065BA00BFF0B50C292BD8DFE801F06F2A6F
:10CDB8002A2A4C2A2A2A2B2A2A2A0700046AB2F885
:10CDC8000CE097881668674D24F480540462036A5F
:10CDD8004468C16923F4005343EA0E3321F4E64161
:10CDE800A84243EA073341EA062100F0B58005F579
:10CDF8000065A84200F0B08092684460C161026496
:10CE08000362F0BD046A96899588D2F800E0554F10
:10CE180024F480740462036A4468C16923F40073CB
:10CE280043EA062321F07301B84243EA052341EAA5
:10CE38000E017ED04C4DA8427BD092684460C161FF
:10CE4800C2630362F0BD046A96899588D2F800E04F
:10CE5800444F24F010040462036A4468816923F093
:10CE6800200321F0807143EA061321F4E641B84219
:10CE780043EA051341EA0E2148D03B4DA84245D06C
:10CE880092684460816182630362F0BD046A938999
:10CE9800B2F804E01768334E24F001040462056A0E
:10CEA8004468816943EA0E0321F4803125F00205C4
:10CEB8009BB221F07301B04243EA050341EA07013E
:10CEC80014D0294DA84211D005F54065A8420DD0CF
:10CED80005F58065A84209D005F58065A84205D00A
:10CEE80092684460816142630362F0BDD689158A05
:10CEF800578A23F0080333433D43D68824F440740B
:10CF080023F00403ADB233432C43E9E7D589178AEC
:10CF1800D68823F0800343EA051324F44064558A35
:10CF280023F0400344EA870443EA061344EA8504ED
:10CF3800A6E7D589178AD68823F4006343EA052330
:10CF480024F44054558A23F4806344EA071443EADE
:10CF5800062344EA051470E7158A24F4804444EA59
:10CF6800851449E7002C0140003401402DE9F04FB9
:10CF7800C822002183B07848784CDFF80492784DB5
:10CF8800784E794FDFF8FC8125F05FFD77487849C6
:10CF9800DFF8F4E1DFF8F4C100221359834200F00E
:10CFA800C180B3F1804F00F0C980AB4200F0C88067
:10CFB800B34200F0C780BB4200F0C680734500F062
:10CFC800C580634500F0C480434500F0C380DFF8A6
:10CFD800C0A153457ED00AF5806A534508BF09238E
:10CFE80079D01432C82AD8D15C4C624D624E604F59
:10CFF80004F1C80802E01434A04568D0A379002BD6
:10D00800F9D023794FEA131909F1FF39B9F1050F5E
:10D0180003F00F03EFD835F8190040FA03F2D207EE
:10D02800E9D54FF0010A0AFA03F3013B184024F04E
:10D038009DF916F809305149184411EBC002DAD0AD
:10D0480051F83000DFF84CE1217A00F138439B0AAF
:10D058001EF8033003F01F0E5B09022B0AFA0EFAC2
:10D0680062D0032B65D0012B03D17B694AEA030305
:10D078007B6193880093B3FA83F3C3F11F039BB2D8
:10D08800DA0800EB820203F00703D2F820E09B00E5
:10D098004FF00F0C0CFA03FC2EEA0C0EC2F820E03D
:10D0A800D2F820E001FA03F343EA0E03136269465B
:10D0B8000023022214348DF804208DF805308DF8F1
:10D0C80006308DF807300EF0FBF9A04596D103B075
:10D0D800BDE8F08F082309EBC3034FF0010B93F869
:10D0E80020A00AF01F034FEA5A1ABAF1020F0BFAEE
:10D0F80003F30BD0BAF1030F0ED0DA457FF471AF0A
:10D10800D1F814A043EA0A034B616AE7D1F818A0E2
:10D1180043EA0A038B6164E7D1F81CA043EA0A03D7
:10D12800CB615EE70023D6E7BB694AEA0303BB612C
:10D138009FE7FB694AEA0303FB619AE70123CAE711
:10D148000223C8E70323C6E70423C4E70523C2E78D
:10D158000623C0E70723BEE7A8580020BC540308ED
:10D16800000400400008004000100040002C01406E
:10D1780000100240904C03089C4C03089047002084
:10D1880048320308004001400014004000340140C8
:10D1980000440140B454030801490248FEF7A4BF03
:10D1A800485900200048014001490248FEF79CBF49
:10D1B800205900200040014001490248FEF794BF71
:10D1C800F85800200004004002494FF08040FEF764
:10D1D8008BBF00BFD058002001490248FEF784BF2A
:10D1E800A8580020002C014001490248FEF77CBFE6
:10D1F800A8580020002C01402DE9F04104684A4D50
:10D20800A30AAB4272D009D8B3F5801F6AD04A3D51
:10D21800AB425AD14FF0700E022608E0434DAB42A4
:10D2280068D00235AB4252D14FF0C00E0426477980
:10D238004FEA970C002961D0B00063468519022790
:10D24800D4F80C809F400CEB4503BFB2384D03F176
:10D25800040C47EA080745F8231045F82C20E76036
:10D26800EFF31181502282F31288821905EBC20272
:10D27800136973B313620433821905EBC202576949
:10D2880017B11F6053690433821905EBC20297690D
:10D2980017B11F6093690433821905EBC202D7697D
:10D2A80017B11F60D36904330027CAB21F6082F325
:10D2B8001188304405EBC000036A6BB9E3684FF688
:10D2C800FE721340E360BDE8F081BDE8F081BDE87F
:10D2D800F08105EB0E03CFE7E36843F00103E36059
:10D2E800BDE8F0814FF0480E0126A0E74FF0200E70
:10D2F80000269CE74FF0980E032698E7BF08022304
:10D3080006FA03F0BB40DB43E768094D9BB23B409C
:10D3180087190CEB470CE3600CF1040345F82C105B
:10D3280045F823209CE700BF4B0010005000100078
:10D33800A858002030B503685C4D18885C4CB4FBD5
:10D34800F2F20139013AAB4294B283B089B282B2A7
:10D3580066D05848834263D0B3F1804F60D0A0F5BF
:10D36800983083425CD000F58060834258D05248A0
:10D3780083425BD000F5806083427DD022F4407206
:10D3880000F58C3092B283421A80D9621C850ED087
:10D39800484A93420BD002F54062934207D002F507
:10D3A8008062934203D002F58062934201D1002249
:10D3B8001A8601225A611A883C4992B242F0010247
:10D3C8008B421A8062D0B3F1804F61D03B4A9342BE
:10D3D80060D002F5806293425ED002F5006293420B
:10D3E8005CD002F5806293425AD002F590329342A3
:10D3F80058D002F54062934256D002F580629342BB
:10D408001ED002F58062934208BF092219D002A8F3
:10D418004FF0012340F8043D0EF01CF803B030BD76
:10D42800254822F07002834292B2A3D101201A80CB
:10D43800D9621C8558611A8892B202431A80C5E7DE
:10D4480008221F4B03EBC20301A893F821408DF873
:10D458000440012300228DF805308DF807308DF83F
:10D4680006200DF0F7FF1B2CD8D1164B019301A80D
:10D478000DF0F0FF03B030BD01201A80D9621C8581
:10D4880058611A8892B202431A809CE70022D8E7B2
:10D498000122D6E70222D4E70322D2E70422D0E70A
:10D4A8000522CEE70622CCE70722CAE7002C014076
:10D4B80000A24A040034014000100040000400406B
:10D4C8004832030819010001204B98422DD0B0F1D1
:10D4D800804F2CD0A3F5943398422AD003F580636B
:10D4E800984228D003F50063984226D003F580635C
:10D4F800984224D003F59033984222D003F5406334
:10D50800984220D003F58063984207D003F58063E2
:10D51800984208BF092202D00020704708220C4B0D
:10D5280003EBC20393F8200070470022F7E70122BB
:10D53800F5E70222F3E70322F1E70422EFE70522E9
:10D54800EDE70622EBE70722E9E700BF002C0140E0
:10D55800483203082DE9F04F013085B0C3B2039378
:10D568000B4602918B4C8C4E002B00F09A80322097
:10D578008A4D8B4FDFF82C9217F0CAFD4FF4FA7AD8
:10D588004FF0100C4FF47A70D9F80430C3F3080345
:10D59800002B40F0DE80EFF31183002B40F0D980A0
:10D5A8002968A26800BF2B689942F9D1D7F800E032
:10D5B80000FB0EF39B1AB3FBFEF300FB01314FF0A7
:10D5C800010E0191D9F80430C3F30803002B40F091
:10D5D8008780EFF31183002B40F082802B68A168CD
:10D5E80000BF2A689342F9D1D7F800B000FB0BF2CC
:10D5F800521AB2FBFBF200FB0323019A9B1AB3F504
:10D608007A7FDFD3BAF1010ABED1039B002B40F029
:10D61800BD804FF47A7ADFF88C9150464FF0100CA9
:10D62800D9F80430C3F30803002B75D1EFF3118345
:10D63800002B71D12968A26800BF2B689942F9D1E3
:10D64800D7F800E000FB0EF39B1AB3FBFEF300FBD8
:10D6580001314FF0010E0191D9F80430C3F30803EA
:10D6680013BBEFF31183FBB92B68A16800BF2A68CD
:10D678009342F9D1D7F800B000FB0BF2521AB2FB73
:10D68800FBF200FB0323019A9B1AB3F57A7FE3D3DD
:10D69800BAF1010AC4D1029B013B0293002B7FF42B
:10D6A80066AF05B0BDE8F08FEFF311888CF31288F0
:10D6B800A1682368DB0344BFC6F800E0A1682B68B3
:10D6C80032685FFA88F888F31188D7F800801A441E
:10D6D80000FB08F35B1AB3FBF8F300FB0233D2E755
:10D6E800EFF311888CF31288A1682368DB0344BF29
:10D6F800C6F800E0A1682B6832685FFA88F888F3FA
:10D708001188D7F800801A4400FB08F35B1AB3FBB2
:10D71800F8F300FB023370E7EFF311828CF3128801
:10D72800D4F808E02368D90303D501233360D4F87B
:10D7380008E02B683168D2B282F311883A6819443C
:10D7480000FB02F3A3EB0E03B3FBF2F300FB013182
:10D758007FE7EFF311828CF31288D4F808E023688E
:10D76800D90303D501233360D4F808E02B68316866
:10D77800D2B282F311883A68194400FB02F3A3EB92
:10D788000E03B3FBF2F300FB013118E7184620F053
:10D79800F9FB3EE710E000E0E8640020EC640020BC
:10D7A800F064002000ED00E0204B5B68C3F3080341
:10D7B80030B4BBB9EFF31183A3B91D4B1D4C1868E6
:10D7C800A16800BF1A689042F9D11B4B1C684FF43E
:10D7D8007A7202FB04F3591AB1FBF4F130BC02FB74
:10D7E80000107047EFF31182102383F31288114958
:10D7F8008C680B6813F4803F104B02D0012018602E
:10D808008C680B49D2B20D68186882F311880A4BEC
:10D8180019684FF47A72284402FB01F31B1B30BCD1
:10D82800B3FBF1F302FB0030704700BF00ED00E0EE
:10D83800EC64002010E000E0F0640020E8640020C0
:10D848002DE9F84F8046FFF7AFFF254E2549DFF851
:10D85800A0E0254A254D844610274FF47A7401200C
:10D86800DEF80430C3F30803D3B9EFF31183BBB96F
:10D878000B68D2F808A000BFD1F800904B45F7D14B
:10D88800D6F800B004FB0BF9A9EB0A09B9FBFBF9C0
:10D8980004FB0393A3EB0C034345E1D3BDE8F88FE6
:10D8A800EFF3118A87F31288D2F808B01368DB0304
:10D8B80044BF2860D2F808B00B68D5F800905FFA2A
:10D8C8008AFA8AF31188D6F800A0994404FB0AF36F
:10D8D800A3EB0B03B3FBFAF304FB0933DAE700BF4E
:10D8E800F0640020EC64002010E000E0E864002010
:10D8F80000ED00E02DE9F04FDFF830C1474A484914
:10D90800484E494D8046102718F1FF38C0F08480F2
:10D91800DCF80430C3F30803002B5CD1EFF3118368
:10D92800002B58D10B68946800BF08688342F9D16E
:10D93800D6F800904FF47A7000FB09FEAEEB040EA7
:10D94800BEFBF9FE00FB03EEDCF80430C3F308036A
:10D958004FF47A740120FBB9EFF31183E3B90B6834
:10D96800D2F808A000BFD1F800904B45F7D1D6F8FF
:10D9780000B004FB0BF9A9EB0A09B9FBFBF904FB9E
:10D988000393A3EB0E03B3F57A7FBDD2DCF8043022
:10D99800C3F30803002BDFD0EFF3118A87F3128853
:10D9A800D2F808B01368DB0344BF2860D2F808B087
:10D9B8000B68D5F800905FFA8AFA8AF31188D6F8CE
:10D9C80000A0994404FB0AF3A3EB0B03B3FBFAF39F
:10D9D80004FB0933D5E7EFF3118487F31288D2F8F3
:10D9E80008901368D80303D501232B60D2F8089058
:10D9F8000B682868E4B284F31188D6F800A04FF4C5
:10DA08007A7400EB030E04FB0AF3A3EB0903B3FBE0
:10DA1800FAF304FB0E3E97E7BDE8F08F10E000E054
:10DA2800EC640020F0640020E864002000ED00E0D1
:10DA380030B4EFF31183102282F312880649074CA1
:10DA48000A680748013200250A602560DBB20268CF
:10DA580083F3118830BC7047EC640020E864002030
:10DA680010E000E02DE9F04FC04B1E788BB0002E7F
:10DA780040F0BC80BE4BBF4C1D78DFF818A3DFF820
:10DA88001893DFF8188305F00105A4F10A0B54F880
:10DA98000A3CBBB1CC2707FB06B7184602F000FDCD
:10DAA80080B154F80A0C02F0F3FC14F8023C8BB96C
:10DAB800242831D0F5B154F80A3C184602F0F0FC9D
:10DAC8000028EED10136032E04F1CC04DFD10BB0CF
:10DAD800BDE8F08F012B23D0022B2BD0032B37D09E
:10DAE800042B67D0052B40D0062B4FD054F80A2CB6
:10DAF8001346D2E754F80A3C23281A4600F08981D5
:10DB08009D4991F832108142C7D19C4BCAF80090C8
:10DB1800C3F80C801346C0E7012304F8023CCAE7A7
:10DB28004D2854F80A2C0CBF0223002304F8023CA9
:10DB38001346B2E700233C2804F8023C45D03E28AF
:10DB4800D4D10122032304F8012C04F8023CB2E7E3
:10DB5800C02814D80022042304F8050C04F8040C87
:10DB680004F8062C04F8023CA5E714F8063C14F85F
:10DB7800052C9A422FD814F8043C834203D0002382
:10DB880004F8023C97E7062304F8023C14F801EC79
:10DB9800BEF1000F00F08281BEF1010F00F0C681D6
:10DBA80001360023032E04F8023C04F1CC047FF470
:10DBB8006EAF8CE714F8043C04F8030C58400523B6
:10DBC80004F8040C04F8023C75E7032204F8013C4D
:10DBD80004F8022C6FE714F8042CF91842400133BA
:10DBE80004F8042C04F8063C887264E7644B18684F
:10DBF80000283FF46CAF03F045FEDFF8A4A1614DA7
:10DC0800DFF8A091DAF8000002F04AFC00283FF49F
:10DC18005EAFDAF8000002F03BFC09281BD03F2871
:10DC280019D02B68002B67D1042800F0A9810C2893
:10DC380000F0E8807F28E5D0A0F12002D2B25E2A69
:10DC4800E0D80BB92028DDD05A1C09F803002A6057
:10DC58001AF00AFFD6E72C68002C5BD14A4FA3467E
:10DC680007F59878BBF1000F08BFBB460837474552
:10DC7800F8D1BBF1000F00F07881083FDBF8000015
:10DC88003A68065D135D9E42204402EB040140F0B1
:10DC98006A81661E4E4422460BB9FD2A5DD906F8F4
:10DCA800013F01322A6010F8013F11F801EF9E454B
:10DCB800F2D00AB15F4512D034481AF0DDFE5F4554
:10DCC80008D35BF8080B1AF0D7FE09201AF0CCFE2F
:10DCD800BB45F6D92E481AF0CFFE2A680024944294
:10DCE80090D2661E4E4416F8010F1AF0BDFE2B683E
:10DCF80001349C42F7D385E70C2800F083800A287A
:10DD080052D00D2850D07F2800F0FD80FF2B3FF621
:10DD180079AF91E71C4E002706F59878BB4602E0DC
:10DD2800083646450DD0224631684846F2F788FF46
:10DD38000028F5D1B346002FF2D1374608364645BC
:10DD4800F1D13B465F469B46002B97D1002F3FF40D
:10DD580059AF0E481AF090FEB3E7511C202009F87D
:10DD68000200296009F801300A46A3E75D42002055
:10DD7800673E0020A66E00209C59002000ED00E0C0
:10DD8800342D00203C2E002040470308E8590308A2
:10DD9800F0590308FC9F0020EFBEADDE0400FA0531
:10DDA800382D00203C2D00201AF0E7FE23217C4866
:10DDB80024F062FE002800F0E180A0EB0900286052
:10DDC80088B1431E19F80310202940F0E78009EBB9
:10DDD800030204E012F8011D202948D10346581E09
:10DDE800002BF7D12B604FF480720021484624F0B5
:10DDF8002CFE6C4B1B78002B3FF469AE6A481AF076
:10DE08003BFEFFE669481AF037FE67481AF034FE11
:10DE1800F8E667496748C978674ADFF8CCE1936252
:10DE2800003118BF012101706449D1624021136398
:10DE380082F8341082F83550614962480B602C3200
:10DE4800CEF80020574A012313701BF077FB564881
:10DE58001AF012FE4FF4006004F044FE5A4B93F897
:10DE68003230232B00F0928014F8023C3CE62B6001
:10DE7800564C002204F5987809F8032002E008348B
:10DE8800444577D02168484607F032FC0028F6D090
:10DE980044456FD2636898470023A3E74C4BADF81D
:10DEA80022E00FCB0DF1280C02AF87E80F004CF8E9
:10DEB80024ED14F8051C14F8033C069404EB010E39
:10DEC800624639464FF0010C06A8CDF81CE0ADF8C3
:10DED80020308DF824C0F5F70FF8E8B9019F00232A
:10DEE80004F8023C002F3FF4EDAD54F80A0C07F09B
:10DEF80031FD013654F80A0CB847032E04F1CC045E
:10DF08007FF4C5ADE3E5013B002232482B6009F8F8
:10DF180003201AF0B1FD75E6029A2F4B0392394699
:10DF2800A4F10A00029307F08EFCD7E714F8053C29
:10DF380014F8032C0694234407936E2A4FF0000329
:10DF480008930993ADF820207FF42AAE06A8F2F7CB
:10DF5800F9FE06A8F2F7EAFE06A8F2F7E7FE06A819
:10DF6800F2F7E4FE1CE62246A3E61C48083F1AF036
:10DF780083FDA6E61A481AF07FFD8DE728681FE79B
:10DF8800074806F04AFD0BB0BDE8F08F154A14F8B3
:10DF9800023CC2F80C80CAF80090A5E5034667E782
:10DFA8003C2D00205D420020F0590308F859030871
:10DFB800784200201C250020E42000206D00010884
:10DFC800382D0020245A03089C5900204047030894
:10DFD800B4320308205A0308EC720020E8590308F9
:10DFE800045A030800ED00E0342D00202DE9F04F1D
:10DFF8002DED028B95B005460CF036FAB14B1C7826
:10E0080024B115B0BDEC028BBDE8F08FDFF820B36A
:10E01800DBF800305805F4D5AB4F3A68002A00F019
:10E028001B81AA4ED6F8283103F5F43348339D42B4
:10E03800C0F01281A64996F82C310968C6F8285113
:10E048000133DBB2890786F82C3101F118815807B2
:10E0580001F05680282B9F4B039301F0A6815E2088
:10E0680090479D4B1B78002B6BD0984E9B4AD6F857
:10E078003031EB1A934200F2C787DFF8B8A29AF85A
:10E088000090B9F1000F33D1DFF86082D8F80000B2
:10E0980002F006FAC0B201280ED90228904F41F0CA
:10E0A8008C823B78002B41F0BE83D6F83831EB1ACE
:10E0B800B3F57A6F81F066848A480268002A40D0F6
:10E0C8009AF80030BBB9884BD8F800001B689B78D9
:10E0D8001E3B012B4FF0020141F2B28304300EF0D7
:10E0E8001DFF012200238AF8002086F8443126E02B
:10E0F8007C4802682AB3D6F8403140F6B731EB1AAB
:10E108008B421ED996F83C31002B01F04D82013B21
:10E11800DBB286F83C31002B01F01B8112F8011BA1
:10E1280096F84471026096F845317048CA1901336F
:10E13800006886F8442186F8453102F0B5F9C6F83A
:10E1480040516B4A039B12781B68012A03F10103B3
:10E158000C9300F0A686674B1B786BB1664F3B6843
:10E1680053B1039B594ED3F80090D6F85831A9EB18
:10E178000303632B00F23886DFF8BC8198F800901F
:10E18800B9F1020F01F0C180554F97F87430032B95
:10E1980000F08087594B1B7873B1594C23685BB1E9
:10E1A8004A4EFFF701FBD6F86431049044F61F622B
:10E1B800C31A934200F2D280524B1B78002B4ED1E7
:10E1C800514B1B7843B1414ED6F8B43203F50043A6
:10E1D800E8339D4280F0DF864C4B1B78002B3FF4E0
:10E1E80010AF3A4E4A4C4B4D06F2BD27206802F05C
:10E1F80057F900283FF405AF206802F049F92B7859
:10E2080080465A1E33B120682A7002F049F9002866
:10E21800F2D1F6E603223946781E24F0FCFB96F884
:10E22800BC3296F8BD2286F8BF8283F47F4383F020
:10E23800FF039B1A1FFA88F89BB2B8EB132FD5D1AE
:10E2480096F8BE22DBB29A42D0D1781E0EF09AF927
:10E258002B7818442870C9E71E4B039301E72E4C0E
:10E268002278002A40F014862C4F3C78002C65D187
:10E278002B4E3078002841F06182144E294CD6F894
:10E28800AC122278284B93FBF2F30B449D4297D3B0
:10E2980096F8B032254AC6F8AC52D75CFB0701F1B4
:10E2A8008F83B90701F1D8837A0701F1248396F89F
:10E2B800B0322178013393FBF1F201FB123386F877
:10E2C800B0327DE75D420020344200205C2100200E
:10E2D800C0410020EC6400203E3900203F0D0300BF
:10E2E8000C0000202C42002028420020244200205C
:10E2F8003F3900204C390020346600205439002072
:10E308005839002098390020A93900205E390020AA
:10E31800643900206839002030390020A1390020F4
:10E32800A0390020A8390020A0860100A4390020C7
:10E33800644B0020304200202E620020054E306ED3
:10E34800002841F06A808146034B87F80090C3F8A3
:10E35800AC5235E7B03900205C21002096F86A31CC
:10E36800002B41F00780DC4B1A6802F00803002BF1
:10E3780048F603414AF60B404BF60F4349F6074768
:10E3880004BF03460F4612F0040F4FF0190118BFDF
:10E398001F46920686F86A1103D547F4804747F06E
:10E3A800200705F003F8C7F30909002841F0758430
:10E3B800CA4B9B79002B41F06984984664204FF042
:10E3C800FF3A4FF0000C0C970D97ADF83CC0CDF814
:10E3D80042C0CDF846C0CDF84AC0CDF83890ADF867
:10E3E8003E80ADF840A08DF84E000CAF0FCFDFF89F
:10E3F80004E386F805C0AEE80F0097E80F00AEE822
:10E4080007002EF8023B71464FF0010C1B0CFE274B
:10E418001F20C82201F81E39B770B27186F807C0EC
:10E42800F07096F87A01307180F0F10383EA0313F3
:10E43800DAB2130983F0E70343EA022383EAC2034B
:10E448001BB283EA0312D2B2C3F3072383EA12137F
:10E4580043EA022383EAC2031BB283F0C80282EABA
:10E468000212D2B2C3F3072383EA121343EA022348
:10E4780083EAC2031BB283EA0C0787EA0717FFB2D5
:10E48800C3F3072282EA171242EA072200EB0C03C1
:10E4980082EAC7070EEB0C0086F87A31378011F84C
:10E4A800013B7B4083EA0313DBB21A0982EA172295
:10E4B80042EA032282EAC3031BB29FB28142378039
:10E4C800EDD183F07C0383EA0313DBB24FEA131E1A
:10E4D8008EEA172E8EEA032E8EEAC30E0FFA8EFEF0
:10E4E8001FFA8EF9DFF810C2A6F800905FFA8EFEC8
:10E4F8004FEA192986F8289086F827E00CF5D17894
:10E5080006F1220ADCF80000DCF80410DCF8082028
:10E51800DCF80C3047460FC70CF1100CD445B84650
:10E52800F0D1DCF8000038606D4F9CF8043088F8B2
:10E53800043007F1270886F8C9E186F8CA9117F868
:10E54800011F206801F0B0FFB845F8D196F86B318B
:10E55800002B40F014876349039A097812680A204F
:10E5680086F86B01002901F0D6805F4F01293888B1
:10E57800089041F2F8830229B7F802E001F0A78376
:10E58800B8880790032901F0E483F88806900429E5
:10E5980001F09D840529388901F094840629B7F88B
:10E5A8000A9001F08B840729B7F80C8001F0838466
:10E5B800FB89059396F87A110C920B4683F030028A
:10E5C80082EA0212D2B217094849099387F07A07FA
:10E5D80047EA02270988337187EAC202444FC1EB30
:10E5E800012187FB013A089B4FF0000C63F30F0CE5
:10E5F800079B6EF31F4C4FF0000E63F30F0E069B44
:10E60800CDF834C012B28A440027C91763F31F4EED
:10E61800C1EB6A2A059BCDF838E082EA021160F363
:10E628000F070020C9B268F30F00C2F3072269F38D
:10E638001F4782EA111263F31F404FF000090F973A
:10E648008DF845A010908DF8449042EA01220DF112
:10E65800300C82EAC107BCE80F003FB287F0C80857
:10E6680088EA0818DFF88CE086F805905FFA88F8E1
:10E67800C7F30727AEE80F0087EA181747EA082309
:10E688009CE8030083EAC8031BB283F023024EF818
:10E69800040B82EA0212D2B2C3F30723099F83EA6A
:10E6A8001213704643EA022383EAC20207F1010CFF
:10E6B80020F814194FF023081621FE27C82386F8DE
:10E6C8007AC1328086F807800EF1020EB770F170B9
:10E6D800B371114612E000BFC0410020A4410020E0
:10E6E800FF220020A842002092710020A4380020B8
:10E6F80003082080642100205E21002010F8013BDF
:10E708004B4083EA0313DBB21A0982EA112242EA78
:10E71800032282EAC3031BB299B270453180EDD15E
:10E7280083F0F40383EA0313DBB24FEA131E8EEA85
:10E73800112E8EEA032E8EEAC30E0FFA8EFE1FFAF2
:10E748008EF8E64FA6F800804FEA182C5FFA8EFE86
:10E7580086F81EE086F81FC07968BA683868FB68D2
:10E7680007F5D178A8E80F0038697969BA6906F21F
:10E77800A317A8E8070006F2C11886F8C1C186F8F1
:10E78800C0E117F8011F206801F08EFEB845F8D1E6
:10E7980096F87271002F40F0E885D14B96F87AE12F
:10E7A800B3F90010B3F90220B3F904309FEDCD6A34
:10E7B800777107EE103A039B1B680C938EF06A037F
:10E7C80083EA031306EE901AD9B20B0983F0D50336
:10E7D80043EA012383EAC1031BB283EA03115242CD
:10E7E800C9B207EE902AC3F3072383EA111343EA59
:10E7F8000123F8EEE77AF8EEE66AB8EEC77A83EA1C
:10E80800C1031BB267EE867A66EE866A27EE067A41
:10E81800002083F0C808CDED0E7ACDED0D6A8DEDA0
:10E828000F7A10901190129088EA081C0DF13009A7
:10E838005FFA8CFCC3F30728B9E80F0088EA1C18B4
:10E8480048EA0C2888EACC08DFF8A8C20FFA88F84A
:10E85800ACE80F0088F01E0799E8070087EA071759
:10E86800FFB2C8F3072383EA171343EA07238CE8A8
:10E87800070083EAC7071C20C8214FF005094FF09D
:10E888001E08FE230EF10102F07086F8729186F8D8
:10E898000780B3700CF10C00B171ACF1100186F86F
:10E8A80004E0378086F87A2111F8013B7B4083EA3F
:10E8B8000313DBB21A0982EA172242EA032282EA28
:10E8C800C3031BB29FB281423780EDD183F0270387
:10E8D80083EA0313DBB24FEA131E8EEA172E8EEA81
:10E8E800032E8EEAC30E0FFA8EFE1FFA8EF9DFF89A
:10E8F800ECC1A6F800905FFA8EFE4FEA192986F857
:10E90800259086F824E00CF5D17806F1220ADCF887
:10E918000000DCF80410DCF80820DCF80C3047466E
:10E928000FC70CF1100CD445B846F0D16E4FBCF8A7
:10E938000030A8F8003007F1240886F8C6E186F808
:10E94800C79117F8011F206801F0AEFDB845F8D14E
:10E9580096F873310393002B40F0038596F87AA15B
:10E968005F4B624AB3F90410B2F90620604FDFF832
:10E9780088C1DFF880E186F804A08AF0220080EAE6
:10E988000010C0B2030983F0590343EA002383EA65
:10E99800C0031BB2B2F5FA6F83EA0310C0B2A8BF76
:10E9A8004FF4FA62C3F30723B2F57A7F83EA1013B0
:10E9B80043EA0023B8BF4FF47A7283EAC000A2F595
:10E9C8007A72642303FB02F28CFB029CD31787FB49
:10E9D8000172C9174FF0000807B2C3EBAC13C1EBC3
:10E9E800A2010DF13009CDF83080CDF83480CDF892
:10E9F8003880CDF83C8087F0C80CADF84230ADF8CF
:10EA08004010C846B8E80F008CEA0C1C5FFA8CFC72
:10EA1800C7F3072787EA1C1747EA0C2787EACC07BA
:10EA2800AEE80F003FB287F04A0383EA0313DBB274
:10EA3800C7F3072181EA131141EA0321724681EAEB
:10EA4800C303D8F800C09DF80C1071710AF10107D2
:10EA580005204A214FF0FE0886F87A7142F810C95D
:10EA680014274FF0C80C86F8730133800EF1040E9A
:10EA7800F17186F80280F77086F806C0184612F819
:10EA8800011B414081EA0111C9B20B0983EA102335
:10EA980043EA012383EAC10109B288B27245308092
:10EAA800EDD181F0140181EA0111C9B24FEA111EBA
:10EAB8008EEA102E8EEA012E8EEAC10E0FFA8EFE15
:10EAC8001FFA8EFC4FEA1C2A044B044886F81DA046
:10EAD8005FFA8EFE86F81CE010E000BF5E21002081
:10EAE800C441002088C3E43AFF220020927100202C
:10EAF8006766666664210020D34D6210DA4F596854
:10EB08009A680068DB68A6F800C007F5D17CACE815
:10EB18000F0038697969B7F81880ACE8030006F285
:10EB2800A317ACF8008086F8BFA1B84686F8BEE106
:10EB380006F2BF1A18F8011F206801F0B5FCC2459B
:10EB4800F8D1CA4BCA4A1B781278013B12F001006F
:10EB5800DBB214BFC0214021172B03D8C54A134488
:10EB68001B7B0393C44B1A8893071ABF002341F0F9
:10EB78001001012312F4027F18BF022312F0100FB4
:10EB880018BF062312F0200F18BF1023002840F0EA
:10EB9800EA864FF0030C96F87AA10C938AF04603A4
:10EBA80083EA0313DAB2130983F0920343EA0223D8
:10EBB80083EAC2031BB283EA0310C0B2C3F307227D
:10EBC80082EA101242EA002282EAC00212B282F0FD
:10EBD800C80E8EEA0E1E00235FFA8EFE9DF80C808A
:10EBE8008DF834800320C2F307228DF837C082EAFB
:10EBF8001E128DF835308DF836108DF8380042EA3F
:10EC08000E2C99E807008CEACE0E0FFA8EFEDFF87C
:10EC18007482F3718EEA0E1CA8E803005FFA8CFC7C
:10EC2800CEF3072E8EEA1C1E4EEA0C2181EACC0C8C
:10EC380096F808E088F800200FFA8CFC8EEA0C0E93
:10EC48008EEA0E1E5FFA8EFECCF3072282EA1E12AF
:10EC580042EA0E22707AB17A96F80BC0737182EA92
:10EC6800CE0E0FFA8EFE80EA0E0080EA0012D2B2B3
:10EC7800CEF3072080EA121040EA022080EAC200A0
:10EC880000B2414081EA0111C9B2C0F3072282EA09
:10EC9800111242EA012282EAC10212B28CEA020C83
:10ECA8008CEA0C1C5FFA8CFCC2F3072282EA1C1265
:10ECB80042EA0C2296F80CE0707BB17B96F8109033
:10ECC80086F804A082EACC0212B28EEA020E8EEA1C
:10ECD8000E1E5FFA8EFEC2F3072282EA1E1242EA75
:10ECE8000E2282EACE0212B2504080EA0010C0B270
:10ECF800C2F3072282EA101242EA002282EAC00224
:10ED080012B2514081EA0111C9B2C2F3072282EA64
:10ED1800111242EA012282EAC102F17B13B281EAAE
:10ED2800030282EA0212D2B2C3F3072383EA121360
:10ED380043EA022383EAC2031BB289EA030282EA96
:10ED48000212D2B2C3F3072383EA121343EA02235F
:10ED580083EAC2031BB283F0320282EA0212D2B201
:10ED6800C3F3072383EA121343EA022383EAC203A5
:10ED78001BB29AB24FF0FE0C0AF10101DBB23280ED
:10ED88004FF0090EC82086F802C04FEA122CA8F1ED
:10ED98000E0286F803E0B07186F87A1186F812C080
:10EDA8000393737458F80E0C5168926838F802ACE3
:10EDB8009DF80C3008F5CA7EAEE8070008F5D27851
:10EDC8008EF80290AEF800A086F8B4C186F8B33188
:10EDD80017F8011F206801F067FBB845F8D1049BBC
:10EDE800C6F86431FFF7E8B9DFF89CA0DFF89C802B
:10EDF80041200DF0F7FDBAF9023088FB0320DB173C
:10EE0800C3EBA00080B20DF0D3FDBAF9003088FB47
:10EE18000320DB17C3EBA00080B20DF0C9FDBAF9DF
:10EE2800043088FB0320DB17C3EBA00080B20DF091
:10EE3800BFFD124B3868197801F036FB96F85C3143
:10EE480013F0010800F0BF830D4AC6F8589101334A
:10EE5800DBB2A2FB0312D20802EB8202A3EB42034D
:10EE680086F85C31FFF788B95E21002078510020D0
:10EE7800673E0020C432030814420020E0720020DC
:10EE8800CDCCCCCC64210020C441002067666666E6
:10EE98008B4B8C49186801F0D3FA00232370FFF7D5
:10EEA800E3B9894F386800283FF455A94FF0000AA4
:10EEB8002346DFF84882854E049554469A4601F069
:10EEC800EFFAF8B1F4B94FF001092546386801F0B6
:10EED800DFFA83B27E2B00F02D8298F80120002AF9
:10EEE8004BD196F84811C1B11B2B86F8482100F088
:10EEF800FB810D2B47D0386888F8019001F0D0FAD3
:10EF08000028E3D15346A24650460CAA7049049DF6
:10EF18001C460DF07FFDFFF71EB97D2B00F0F18335
:10EF280096F84C2122B180F02003DBB286F84C1110
:10EF380096F84721062A10D8B6F84A1138681944B5
:10EF4800A6F84A11B118013281F8503186F84721E4
:10EF580001F0A6FA0028B9D1D4E7B6F84A2188F812
:10EF6800019013449BB21A0A52FA83F3FF2BA6F8B6
:10EF78004A31386802D1574CA1E7386801F090FA55
:10EF88000028A3D1BEE73868A6F84A2101F088FA1C
:10EF980000289BD1B6E796F8B832C6F8B452012BD0
:10EFA80040F2068396F8B9224B49981801EB800184
:10EFB800013202F001024F6A86F8B922BFB1474C0C
:10EFC8000D940DF15009123CA52349F8204D8022DB
:10EFD80086F8103115232946484686F8112186F807
:10EFE8001231B847002840F0698296F8B8323C4A96
:10EFF800013382FB0312A2EBE37202EB42029B1A7B
:10F0080086F8B832FFF7E8B8364A374B92F80BE083
:10F01800039A1B881168D6F834213448891A4FF4AA
:10F028007A72DFB202FB0EF21B0A877707759142EC
:10F038004FF00007C37743758770077180F0A5828A
:10F048002B4B2C491A689B68C6F8305181FB02E7A4
:10F05800D21781FB03E1C2EBA702DB17C3EBA103C5
:10F0680011124FEA232C4FF0F40E02770127417753
:10F0780080F8203030217522782380F821C080F86C
:10F088001AE0C77680F8221080F8232080F8243010
:10F09800FEF7F3BF184B0493186801F0F5F9002840
:10F0A8003FF478A8049B0121186801F0E9F90222CD
:10F0B800002387F8742088F80030FFF76BB800BF8A
:10F0C8009C390020F0380020204200205C210020DC
:10F0D800A2220020AC220020C43203088122002092
:10F0E80056555555D83F0020D03F00206C39002098
:10F0F800B4410020676666664C6300200C0000205F
:10F108005E2090473B6802209847C74BC74AB3F92F
:10F118004C3082FB03124FEAE378C8EBA2080FFADF
:10F1280088F85FFA88F00DF04DFFC8F307200DF05E
:10F1380049FF3B685E2098473B6803209847BC4BD3
:10F148001B78D90740F120811FF09EFEB94B9FED37
:10F15800BA7AD3ED037A67EE877AFCEEE77ACDEDDB
:10F16800037ABDF80C30002800F06383D8B24FEA68
:10F1780013280DF027FF40460DF024FFAF4B1B78F6
:10F18800042B77D0DFF8E4A2B6F82E119AF8002005
:10F19800DFF8DC9291FBF2F302FB13139BB2B9F890
:10F1A8000010A6F82E314FEA03181FFA88F86423D6
:10F1B80003FB01235200B3FBF2F348EA0328C3F32D
:10F1C80003225E203B681FFA88F848EA020898473D
:10F1D8003B68062098475FFA88F00DF0F3FE4FEA87
:10F1E80018200DF0EFFE9649B6F82E214B7AB9F8A3
:10F1F80000900132012BA6F82E2100F08B854A7B66
:10F2080009EB89031FFA83F9002A40F0B6833B68AB
:10F218005E2098473B683A2098478A4BA3FB0938F9
:10F228004FEA58181FFA88FA5FFA8AF00DF0CAFEFA
:10F238004FEA1A200DF0C6FE3B685E2098473B68EF
:10F248003B209847642303FB18939BB27748053308
:10F2580080FB0320DB17C3EBA000C0B20DF0B2FEA9
:10F2680000200DF0AFFEDFF8F48198F80630002B8F
:10F2780040F0108396F82C313A68FEF7EBBEDFF8C1
:10F28800F4819FED718A4FF0240A5E209047504622
:10F298003B6898476D4BF8EC016A9B8A07EE103A79
:10F2A800F8EEE66AB8EEC77A0AF1010AC6EE877A7E
:10F2B8005FFA8AFA67EE887AFDEEE77ACDED037A8F
:10F2C800BDF90C905FFA89F00DF07CFEC9F30720B8
:10F2D8000DF078FEBAF1270F01D03A68D5E796F815
:10F2E8002C313A68FEF7B3BE386801F0D9F8002827
:10F2F8007FF401AE386886F8469188F8019001F0ED
:10F30800CFF800287FF4E2ADFCE5FEF74DFA504B4C
:10F318001B68A0EB030A40F6B8339A4500F2E68171
:10F328004C4A13793A2B00F0F783002388F8003011
:10F33800FEF730BF386886F8465186F8475186F898
:10F34800489188F8015001F0ABF800287FF4BEAD71
:10F35800D8E596F8441196F845313F484A1CFEF71F
:10F36800E6BE013B86F8733139E5013F86F87271D4
:10F37800FFF7EEBA013B86F86A31FFF7E7B8013BC1
:10F3880086F86B31FFF704BA344A354BB2F8088077
:10F39800A3FB08384FEA98085FFA88F00DF012FED0
:10F3A8004FEA18200DF00EFEE8E64FF0000A5E2046
:10F3B800D3F8008086F82CA190473B68DFF8B89016
:10F3C8001720984750460DF0FDFD264BA3FB082358
:10F3D8009B0BA9FB03125209C2EB0212A3EB820397
:10F3E800D8B20DF0EFFD3B685E2098473B681820C7
:10F3F80098471D4BA3FB08239B09A9FB031252093D
:10F40800C2EB0212A3EB8203D8B20DF0DBFD50462B
:10F418000DF0D8FD3A68FEF722BE0024DFF85C80C4
:10F42800A1464FF0500A2EE0DC4800206766666669
:10F43800673E0020E83F0020CDCC4C3EA838002095
:10F44800D83F00201F85EB5100007A44CC410020B2
:10F45800346200201C62002024420020A4410020C5
:10F46800CDCCCCCC73B2E745D34D6210E63F00203B
:10F47800D03F0020FC41002089888888F1A301083A
:10F48800DBB283F3118816F804B0601C5946304487
:10F498000DF0A2F9002840F048810BF101031C444B
:10F4A800EFF311838AF31288326E9442E8DB00226C
:10F4B800DBB2326683F31188FEF746BF0C9DA54286
:10F4C8004FF000014FD941F2210014F8013B81EAC5
:10F4D80003235A0013F4004F80EA020192B289B262
:10F4E80008BF11464A0080EA020311F4004F99B29E
:10F4F80093B218BF0B46590080EA010213F4004F7B
:10F5080089B293B208BF0B465A0013F4004F80EA41
:10F51800020192B289B208BF11464A0080EA02038A
:10F5280011F4004F99B293B218BF0B465A0013F466
:10F53800004F80EA020192B289B208BF11464B001F
:10F5480011F4004F80EA03029BB292B208BF1A4638
:10F55800510080EA010312F4004F9BB289B218BF30
:10F568001946AC42B1D14846F1F722FCB6490C9C89
:10F57800B648641A152CA8BF1524224622F06AF949
:10F58800B34A96F8B832147031E5B24B039A1B7837
:10F598001268C6F83421013B012B3FF651AD102209
:10F5A8000223827003714BE50DF0EEFCFEF7C7BD38
:10F5B800A94A02EB8302576A00E50DF0D5FC012346
:10F5C8003B70FEF779BDA54B1B88DA0515D4D80624
:10F5D80000F17A83990600F1AD835A0600F1B083F1
:10F5E800180700F1B083D90700F1B08313F0020FB8
:10F5F8000CBF4FF004084FF00C08994B994A1B7840
:10F60800D27803F001030AB143F0020353200493B4
:10F618000DF0E8F9944A128802EB820202EB8202AA
:10F62800900080B20DF0C4F900200DF0C1F98F4AA6
:10F638008F4912883868C2EBC212520081FB02312E
:10F6480011444FEAE27ACAEB612A5FFA8AFA514614
:10F6580000F02AFF874B38681A78049B48EA0308A9
:10F66800844B8AEA020A002183F800A000F01CFFFC
:10F678004146386800F018FF7E4B7E4A1B78386890
:10F6880088EA0303DBB21946137000F00DFF96F801
:10F698005C31002B7FF4D8AB4F200DF0A3F920F09C
:10F6A80093FC20F091FC20F08FFC0121386800F0D9
:10F6B800FBFE714A6F4B92F800801B786D4A3868E0
:10F6C80008F0010883F001034146137000F0ECFED6
:10F6D800684B684A1B78386888EA03031946137030
:10F6E80000F0E2FE96F85C31FFF7AEBB634AB2F871
:10F6F8005E3100210133A2F85E3188F80010FEF770
:10F7080049BD386886F84C9100F0CAFE00287FF49D
:10F71800DDABFFF7F7BB8846894608460691079197
:10F728008E4608910591FEF745BF41463A200CF0F8
:10F73800AFFF40EA09095FFA89F9AEE65049514B33
:10F748000093A1F13F07504B504A0B9101F8404CF0
:10F758000CA84F490A97F1F703FC0A9F7B1C0A93F0
:10F768003C700A9B2922591C0A911A700A9BEA22AA
:10F77800591C0A911A700A9BC822591C0A910CA894
:10F788001A7021F0F9F800F101080CA942460A980C
:10F7980022F060F80A9A02EB080301330A9302F890
:10F7A80008400A9B5A1C0A921C700A9B5A1C0A920F
:10F7B8001C700A9B5A1C0A921C700A9B5A1C0A92BB
:10F7C8001C700A9B5A1C0A921C700A9B5A1C0A92AB
:10F7D8001C700A9B5A1C0A921C700A9B5A1C0A929B
:10F7E8001C700A9B5A1C0A921C700A9B5A1C0A928B
:10F7F8001C700A9B5A1C0A921C700A9B5A1C0A927B
:10F808001C700A9B0122991814A80A911A7050F8C2
:10F81800283DDB1B3B700AF0CDFD184B3470C3F854
:10F82800AC52FEF7CDBCC6F8385187F80090FEF709
:10F8380043BCDBF80020D2067FF598AC804698E4FC
:10F8480000F01EFEFEF74DBC6C220020045B002079
:10F85800195B0020A8380020C43203081442002095
:10F86800673E0020C0420020D03F0020A43800207E
:10F8780003082080E0720020845100205C210020D1
:10F88800F03800207E420020485A0308505A0308E6
:10F898005C5A03083B68DFF87492DFF86CA25E20BC
:10F8A80098473B6828209847D9F800308AFB032AF4
:10F8B800DB17C3EBAA0A5FFA8AF00DF083FBCAF3E1
:10F8C80007200DF07FFB3B685E2098473B680420CB
:10F8D8009847B8F80830002B40F00182D9F8083072
:10F8E80083F310085FFA88F00DF06CFBC8F307206B
:10F8F8000DF068FBBEE47A4B7A4A0D93A3F14008F9
:10F908001268002103F8401C212388F80230D30034
:10F9180040F1F48174490327744B1B88580500F1A2
:10F92800EA81DA0700F1098203F00203704A002B2A
:10F938001CBF03271146DFF8D8913A46484621F004
:10F9480089FF07EB090314A80133A9F1020140F864
:10F95800203D00225B1A07F8092088F801300AF0D8
:10F9680029FDFEF7A4BC634AD278002A0CBF4FF0E9
:10F97800040C4FF0050CFFF70EB99AF8003099FB0C
:10F98800F3F944E40123D8F800003B7000F080FD4F
:10F998000746D8F8000000F07BFD79067EF48CABB2
:10F9A8008E287EF489AB9AF80030002B7EF4A0AB49
:10F9B800514B524A1A602D2386F83C31FEF783BB1F
:10F9C800DFF850919FED4E8AB9F90230444A0D9202
:10F9D80007EE903AF8EEE77A0DF1500867EE887A6C
:10F9E800A2F14003FDEEE77AA2F13D0148F8201D9F
:10F9F80002F8400C0822CDED037A5A701E229A7044
:10FA0800BDF80C104046F1F7ADF9B9F9003007EE32
:10FA1800903AF8EEE77A404667EE887AFDEEE77AA4
:10FA2800CDED037ABDF80C10F1F79CF9B9F9043063
:10FA380007EE903AF8EEE77A404667EE887AFDEEF0
:10FA4800E77ACDED037ABDF80C10F1F78BF9404653
:10FA58000AF0B0FCFEF725BC214A2A4B0D920DF1A5
:10FA68005008A2F13D0048F8200D1988DFF89C9055
:10FA7800A2F1400300204FF00A0E02F8400C0822C1
:10FA880083F801E040469A70F1F76CF9D9F8003034
:10FA98001D49DA1781FB0313C2EBA30399B2404651
:10FAA800F1F760F903F090FCD9F808900C9B4FEA45
:10FAB8001942591C0C911A700C9B4FEA1922591CB7
:10FAC8000C911A700C9B5A1C0C9283F800900C9B9A
:10FAD8005A1C0C92187040460AF06CFCFEF7E4BB06
:10FAE800F038002090600020345A030814420020A7
:10FAF800445A0308C04200202C4200206C390020E0
:10FB080058A08B41D03F002067666666B44100204C
:10FB1800B3380020C44100209178049210461DF0AB
:10FB280059FB049A00287FF400AC9349934F944BF7
:10FB3800944E09880592944AF961F863B6F85E1103
:10FB480018689B68C7F86CA0F862FB641068F965D0
:10FB5800049200F05BFA824600287EF416AB049B00
:10FB68004946186800F08CFC059A96F86031D278FE
:10FB78000692642B4FF0040287F8742040F0168137
:10FB880096F86131072B08BF86F861A196F86131B4
:10FB9800089307EB0319D9F804100591084620F0DB
:10FBA800EBFED9F8081007915FFA80F9084620F0B3
:10FBB800E3FE5FFA80FA089B74480599059009EB03
:10FBC8000A020832C27123F00F0282726F4A03F0F0
:10FBD8000F0353736D4B0AEBC900987318464A46D6
:10FBE8000F3021F037FE6A4B079909F109001844D4
:10FBF800524621F02FFE0598C37903F10109CBB1D4
:10FC0800013B5FFA83FC0CF1080CDFF89CE18444AB
:10FC18000023073010F8012B5A409300D10883EADB
:10FC2800420301F0180153404EFA01F25340844553
:10FC3800DBB2EFD1564A069809F8023021F0E6FD0A
:10FC480096F861310022013386F8613186F8602127
:10FC5800059BDDF814909B785BB1049B19F80410A0
:10FC6800186800F021FC013499F80230E4B2A3428C
:10FC7800F3D896F860310322013386F8603187F8AB
:10FC8800742088F80020049BFFF706BA3C4B804696
:10FC9800B3F900A06420FEF794BB374B3D4A1B889C
:10FCA800927903EB830303EB83034FEA83081FFA7C
:10FCB80088F8002A54D14FF0FF330FFA83FA03F083
:10FCC80083FB40B2FEF77DBB4FF0340895E49846BD
:10FCD80099461846069307930593FEF76BBC03F005
:10FCE80073FB0DF06FF900200DF06CF996F82C31CC
:10FCF8003A68FEF7AFB9032727491CE6DBF800305E
:10FD0800264A274903F48003002B16BF114604270F
:10FD1800032701E63B685E2098473B6839209847EF
:10FD28005FFA89F00DF04EF94FEA19200DF04AF903
:10FD3800FFF799BA4FF024085FE41A490427FAE557
:10FD48004FF0100859E44FF0200856E44FF0080827
:10FD580053E498469946184606930593FEF72ABC3D
:10FD6800074B1B68A9E798469946184606930793D8
:10FD78009E460593FEF71EBCD03F00200C000020D5
:10FD8800B44100205C2100204C6300200C66002058
:10FD980012660020A4410020385A0308345A030888
:10FDA8002C5A03083C5A03080007090E97F8759067
:10FDB8004B494C4A059219F00F0F04BF09F101098C
:10FDC8005FFA89F9B9F1070F28BF4FF001094FEA27
:10FDD800091A07EB0A035FFA8AFC187C0023095CFE
:10FDE800937202F10D0307EB0A024CEA00000129A5
:10FDF8001870D26803F1010E0CD90239C9B2881CF7
:10FE08001844734603F8012B83424FEA1222F9D1B2
:10FE180001318E44BA4422F0600309F101099AF8CD
:10FE280011205FFA89F91343B9F1080F8EF80030F1
:10FE38000EF1010351D04FEA091A07EB0A012A4AC9
:10FE4800087C2749095C9A1A02EB010E0CF1100C88
:10FE5800BEF1130F5FFA8CFCC5DDD2B2931DDBB285
:10FE68000598DFF88CE043F04001C17103F1010C03
:10FE7800CBB105325FFA82FA0AF1080A82440023FC
:10FE88000EF1010010F8011B59408B0083EA410371
:10FE9800CA084B40154902F0180241FA02F25340D1
:10FEA8008245DBB2EED106980CF80E3087F87590D3
:10FEB80021F0ACFCCCE60593FEF77CBB9846059395
:10FEC800FEF778BB984699460593FEF773BB9846AC
:10FED800994618460593FEF76DBB034A9A1ABCE784
:10FEE800C43203080C660020196600200007090EBA
:10FEF80012660020436A8269D154436A0169826BA1
:10FF080001338B4228BF00234362002A2FD0EFF32E
:10FF18001181502383F31288836B1A68D2072CD47B
:10FF280070B45E686EB9456A826A954217D0846972
:10FF38001444DC600ED9AA1A5A608562002280F83F
:10FF480054201A6842F00102C9B21A6081F311887C
:10FF580070BC70470469A21A5A608662EEE70123F2
:10FF680080F85430C9B281F3118870BC7047026DB3
:10FF7800136843F0800313607047C9B281F3118896
:10FF8800704700BF426B10B462B1436CC2684469E9
:10FF9800D11A013B615C5DF8044B08BF134643640A
:10FFA800C8B27047016A4369C4685B5C0131A14209
:10FFB80028BF114601625DF8044BD8B2704700BFF4
:10FFC800836B13B190F854007047836A406A181A1B
:10FFD800B0FA80F040097047416A836A99420AD3AF
:10FFE800CB1A816B026961B14968501E0B44834288
:08FFF8000AD2C01A7047026929
:020000040801F1
:100000001144CB1A816B0029F2D1501EC01A7047DF
:1000100000207047436B43B1426C5B6893422FBF33
:10002000981AC0689B1AC0187047C269036A9A423E
:100030002FBFD01AC0688018C01A70470A4B30B55D
:1000400003F1140493F900205D78072AC8BF143A1D
:10005000811804330D7313F8025C855413F8012CD6
:100060000A76A342EED130BDF832030803682DE9C9
:10007000F041DF691FB13B46BDE8F0411847002A57
:10008000164611DD04460D460E4400E023689B68C9
:10009000204698470028F9D0236815F8011B1B68F3
:1000A00020469847AE42F1D1BDE8F08100232522D9
:1000B000027043708370C37070472D2343702E23EA
:1000C00003712F23C371704730B50446006D617111
:1000D0000368A26823F00103036087B0A37900924C
:1000E00013F004023DD04FF4805213F0020301924A
:1000F00044D102934FF480630022039311F0010373
:10010000059237D1049308238D07694648BF0493AD
:100110000BF024FC6079236DA17900F00202002A23
:1001200015BF4FF440324FF480324FF400340024B6
:1001300010F0010F586808BF2246CC074CBF02439D
:1001400020EA02025A609A6809074CBF42F008028E
:1001500022F008029A601A6842F001021A6007B0A1
:1001600030BD13F0020301920BD04FF4005513463B
:100170000295C1E7042304930C23C5E74FF4005311
:10018000B7E70293B8E700BF10B50446006DA16061
:10019000036823F001030360A37986B013F004021F
:1001A000009141D04FF4805213F00203019244D1E8
:1001B00002934FF4806362790393D1074FF00003F9
:1001C0000493059345BF0423049308230C23694635
:1001D000920748BF04930BF0C1FB6079236DA179AE
:1001E00000F00202002A15BF4FF440324FF4803273
:1001F0004FF40034002410F0010F586808BF224665
:10020000CC074CBF024320EA02025A609A680907F1
:100210004CBF42F0080222F008029A601A6842F0CD
:1002200001021A6006B010BD13F00203019207D05C
:100230004FF4005113460291BDE74FF40053B7E766
:100240000293B8E700231922036042701A22C27099
:10025000012243604271C371704700BF1D4B70B5EE
:100260009C68236D626BDD69C2B1A36B2BB12B0758
:1002700002D5236D08221A6270BD2A06F7D5A26A3C
:10028000616A8A4220D0511CA069A162825C206907
:10029000266D81423285EAD3A362E8E7A906E4D558
:1002A000E26A22B1988C216B80B29047DDE7E16968
:1002B0009B8C6069DBB24E1CE6614354E169E368E4
:1002C000994228BFE261D0E7226D136823F08003D2
:1002D0001360CCE7502C00201D4B70B55C68236D7B
:1002E000626BDD69C2B1A36B2BB12B0702D5236D05
:1002F00008221A6270BD2A06F7D5A26A616A8A428C
:1003000020D0511CA069A162825C2069266D8142C7
:100310003285EAD3A362E8E7A906E4D5E26A22B10E
:10032000988C216B80B29047DDE7E1699B8C606916
:10033000DBB24E1CE6614354E169E368994228BF91
:10034000E261D0E7226D136823F080031360CCE7ED
:10035000502C00201D4B70B51C68236D626BDD694D
:10036000C2B1A36B2BB12B0702D5236D08221A62F1
:1003700070BD2A06F7D5A26A616A8A4220D0511C54
:10038000A069A162825C2069266D81423285EAD330
:10039000A362E8E7A906E4D5E26A22B1988C216B52
:1003A00080B29047DDE7E1699B8C6069DBB24E1C4F
:1003B000E6614354E169E368994228BFE261D0E70E
:1003C000226D136823F080031360CCE7502C0020CB
:1003D00070B4EFF31186502383F31288836B1A688D
:1003E000D20720D45D686DB9446A826A944217D0FE
:1003F00081691144D9600ED9A21A5A608462002220
:1004000080F854201A6842F00102F1B21A6081F3B8
:10041000118870BC704701698A1A5A608562EEE7DC
:10042000012380F85430F1B281F3118870BC704719
:1004300003685B6A03B11847704700BF03681B6A13
:1004400003B11847704700BF03682DE9F041DF6929
:100450001FB13B46BDE8F0411847002A164611DDA2
:1004600004460D460E4400E023689B6820469847EA
:100470000028F9D0236815F8011B1B68204698470F
:10048000AE42F1D1BDE8F08103689B69184700BF17
:1004900003685B69184700BF0368DB68184700BF43
:1004A00003689B68184700BF03685B68184700BF74
:1004B00003681B68184700BF054B53F8203033B161
:1004C0001A689B88918A0B4218BF1B04936170477E
:1004D000B864002003682DE9F04F03F13845644EFD
:1004E000AD0A0124755D05F01F066D09022D04FAA1
:1004F00006F400F0A280032D00F0A480012D52D05C
:100500008088B0FA80F4C4F11F04A4B2E50803EBBC
:10051000850504F007042E6AA4000F27A74026EAE9
:1005200007062E622E6A01F0030702FA04F47A1E0F
:100530003443012AC1F3810CC1F300182C62C1F3CA
:10054000411135D9C60700F19780850700F1A380D6
:10055000440700F1B180020700F1BF80C60600F138
:10056000CD80850600F1DB80440600F1E9800206BB
:1005700000F1F780C60500F10581850500F11381C2
:10058000440500F12181020500F12F81C60400F12C
:100590003D81850400F14B81440400F1598102043E
:1005A00055D4BDE8F08F334D6E6934436C61A7E7D5
:1005B000002422464FF0010E4FF0030904E00132FF
:1005C000102A04F10204ECD00EFA02F636EA000515
:1005D000F5D1D3F808A009FA04F5ED430AEA050AB3
:1005E000C3F808A0D3F808B00CFA04FA4AEA0B0AD8
:1005F000C3F808A0B3F804A01FFA8AFA2AEA06068C
:100600009E80B3F804A008FA02F646EA0A06B6B2DB
:100610009E801E682E401E60D3F800A007FA04F6E4
:1006200046EA0A061E60D3F80CA001FA04F605EAB1
:100630000A0A46EA0A05DD60C1E70E4DAE69344399
:10064000AC615DE70B4DEE693443EC6158E71A6825
:1006500022F040421A601A6842EA87771F60DA681F
:1006600022F0404242EA8171D960BDE8F08F00BFBC
:10067000B4540308001002401A6822F003021A6002
:100680001A683A431A60DA6822F003020A438507BF
:10069000DA607FF55DAF1A6822F00C021A601A6802
:1006A00042EA87021A60DA6822F00C0242EA81020A
:1006B0004407DA607FF54FAF1A6822F030021A6003
:1006C0001A6842EA07121A60DA6822F0300242EA37
:1006D0000112DA6002077FF541AF1A6822F0C0020A
:1006E0001A601A6842EA87121A60DA6822F0C002B9
:1006F00042EA8112C606DA607FF533AF1A6822F447
:1007000040721A601A6842EA07221A60DA6822F414
:10071000407242EA01228506DA607FF525AF1A6849
:1007200022F440621A601A6842EA87221A60DA6884
:1007300022F4406242EA81224406DA607FF517AF74
:100740001A6822F440521A601A6842EA07321A60A4
:10075000DA6822F4405242EA0132DA6002067FF59A
:1007600009AF1A6822F440421A601A6842EA8732D6
:100770001A60DA6822F4404242EA8132C605DA6041
:100780007FF5FBAE1A6822F440321A601A6842EA1A
:1007900007421A60DA6822F4403242EA01428505D3
:1007A000DA607FF5EDAE1A6822F440221A601A680A
:1007B00042EA87421A60DA6822F4402242EA814221
:1007C0004405DA607FF5DFAE1A6822F440121A6041
:1007D0001A6842EA07521A60DA6822F4401242EAC2
:1007E0000152DA6002057FF5D1AE1A6822F44002A8
:1007F0001A601A6842EA87521A60DA6822F44002E4
:1008000042EA8152C604DA607FF5C3AE1A6822F06C
:1008100040721A601A6842EA07621A60DA6822F0C7
:10082000407242EA01628504DA607FF5B5AE1A686B
:1008300022F040621A601A6842EA87621A60DA6837
:1008400022F0406242EA81624404DA607FF5A7AE9A
:100850001A6822F040521A601A6842EA07721A6057
:10086000DA6822F0405242EA0172DA6097E600BF8D
:10087000036803F138422DE9F04F920A584DAA5C03
:1008800002F01F0552090124022A04FA05F400F0BF
:100890008C80032A00F08E80012A3CD001F00307EF
:1008A0007A1E012AC1F3810CC1F300188088C1F3BC
:1008B000411135D9C60700F19780850700F1A38063
:1008C000440700F1B180020700F1BF80C60600F1C5
:1008D000CD80850600F1DB80440600F1E980020648
:1008E00000F1F780C60500F10581850500F113814F
:1008F000440500F12181020500F12F81C60400F1B9
:100900003D81850400F14B81440400F159810204CA
:1009100055D4BDE8F08F334A55692C435461BDE787
:10092000002422464FF0010E4FF0030904E001328B
:10093000102A04F10204ECD00EFA02F636EA0005A1
:10094000F5D1D3F808A009FA04F5ED430AEA050A3F
:10095000C3F808A0D3F808B00CFA04FA4AEA0B0A64
:10096000C3F808A0B3F804A01FFA8AFA2AEA060618
:100970009E80B3F804A008FA02F646EA0A06B6B268
:100980009E801E682E401E60D3F800A007FA04F671
:1009900046EA0A061E60D3F80CA001FA04F605EA3E
:1009A0000A0A46EA0A05DD60C1E70E4A95692C434A
:1009B000946173E70B4AD5692C43D4616EE71A68DA
:1009C00022F040421A601A6842EA87771F60DA68AC
:1009D00022F0404242EA8171D960BDE8F08F00BF49
:1009E000B4540308001002401A6822F003021A608F
:1009F0001A683A431A60DA6822F003020A4385074C
:100A0000DA607FF55DAF1A6822F00C021A601A688E
:100A100042EA87021A60DA6822F00C0242EA810296
:100A20004407DA607FF54FAF1A6822F030021A608F
:100A30001A6842EA07121A60DA6822F0300242EAC3
:100A40000112DA6002077FF541AF1A6822F0C00296
:100A50001A601A6842EA87121A60DA6822F0C00245
:100A600042EA8112C606DA607FF533AF1A6822F4D3
:100A700040721A601A6842EA07221A60DA6822F4A1
:100A8000407242EA01228506DA607FF525AF1A68D6
:100A900022F440621A601A6842EA87221A60DA6811
:100AA00022F4406242EA81224406DA607FF517AF01
:100AB0001A6822F440521A601A6842EA07321A6031
:100AC000DA6822F4405242EA0132DA6002067FF527
:100AD00009AF1A6822F440421A601A6842EA873263
:100AE0001A60DA6822F4404242EA8132C605DA60CE
:100AF0007FF5FBAE1A6822F440321A601A6842EAA7
:100B000007421A60DA6822F4403242EA014285055F
:100B1000DA607FF5EDAE1A6822F440221A601A6896
:100B200042EA87421A60DA6822F4402242EA8142AD
:100B30004405DA607FF5DFAE1A6822F440121A60CD
:100B40001A6842EA07521A60DA6822F4401242EA4E
:100B50000152DA6002057FF5D1AE1A6822F4400234
:100B60001A601A6842EA87521A60DA6822F4400270
:100B700042EA8152C604DA607FF5C3AE1A6822F0F9
:100B800040721A601A6842EA07621A60DA6822F054
:100B9000407242EA01628504DA607FF5B5AE1A68F8
:100BA00022F040621A601A6842EA87621A60DA68C4
:100BB00022F0406242EA81624404DA607FF5A7AE27
:100BC0001A6822F040521A601A6842EA07721A60E4
:100BD000DA6822F0405242EA0172DA6097E600BF1A
:100BE00010B50409013C052C17D80D4B33F814201F
:100BF00000F00F0042FA00F313F001030DD00123BF
:100C000003FA00F00138104020F0B4FB054A064B0F
:100C1000125D104403EBC00010BD002010BD00BFEA
:100C2000904C03089C4C0308904700202DE9F04F9E
:100C30004A484B4B4B4C4FF090414FF0010A4FF05C
:100C400002094FF004084FF0080C4FF0100E202757
:100C50004026802530F8022B12F0010F03D01960D6
:100C6000A3F804A0083312F0020F03D01960A3F810
:100C70000490083312F0040F03D01960A3F8048025
:100C8000083312F0080F03D01960A3F804C008332A
:100C900012F0100F03D01960A3F804E0083312F02B
:100CA000200F02D019609F80083312F0400F02D04D
:100CB00019609E80083312F0800F02D019609D8069
:100CC000083312F4807F05D04FF4807B1960A3F8BD
:100CD00004B0083312F4007F05D04FF4007B196094
:100CE000A3F804B0083312F4806F05D04FF4806B82
:100CF0001960A3F804B0083312F4006F05D04FF464
:100D0000006B1960A3F804B0083312F4805F05D0BB
:100D10004FF4805B1960A3F804B0083312F4005F4D
:100D200005D04FF4005B1960A3F804B0083312F447
:100D3000804F05D04FF4804B1960A3F804B00833FE
:100D4000D20B04D04FF4004219609A80083301F5A9
:100D50008061A1427FF47EAFBDE8F08F904C030824
:100D60009047002000180048002867D003682DE94C
:100D7000F04F03F138445C4EA40A0125345D04F0C1
:100D80001F066409022C05FA06F558D0032C00F062
:100D9000A580012C58D08088B0FA80F4C4F11F04DB
:100DA000A4B2E50803EB850504F007042E6AA4004D
:100DB0000F27A74026EA07062E622E6A01F00307D6
:100DC000A2407C1E3243012CC1F3810CC1F30018F8
:100DD0002A62C1F341113CD9C60700F18980850719
:100DE00000F19580440700F1A380020700F1B18073
:100DF000C60600F1BF80850600F1CD80440600F1F3
:100E0000DB80020600F1E980C60500F1F780850568
:100E100000F10581440500F11381020500F12181F3
:100E2000C60400F12F81850400F13D81440400F1E6
:100E30004B81020400F15981BDE8F08F70472B4CC3
:100E4000A6693543A561A6E7284C66693543656107
:100E5000A1E7002422464FF0010E4FF0030904E001
:100E60000132102A04F10204E6D00EFA02F636EA44
:100E70000005F5D1D3F808A009FA04F5ED430AEA14
:100E8000050AC3F808A0D3F808B00CFA04FA4AEA35
:100E90000B0AC3F808A0B3F804A01FFA8AFA2AEADA
:100EA00006069E80B3F804A008FA02F646EA0A068F
:100EB000B6B29E801E682E401E60D3F800A007FACE
:100EC00004F646EA0A061E60D3F80CA001FA04F6FE
:100ED00005EA0A0A46EA0A05DD60C1E7034CE6694D
:100EE0003543E56157E700BFB454030800100240E2
:100EF0001A6822F003021A601A683A431A60DA6824
:100F000022F003020A438507DA607FF56BAF1A68A7
:100F100022F00C021A601A6842EA87021A60DA6844
:100F200022F00C0242EA81024407DA607FF55DAFED
:100F30001A6822F030021A601A6842EA07121A6030
:100F4000DA6822F0300242EA0112DA6002077FF525
:100F50004FAF1A6822F0C0021A601A6842EA87127C
:100F60001A60DA6822F0C00242EA8112C606DA602C
:100F70007FF541AF1A6822F440721A601A6842EA9B
:100F800007221A60DA6822F4407242EA01228506DA
:100F9000DA607FF533AF1A6822F440621A601A688B
:100FA00042EA87221A60DA6822F4406242EA812229
:100FB0004406DA607FF525AF1A6822F440521A60C1
:100FC0001A6842EA07321A60DA6822F4405242EAAA
:100FD0000132DA6002067FF517AF1A6822F4404248
:100FE0001A601A6842EA87321A60DA6822F44042CC
:100FF00042EA8132C605DA607FF509AF1A6822F449
:1010000040321A601A6842EA07421A60DA6822F42B
:10101000403242EA01428505DA607FF5FBAE1A688C
:1010200022F440221A601A6842EA87421A60DA689B
:1010300022F4402242EA81424405DA607FF5EDAEB7
:101040001A6822F440121A601A6842EA07521A60BB
:10105000DA6822F4401242EA0152DA6002057FF5B2
:10106000DFAE1A6822F440021A601A6842EA875218
:101070001A60DA6822F4400242EA8152C604DA6059
:101080007FF5D1AE1A6822F040721A601A6842EAFF
:1010900007621A60DA6822F0407242EA016285044F
:1010A000DA607FF5C3AE1A6822F040621A601A68EF
:1010B00042EA87621A60DA6822F0406242EA81629C
:1010C0004404DA607FF5B5AE1A6822F040521A6027
:1010D0001A6842EA07721A60DA6822F0405242EA5D
:1010E0000172DA6002047FF5A7AE1A6822F040426E
:1010F0001A601A6842EA87771F60DA6822F0404275
:1011000042EA8171D960BDE8F08F00BF002852D05B
:10111000036803F138422DE9F04F920A504DAA5C62
:1011200002F01F0552090124022A04FA05F443D0F3
:10113000032A00F09080012A43D001F003077A1EB1
:10114000012AC1F3810CC1F300188088C1F3411159
:101150003CD9C60700F18880850700F194804407D8
:1011600000F1A280020700F1B080C60600F1BE8047
:10117000850600F1CC80440600F1DA80020600F119
:10118000E880C60500F1F680850500F1048144057C
:1011900000F11281020500F12081C60400F12E81C8
:1011A000850400F13C81440400F14A81020400F10D
:1011B0005881BDE8F08F70472A4A95692C439461A5
:1011C000BBE7284A55692C435461B6E70024224600
:1011D0004FF0010E4FF0030904E00132102A04F130
:1011E0000204E6D00EFA02F636EA0005F5D1D3F88D
:1011F00008A009FA04F5ED430AEA050AC3F808A0B5
:10120000D3F808B00CFA04FA4AEA0B0AC3F808A0AB
:10121000B3F804A01FFA8AFA2AEA06069E80B3F8F9
:1012200004A008FA02F646EA0A06B6B29E801E68D4
:101230002E401E60D3F800A007FA04F646EA0A061C
:101240001E60D3F80CA001FA04F605EA0A0A46EA81
:101250000A05DD60C1E7034AD5692C43D4616CE718
:10126000B4540308001002401A6822F003021A6006
:101270001A683A431A60DA6822F003020A438507C3
:10128000DA607FF56CAF1A6822F00C021A601A68F7
:1012900042EA87021A60DA6822F00C0242EA81020E
:1012A0004407DA607FF55EAF1A6822F030021A60F8
:1012B0001A6842EA07121A60DA6822F0300242EA3B
:1012C0000112DA6002077FF550AF1A6822F0C002FF
:1012D0001A601A6842EA87121A60DA6822F0C002BD
:1012E00042EA8112C606DA607FF542AF1A6822F43C
:1012F00040721A601A6842EA07221A60DA6822F419
:10130000407242EA01228506DA607FF534AF1A683E
:1013100022F440621A601A6842EA87221A60DA6888
:1013200022F4406242EA81224406DA607FF526AF69
:101330001A6822F440521A601A6842EA07321A60A8
:10134000DA6822F4405242EA0132DA6002067FF59E
:1013500018AF1A6822F440421A601A6842EA8732CB
:101360001A60DA6822F4404242EA8132C605DA6045
:101370007FF50AAF1A6822F440321A601A6842EA0E
:1013800007421A60DA6822F4403242EA01428505D7
:10139000DA607FF5FCAE1A6822F440221A601A68FF
:1013A00042EA87421A60DA6822F4402242EA814225
:1013B0004405DA607FF5EEAE1A6822F440121A6036
:1013C0001A6842EA07521A60DA6822F4401242EAC6
:1013D0000152DA6002057FF5E0AE1A6822F440029D
:1013E0001A601A6842EA87521A60DA6822F44002E8
:1013F00042EA8152C604DA607FF5D2AE1A6822F062
:1014000040721A601A6842EA07621A60DA6822F0CB
:10141000407242EA01628504DA607FF5C4AE1A6860
:1014200022F040621A601A6842EA87621A60DA683B
:1014300022F0406242EA81624404DA607FF5B6AE8F
:101440001A6822F040521A601A6842EA07721A605B
:10145000DA6822F0405242EA0172DA6002047FF553
:10146000A8AE1A6822F040421A601A6842EA8777EA
:101470001F60DA6822F0404242EA8171D960BDE81B
:10148000F08F00BF10B1036882881A85704700BFD3
:1014900010B1036882889A61704700BF38B1002993
:1014A0008388026814BF002110218B40936170472C
:1014B0000E4B1B8801463BB90D4B0E4A1B7810683A
:1014C0000BB981F00101E9E70B4B5A691AB118B960
:1014D0001A68106058747047084A18681188084ADA
:1014E00092FBF1F20121026059747047C46400203C
:1014F000C6640020C8640020CC640020E46400209E
:1015000020A1070010B40A4B0A4A1C78012383402B
:10151000234052F8200029B9B3FA83F149095DF854
:10152000044BBBE7191C18BF01215DF8044BB5E75C
:10153000B4640020B864002030B1036882881B8A3C
:101540001A4214BF01200020704700BF2DE9F0416E
:101550000B4E346873691C400FD0DFF828800127D8
:10156000B4FA84F3C3F11F0307FA03F558F8230014
:1015700003689847AC437561F2D1BDE8F08100BFC4
:10158000000401404C5800202DE9F0410B4E346816
:1015900073691C400FD0DFF828800127B4FA84F368
:1015A000C3F11F0307FA03F558F8230003689847AF
:1015B000AC437561F2D1BDE8F08100BF0004014089
:1015C0004C5800202DE9F0410B4E346873691C40E3
:1015D0000FD0DFF828800127B4FA84F3C3F11F038A
:1015E00007FA03F558F8230003689847AC43756180
:1015F000F2D1BDE8F08100BF000401404C5800204A
:101600002DE9F0410B4E346873691C400FD0DFF8B0
:1016100028800127B4FA84F3C3F11F0307FA03F506
:1016200058F8230003689847AC437561F2D1BDE8D0
:10163000F08100BF000401404C5800202DE9F0412A
:101640000B4E346873691C400FD0DFF828800127E7
:10165000B4FA84F3C3F11F0307FA03F558F8230023
:1016600003689847AC437561F2D1BDE8F08100BFD3
:10167000000401404C5800202DE9F0410B4E346825
:1016800073691C400FD0DFF828800127B4FA84F377
:10169000C3F11F0307FA03F558F8230003689847BE
:1016A000AC437561F2D1BDE8F08100BF0004014098
:1016B0004C5800202DE9F0410B4E346873691C40F2
:1016C0000FD0DFF828800127B4FA84F3C3F11F0399
:1016D00007FA03F558F8230003689847AC4375618F
:1016E000F2D1BDE8F08100BF000401404C58002059
:1016F000084A094808B5936943F001039361002142
:10170000402221F0A6F9054B4FF0FF321A60C3F8D2
:10171000032008BD001002404C5800208C580020C7
:1017200003685B6A184700BF2DE9F041044618467C
:101730000D46164698461FF023F92768E67228449E
:10174000A07229467D69434632462046AC46BDE834
:10175000F0416047036810B504461B68984723684A
:1017600020469B689847A37B0133A37310BD00BF3D
:1017700010B5036804469B689847FF2301226373F2
:10178000227310BD064B984202D04FF0FF307047D5
:10179000044A538B01339BB25383508B80B2704702
:1017A000003800408464002038B58368044615463C
:1017B00013B11A689B881385606840F2E93300E032
:1017C0007BB30289013B12F0020F9BB2F8D0017388
:1017D00040F2E93300E023B30289013B12F0010F2C
:1017E0009BB2F8D0037B606840F2E93300E0DBB1E4
:1017F0000189013B11F0020F9BB2F8D0057340F252
:10180000E93300E083B10289013B12F0010F9BB282
:10181000F8D0037BA36813B11A689B8893610120F9
:1018200038BDFFF7AFFFDEE7FFF7ACFFF2E700BF21
:10183000F0B50D460178012983B00446164618D04C
:10184000022902D0002003B0F0BD80681F46FFF7D8
:1018500019FE45F080016068EFF770FE3B463246A6
:1018600000216068EFF7BAFDA068FFF711FE0120C4
:10187000E9E790F90400421CE4D00228E2DC617937
:1018800000962A46F0F75EFBDDE700BF427A02B918
:10189000704710B504460368406804F10A01984790
:1018A0000023637210BD00BF437A5A1C0344D2B2B6
:1018B00042729972037A934200D802B9704710B508
:1018C00004460368406804F10A01984700236372E4
:1018D00010BD00BF98B10B4B012210B402FA01F108
:1018E00003F1750402E00333A34209D01A7882425F
:1018F000F9D15A780A42F6D001205DF8044B7047BE
:101900000020FAE70C33030830B40A4D002305F138
:10191000140401E0272B09D003EB43020133A15C3F
:101920008142F7D12A4430BC907D7047002030BC02
:10193000704700BFF83203082DE9F34105690646F8
:101940000F467DBBD0F80080C8F30A0323B3002301
:10195000D6F80080019314F0DFFF042819D1224C3F
:10196000236943F001032361BBB2A8F8003014F0EF
:10197000D3FF04282ED108F102030193019B3F0CF1
:101980001F8014F0C9FF2369042823F00103236199
:1019900025D06FF0010505E014F0BEFF042805D046
:1019A0004FF0FF35284602B0BDE8F0810E4C2369A8
:1019B00043F002032361C4F81480236943F0400319
:1019C000236114F0A9FF2369042823F00203236193
:1019D000BDD0E5E7236923F001032361D9E733682C
:1019E00004333360DEE700BF00200240F8B5044650
:1019F0000D468E180027B54201D12069F8BDE36875
:101A0000591CE160234415F8012B1A720429F2D104
:101A1000A1682046FFF790FFE7602061EBE770B513
:101A2000448806460D46C4F30B042246002128468E
:101A300021F00FF833690A4A934209D3094A9342C5
:101A400006D2224628461946BDE870401FF006BF60
:101A500023B121462846BDE87040184770BD00BF3D
:101A6000008D0308EA8D0308064B07498B4202D319
:101A70000023184670471A88C2F30B029042F8D030
:101A80001433F3E7A0880308008D0308024A1368A3
:101A900023EA000010607047B434002008B511F04C
:101AA00003FE024B024ADA60FEE700BF00ED00E0F1
:101AB0000400FA05024A034B1278197812F03ABF73
:101AC000C01D0020C11D00202DE9F04F2DED028B1F
:101AD000A0F10A0389B00C46ED2B00F27286DFE814
:101AE00013F022017006700670067006700670060C
:101AF0007006700670067006700670067006700636
:101B00007006700670067006700670067006700625
:101B100070062F0270067006700636067006700694
:101B2000700699017006560170063E017006330179
:101B300070062802700603027006EF017006700638
:101B40007006EA01E4017006D20170067006CC014D
:101B50007006A5017006700670068A04700670068D
:101B6000700670066C0470060201700645063205A8
:101B70007006700670067006700670067006060520
:101B80007006D8047006A50470066F0570065C0622
:101B900070067006700670060503FB05F405C305A4
:101BA000EE00700670062803A60270066F02E902B6
:101BB0007006700670067006DE0270067006BD02C2
:101BC000700670067006AF02F303BB037A0370065B
:101BD000700670066C03700670064C037006700683
:101BE0007006700670067006700670067006700645
:101BF00070067006700670067006050370067006A3
